:10000000A0390020C11C0000191D00007D17000050
:100010007D1700007D1700007D1700007D17000090
:100020007D1700007D1700007D17000041170000BC
:100030007D1700007D170000FD1600007D170000F1
:10004000A517000073A80000A5170000A517000061
:10005000A5170000A5170000A5170000A5170000B0
:10006000A5170000A5170000A5170000A5170000A0
:10007000A5170000A5170000A5170000A517000090
:10008000A5170000A5170000A5170000A517000080
:10009000A5170000A5170000A5170000A517000070
:1000A000A5170000A5170000A5170000A517000060
:1000B000A5170000A5170000A5170000A517000050
:1000C000A5170000A5170000A5170000A517000040
:1000D000A5170000A5170000A5170000A517000030
:1000E000A5170000A5170000A5170000A517000020
:1000F000A5170000A5170000A5170000A517000010
:100100007BB972B90029BEBF00204FF0004106E064
:1001100008BF00281CBF6FF000414FF0FF3000F017
:10012000BDB9ADF1080C6DE904CE002909DB002B47
:100130001ADB00F04DF8DDF804E0DDE9022304B03D
:100140007047404261EB4101002B1BDB00F040F89F
:10015000DDF804E0DDE9022304B0404261EB410137
:10016000524263EB43037047524263EB430300F098
:100170002FF8DDF804E0DDE9022304B0404261EB32
:1001800041017047524263EB430300F021F8DDF870
:1001900004E0DDE9022304B0524263EB43037047FD
:1001A00053B94AB9002908BF00281CBF4FF0FF31DE
:1001B0004FF0FF3000F072B9ADF1080C6DE904CEDC
:1001C00000F006F8DDF804E0DDE9022304B0704732
:1001D0002DE9F047089E04468846002B4BD18A4201
:1001E000154667D9B2FA82F24AB1C2F1200701FA84
:1001F00002F320FA07F7954047EA030894404FEAD4
:10020000154E230CB8FBFEF71FFA85FC0EFB178872
:1002100043EA084307FB0CF1994209D9EB1807F1AF
:10022000FF3080F01B81994240F21881023F2B443D
:100230005B1AA4B2B3FBFEF00EFB103344EA034496
:1002400000FB0CFCA44509D92C1900F1FF3380F008
:100250000781A44540F2048102382C4440EA07405B
:10026000A4EB0C0400271EB1D4400023C6E90043D0
:100270003946BDE8F0878B4209D9002E00F0EB80AB
:100280000027C6E9000138463946BDE8F087B3FAD1
:1002900083F7002F47D18B4202D3824200F2FA80CB
:1002A000841A61EB030301209846002EE0D0C6E9D2
:1002B0000048DDE702B9FFDEB2FA82F2002A40F020
:1002C0008F80491B4FEA154E1FFA85F80127B1FBB5
:1002D000FEFC230C0EFB1C1143EA014308FB0CF14E
:1002E000994207D9EB180CF1FF3002D2994200F283
:1002F000CD808446591AA3B2B1FBFEF00EFB101458
:1003000043EA044408FB00F8A04507D92C1900F182
:10031000FF3302D2A04500F2B6801846A4EB0804D1
:1003200040EA0C409FE7C7F1200CBB4022FA0CFECC
:100330004EEA030E01FA07F420FA0CF521FA0CF349
:100340004FEA1E482543B3FBF8F92C0C08FB193380
:100350001FFA8EFA44EA034309FB0AF49C4202FAAC
:1003600007F200FA07F10BD91EEB030309F1FF3086
:1003700080F087809C4240F28480A9F10209734496
:100380001B1BADB2B3FBF8F008FB103345EA034486
:1003900000FB0AFAA24508D91EEB040400F1FF3362
:1003A0006BD2A24569D90238744440EA0940A0FBE7
:1003B0000289A4EB0A044C45C2464B4654D351D0A3
:1003C000002E69D0B1EB0A0564EB030404FA0CFCBF
:1003D000FD40FC404CEA0505C6E90054002747E70C
:1003E000C2F1200320FA03F7954001FA02F021FA46
:1003F00003F34FEA154E3843010CB3FBFEF71FFA27
:1004000085F80EFB173341EA034107FB08F38B42E3
:1004100004FA02F407D9691807F1FF3C2FD28B4286
:100420002DD9023F2944CB1A81B2B3FBFEF00EFB5B
:10043000103341EA034100FB08F38B4207D96918E6
:1004400000F1FF3C17D28B4215D902382944C91A52
:1004500040EA07473BE73746304609E70746E7E605
:100460001846FBE64145ABD2B8EB020A69EB0E0237
:1004700001381346A4E76046E9E7184695E7674662
:10048000D1E781467CE702382C4447E7ACF1020C07
:100490002B442FE7384608E73746E9E6704700BFA8
:1004A00043685B68184743681B6A03B11847704785
:1004B0004368DB6A03B118477047000038B5084C41
:1004C0004FF0FF3120460EF0B7FA054601F0A8FDC7
:1004D00010B128460EF0D6FA0FF0EAFFF0E700BFA1
:1004E000DC47002010B50F480F4C0FF059FB20607F
:1004F00098B1FFF7DDFF2068FFF7D5FF226853684A
:1005000023B19B6C13B10949104698472068436892
:100510009B6A2BB19847002010BD6FF01500FBE7D8
:100520001846F9E7F61001000400002065050000F8
:100530002DE9F04107460E4615469846002425B1A0
:100540007B689B6923B94445F9D32046BDE8F08117
:100550002A463146384698470028F4D02D1A0444DC
:100560000644ECE72DE9F0414E4D4F4C8AB02F4642
:10057000286843685B6C7BB1984768B1286843681A
:100580001B6C4BB1984738B1286843685B6B33B933
:10059000386843685B6A83BB0AB0BDE8F08198475E
:1005A0000028F5D02668002E4FD1334601220DF1E8
:1005B00003012868FFF7BCFF0128D9D19DF803305B
:1005C000012B1CD0022BE7D104230DEB03011A46AB
:1005D0003868FFF7ADFF002134480EF027FA0646D1
:1005E00038B10223042203750DEB020108300EF02E
:1005F0007DFABDF80630236017E09847CCE7032367
:100600001A4601A92868FFF793FF9DF8063028488D
:10061000236031460EF00AFA064630B10023037516
:10062000032201A908300EF061FA224B1E60214E10
:10063000306850B108300EF072FA2368984204D244
:1006400030680EF01FFA00233360DFF868803868E6
:10065000D8F8003022686BB943689B69212A28BF0B
:1006600021222BB101A9984723681B1A23607FE739
:100670001846F9E79E68998900233144FFF758FF2F
:10068000D8F8001026688B89361A03448B812660BF
:10069000002E7FF46DAF08480EF0E7F9C8F800604F
:1006A00066E700BF0400002008000020EC4700209F
:1006B0000C48002000000020DC470020F8B505466B
:1006C0000F464FF02002EFF3118382F31188234C81
:1006D0002068FFF7EDFE2068FFF7E5FE002D36D11C
:1006E0002E4604212068FFF7DBFEFF212068FFF77C
:1006F000D7FEB11DC9B22068FFF7D2FEAA2120683B
:10070000FFF7CEFE36B1013D15F8011F206809BB89
:10071000FFF7C6FEF9B22068FFF7C2FEC7F3072154
:100720002068FFF7BDFEC7F307412068FFF7B8FE5A
:10073000390E2068FFF7B4FEFEE701332F2A08BF09
:100740001E46EA5C002AF8D135449E1BC9E7002604
:100750003346F6E7FFF7A4FED6E700BF040000200B
:100760002DE9F0411C481C4E1C4D86B001F05EFC8A
:1007700000236FF00802CDE90232CDE90433CDE960
:1007800000334FF42072164B164917480FF09AFFAA
:100790004FF0FF3130460EF04FF9037D012B044638
:1007A0000DD0032B08D102212868FFF779FE04F150
:1007B0000807A3892BB920460EF064F9E8E7042165
:1007C000F2E73846D5F800800EF0A1F90146404620
:1007D000FFF766FEEDE700BFCC47002004000020D5
:1007E000BD040000E82D00200C00002008B50446E0
:1007F000084611461A46A0470FF084FE01F03CFA65
:1008000010B504464FF0FF3120460FF009FC0346B7
:100810000028F7D008334268BFF35B8F53E8001F0E
:1008200021F0010C43E800CEBEF1000FF6D1BFF37A
:100830005B8FCB0700D590470FF03AFEE2E770B52B
:10084000C66890F90B000C254D43884206EB050461
:10085000B4BF71592146202492FBF4F401EB8401CA
:10086000196002F01F0070BD07B501ABFFF7E7FF8D
:10087000019A012303FA00F013680343136003B0E5
:100880005DF804FB07B501ABFFF7D9FF019A01231F
:1008900003FA00F0136823EA0003136003B05DF865
:1008A00004FB10F0010005D04FF02003EFF311809E
:1008B00083F3118870472DE9F8430446436805899E
:1008C000006894F80AC05D43FF222844E2720021C8
:1008D0004FF00C0E8C4505DC00252389AB4222DC51
:1008E000BDE8F883D4F80C80B5FBF3F20EFB01F7FA
:1008F0001F2A08EB0706C8BF1F324FEA930306F111
:100900000409C8BF520903F10303C6E9019923F0A2
:100910000303D4BFE17248F8070001F10101C8BF29
:1009200000EB8200D6E76268E36820686A438118BA
:100930001E1D86509A684A609A6820461160996028
:100940002A460021FFF790FF0135C6E72DE9F04F59
:100950008BB0867A00AFC7E90232B3000A3303F4E2
:10096000FF63ADEB030D4368E94603334A4623F0CA
:10097000030342F8043904464FF0FF3500234FF0DB
:100980000C0C581E9E42786209DD2BB1106880085D
:10099000033020F003005060506888420BD27B6A1D
:1009A000013314D13A6D002313606FF00B002C3724
:1009B000BD46BDE8F08FE0680CFB030000F1040EBB
:1009C00040680432704518BF1D460133D9E76E1CDC
:1009D000E8D0207CFFF765FF0C236B431A1DE3680A
:1009E000386213441E68B34277D0D6E90013196009
:1009F000316859F825204B6023682946F31A2046B0
:100A000093FBF2F2FFF73EFFA9EB890305F1010B1F
:100A10003B6109EB85057A6A0BF1FF339A4216DCDC
:100A2000237CD90702D53B6A83F31188FB681A46F9
:100A30007B6A136023687A6AF31A59F8222093FBC1
:100A4000F2F3BA6813603B6D00201E60AFE72368C5
:100A500055F8042BF31A93FBF2F33A699B00BB6140
:100A600005EB450313447B614FF0010AD5F8008084
:100A70000AFB08F3FB61F3187B60BB6959460AEB7C
:100A800003022046FFF7F0FE7B682268218908F107
:100A9000FF389844A8EB020862684A4390450AD29E
:100AA000E2687969F8690A44111D3150916859600A
:100AB00091680B6093600AF1010ABAF1040FD5D175
:100AC000237CD80702D53B6A83F31188207CFFF78B
:100AD000E8FE0BF1010B38629DE7013D6A1CA6F1AF
:100AE0000C037FF47FAF00269AE72DE9F04F87B023
:100AF000837A9B000A3303F4FF6300AFADEB030D71
:100B00004368E946033323F003030446C9F8003081
:100B10004D46012081426ED2207C0D461646FFF7DD
:100B2000C0FE804659F82530FB6003FB06FB2368B6
:100B3000BB6032462946204603EB0B0AFFF794FEC2
:100B4000E2680C2303FB0522BB68111D43F80B1060
:100B50009368CAF804309368C3F800A0C2F808A0EC
:100B6000237CDA0701D588F31188207CFFF799FEF2
:100B70008046002D48D007F114033246294620460E
:100B8000FFF75DFE7A69042390FBF3F083001068A1
:100B9000D84000F00F000F2836D126F00303BB60C9
:100BA000FB684FF0000A013BBA68F968B4F808C066
:100BB000524401FB02FB616803EB0B0001FB0CF1EB
:100BC00088420FD2294620467B60FFF75BFE2268F1
:100BD0007B6852F80B0002EB0B014968086052F881
:100BE0000B2051600AF1010ABAF1040FDCD196FB27
:100BF000FAF6013D96E72B689B08033323F00303C5
:100C000045F8043F013085E7237CDB0701D588F3F5
:100C100011881C37BD46BDE8F08F002070470000EA
:100C20000B6801330B60014B1B681847E044002040
:100C30002DE9F04F85B09B460E9CDFF890A0012C6B
:100C4000B8BF0124012B0CBF30232023154680465A
:100C500089460194029301260A2700220AF1010421
:100C60000AB9AA451FD2B5FBF4F049463030C04757
:100C700001360122013F012FB5FBF4F14FF00A03C9
:100C800004FB1155BAFBF3FAE8D1494605F13000EF
:100C9000C047BBF1030F03D1019B9C1B002C0FDC51
:100CA00005B0BDE8F08F019BBB42E3DBBBF1020F57
:100CB000E0D84946029803920136C047039AD9E723
:100CC00049462020C047013CE8E700BFFFC99A3BE6
:100CD00030B58A680C68551C14B14B68934201DC2E
:100CE0008D6030BD013B934208BF00228D600CBF78
:100CF000E254A054F5E70000014B1860704700BFB4
:100D0000E04400202DE9F04F89B01C464FF0000A66
:100D1000531E06460F4604934FF0FF39D046002578
:100D200005E06DB9252800F012813946B047049BD3
:100D300013F8010F04930028F3D109B0BDE8F08F38
:100D4000642861D019D839280AD8312850D22D28E2
:100D50003CD030283DD0252808D13946B047DEE7C1
:100D6000582800F08880632800F0EB803946252061
:100D7000B047049B39461878F0E7702871D006D840
:100D8000692841D06C283CD06828D0D0EEE775287F
:100D900057D017D87328E9D1236804F1040B1C46F7
:100DA000254615F8010B002840F0C080B8F1030F6C
:100DB00040F0D680E41AA9EB0404002C00F3BC80B8
:100DC0005C46ACE7782856D07A28DEE74FF0030877
:100DD000ADE7B9F1000F0EDAB8F1000F00F0BD80F9
:100DE000A0F13009B8F1000F08BF4FF002089EE7EC
:100DF000B9F1000FF4DB0A2303FB0909A9F130095B
:100E0000F0E70AF1010A92E7BAF1010FC5BF073412
:100E100024F0070325681D68D4BF043403F10804D7
:100E2000002D05DA39462D20B0476D4209F1FF3912
:100E3000CDF8009043462A4639463046FFF7F8FE83
:100E40006DE7BAF1010FC5BF073424F0070322682C
:100E50001A68CDF80090CCBF03F10804043443466F
:100E6000EAE739463020B04739467820B0474FF09E
:100E700008094FF00108BAF1010FC7BF073424F089
:100E8000070323680593C2BF03F108041B68059399
:100E90004FF008024FF00003D8BF043403930793C8
:100EA00093460BF1FF3B059B4FEA8B0023FA00F0C2
:100EB00010F00F0009D1079B13B9BBF1000F24D12B
:100EC0004FF0300C07E0069AEBE709288CBF4FF093
:100ED000570C4FF0300C394660440692B047039BE4
:100EE000079501330393BBF1000FECD1B8F1030F69
:100EF0007FF415AF039BC3EB4905002D7FF70FAFC0
:100F000039462020B047013DF7E7531E914506932F
:100F1000E9DBB8F1010F03D139463020B047E2E7F1
:100F2000B8F1020FDFD139462020F7E739460393A5
:100F30002C46B047039B33E739462020B047013C9D
:100F40003BE72068251D3946B0472C46E7E6AA4610
:100F5000A8464FF0FF390125E9E64FF00108E6E623
:100F60005C460546E3E6000013B502AC002344F8F6
:100F7000043D02460B4603482146FFF7C3FE02B07C
:100F800010BD00BF210C00000FB407B504A951F833
:100F9000040B0191FFF7E8FF03B05DF804EB04B028
:100FA000704700000CB430B585B008ABCDE9010145
:100FB00053F8042B00930446002501A90648039525
:100FC000FFF7A0FEDDE902309842B8BF255405B016
:100FD000BDE8304002B07047D10C000070470000FF
:100FE00010B54FF02003EFF3118483F3118800F064
:100FF00025F8084A0123C2F840354FF08042C2F874
:101000007835054B4FF0FF329A62DA6284F311882B
:10101000002010BD00E0014000ED00E0054B1B6822
:10102000082B01BF044B1868B0FA80F0400918BFC4
:1010300000207047300100103401001008B54FF057
:1010400080430022C3F80C21C3F81021C3F83825CF
:101050004FF0805203F54043D2F80414C3F8201532
:10106000D2F80814C3F82415D2F80C14C3F82815C4
:10107000D2F81014C3F82C15D2F81414C3F8301594
:10108000D2F81814C3F83415D2F81C14C3F840155C
:10109000D2F82014C3F84415D2F82414C3F8481524
:1010A000D2F82814C3F84C15D2F82C14C3F85015F4
:1010B000D2F83014C3F85415D2F83414C3F86015BC
:1010C000D2F83814C3F86415D2F83C14C3F8681584
:1010D000D2F84014C3F86C15D2F84424C3F8702534
:1010E000FFF79CFF10B1334B334A1A60FFF796FFAE
:1010F00018B1324BFB22C3F81825FFF78FFF48B118
:101100002F49304B0A681B6822F00F0203F00F03CF
:1011100013430B60FFF782FF18B12B4B4FF40072A3
:101120001A604FF08043D3F80024D20744BF6FF019
:101130000102C3F800244FF01023D3F80022002A44
:1011400003DBD3F80432002B2FDA204B0122C3F843
:101150000425D3F80024002AFBD04FF010221221DE
:10116000C2F80012D3F80024002AFBD04FF010235D
:101170001222C3F80422154B1A46D3F80014002992
:10118000FBD00021C3F80415D2F80034002BFBD0AB
:10119000BFF34F8F0E490F4BCA6802F4E06213434E
:1011A000CB60BFF34F8F00BFFDE70B4B0B4A1A60BC
:1011B00008BD00BF8C5600404881030000F000408D
:1011C000E40E0040580200104096024000E001404A
:1011D00000ED00E00400FA05E44400200090D00394
:1011E00013B5114CBFF35B8F2068BFF35B8F60B901
:1011F0000E480EF0D5FCBFF35B8F54E8003F44E887
:101200000002002AF9D1BFF35B8F436804221B68F8
:101210000DEB02019847002802DA00F04DFA019028
:10122000019802B010BD00BF780000205B110100E2
:101230000A2838B50446074D04D1286843680D21B3
:101240005B68984728684368E1B25B689847204626
:1012500038BD00BF7C00002010B5044C204600F0D3
:1012600017FE2046BDE81040FFF746BD31120000D2
:1012700008B504480EF094FC034B1860FFF7ECFF30
:10128000002008BD651101007C00002010B54FF062
:101290002003EFF3118283F31188114C237823B9D3
:1012A00082F311886FF0440010BD013BDBB2237064
:1012B00023B182F311886FF00F00F5E7094B18781E
:1012C000012128B1217082F311886FF00A00EBE749
:1012D000197082F31188044A11601870E4E700BFA6
:1012E00082000020810000200400004008B5002298
:1012F0001046012100F00CFC002000F0D7FB00207C
:1013000008BD0000F8B54FF02002EFF3118382F31F
:101310001188264A1078441C147070B183F3118828
:101320004FF08043D3F80C3403F00113B3F1011FE5
:101330000CBF00206FF0430007E01D4D2F782FB148
:10134000107083F311886FF00A00F8BD01262E702B
:1013500083F311884FF0804419B3384600F0B6FB90
:10136000C4F80071D4F80433C4F804632660D4F8D8
:10137000002192B10022C4F800210E4A13F0010F9F
:101380004FF0010308BFC4F808330020C2F88031D1
:1013900000F08CFB00232B70C2E720BF40BF20BFB2
:1013A000E5E7C4F800112660F4E700BF82000020E2
:1013B0008100002000E100E070B54FF02002EFF363
:1013C000118382F31188224D2A788AB183F3118820
:1013D0004FF08042D2F81C34D2F8182403F00303F3
:1013E00043F48033934314BF6FF04300002070BD7B
:1013F00001242C7083F311884FF08043154EC3F8FD
:1014000004210225C3F81815C3F8045311F0030191
:1014100034604FF01806C3F80863C3F80C21C3F812
:101420001021D5D11022C3F83825C3F80463D3F8AE
:101430001824D20302D4C3F80453C9E7C3F8044301
:10144000FFF760FF0028C3D1034BC3F80041BFE79B
:10145000800000200800004000E100E0F8B54FF0F7
:1014600080430546D3F808C1D3F80423D3F80071AC
:10147000D3F80403D3F80461D3F80C11D3F8104166
:10148000003402F0010218BF0124BCF1000F03D0A8
:101490004FF0000CC3F808C1002F41D04FF080433B
:1014A0000027C3F8007152B14FF08043224F012250
:1014B0004FF0020CC3F80823C7F800C01A61EEB958
:1014C00059B11D4B4FF08046002119602846C6F8DF
:1014D0000C11FFF7DBFE0123736174B14FF0804301
:1014E00000210124C3F810112846C3F80443FFF774
:1014F00009FF10B9114BC3F80041F8BD4FF080430C
:101500000022C3F804218207DAD50222C3F8082397
:10151000D3F81C349B07D3D10029DFD00124D0E7B6
:10152000002ACCD04FF08043D3F80C3403F00113E1
:10153000B3F1011FC3D1B7E7340C004000E100E074
:1015400070474FF02003EFF3118083F31188704749
:101550000D4A002310B5C2F84031FFF7F2FF0B49E6
:10156000D2F804350C6840F247121B1B23F07F436E
:10157000B3FBF2F302FB03420A6080F311881846C2
:10158000BDE810400FF0A8BA001001408400002010
:1015900037B51F480EF004FB002835D043681D4DB9
:1015A0001B6801219847002440F24713C5F80845FD
:1015B000C5F840354FF48033C5F84433C5F80433DB
:1015C00003F1804303F58A534FF400321C601B681B
:1015D0000193019B104B0121C3F880211120224669
:1015E00000F096FA112000F061FA0C4A0123136012
:1015F0002B60D5F8043503F2471323F07F43C5F879
:101600004035204603B030BD4FF0FF30FAE700BF51
:10161000841101000010014000E100E008100140C9
:1016200070B54CF66905B0F1FF3F14BF02462A467B
:10163000134CFFF786FF134BD4F804151E68531E96
:10164000AB42A1EB0602A8BF2B4622F07F4240F23C
:10165000471502F5A37223EAE37305FB0323B3FBEB
:10166000F5F305FB0363591A21F07F411F2998BF49
:101670005B1923F07F43C4F8403580F3118870BDB7
:10168000001001408400002008B5FFF75AFF084B06
:10169000084AD3F8043512689B1A23F07F4340F2BE
:1016A0004712B3FBF2F380F31188184608BD00BF60
:1016B000001001408400002008B5FFF742FF064BF0
:1016C000064AD3F80435126880F31188981A20F07E
:1016D0007F40104408BD00BF00100140840000207E
:1016E00004488168406A884203D003494FF0805221
:1016F0000A607047382D002004ED00E0202080F3C0
:1017000011880D498A684FF028001044EFF3098CC6
:1017100080E8F01F094F4FF000664A6A8A603E6019
:10172000506E0023536680F3118802F1280090E880
:10173000F01F8CF309887047382D002004ED00E07D
:101740001EF0040F0CBFEFF30880EFF309808169EE
:1017500031F8021C11F0FF010229FFD000B500F0A2
:101760005BFA00BD014910220A60704710ED00E0ED
:10177000404080F3118830BF704700BF404080F385
:101780001188DFF81CC0DCF800C01CF4006C0CBF32
:10179000EFF30880EFF3098000B500F019F900BD00
:1017A00004ED00E000B572B60B4A106A00281EBFB7
:1017B000002111620EF01CFA62B6EFF30580A0F171
:1017C00010004FEAC0000549014409C998475DF877
:1017D00004EB034800470000382D00209C0E010058
:1017E000E1160000044800232021C2180133302BE9
:1017F00082F80013F9D1704700E100E0084A094976
:10180000936809689966084958664B6843F08053A5
:101810004B60002383F311889368986E704700BF74
:10182000382D0020701C010000ED00E038B5194C87
:1018300005461948FFF7A8FBA36AD90602D5174841
:10184000FFF7A2FBA36A1A0702D51548FFF79CFB16
:10185000A36A9B070ED51348FFF796FB616BA36A3B
:10186000180607D51048FFF78FFB1DB1A36A23F0B8
:101870008003A362074CA26AD20702D50B48FFF788
:1018800083FBA36A9B0602D50948FFF77DFB002076
:1018900038BD00BF00ED00E0F31201000A130100A3
:1018A0001C130100301301004913010060130100F3
:1018B0008013010038B51B4C05461B48FFF764FB3D
:1018C000A36AD80404D51948FFF75EFB002038BD91
:1018D000A36A190501D51648F6E7A36A9A0514D537
:1018E0001448FFF751FBA16BA36A1B0407D51248EC
:1018F000FFF74AFB1DB1A36A23F40043A362094B1F
:101900009B6A5805E2D50D48DEE7A36A5905FAD46B
:10191000A36ADA0501D50A48D6E7A36A9B04D5D5A0
:101920000848D1E700ED00E0A41101000A1301000E
:101930001C130100BB110100D5110100EB110100C6
:10194000071201008013010010B5194C1948FFF768
:101950001BFBA36A9A0102D51748FFF715FBA36A80
:10196000DB0102D51548FFF70FFBA36A180302D568
:101970001348FFF709FB0E4CA36A590302D511481F
:10198000FFF702FBA36A9A0302D50F48FFF7FCFAA0
:10199000A36ADB0302D50D48FFF7F6FA044A936AFF
:1019A0006FEA03436FEA13439362002010BD00BF48
:1019B00000ED00E0B0130100C9130100DD130100C8
:1019C000F8130100171401003D1401005814010020
:1019D00038B5274C6368C3F30803DA1E0546092AA5
:1019E0003AD8DFE802F0053335303939393939373B
:1019F0002048FFF7C9FAE36A9A0703D51E48FFF7A4
:101A0000C3FA02E0E36A5B0005D400202946BDE882
:101A1000384000F0CFB81948FFF7B6FA184B1B78DA
:101A20002BB10120FFF702FF0628EFD138BD154B7F
:101A30001B781BB10120FFF73DFFF5E7124B1B8818
:101A40009BB2002BE1D0FFF77FFFEDE70020E9E735
:101A50000020F0E70D48D2E70D480E49A3F110022F
:101A60000F2BD8BF01460C48FFF78EFACDE700BF19
:101A700000ED00E04E120100661201008812010024
:101A800028ED00E029ED00E02AED00E0A8120100B9
:101A90002012010035120100DF120100024A5369D1
:101AA00043F010035361704700ED00E043B2002B98
:101AB00008DB012200F01F0002FA00F05B09024A75
:101AC00042F82300704700BF00E100E043B2002B62
:101AD0000DDB01225B0900F01F0002FA00F0203349
:101AE000034A42F82300BFF34F8FBFF36F8F704755
:101AF00000E100E04209054B00F01F0053F82220EE
:101B0000012303FA00F01040704700BF00E100E03D
:101B100043B2002BA8BF03F1604301F101014FEA7A
:101B20004111AEBF03F5614300F00F00034BC9B292
:101B3000ACBF83F800131954704700BF14ED00E0E8
:101B4000FFF71CBE08B572B6044B186A18B1002224
:101B50001A620EF04DF862B608BD00BF382D0020A5
:101B600070470000F8B50C4616461F4604220A9B33
:101B7000099905460EF034FEA6F1200121440C4AD5
:101B800021F00701002322F00102C5E91333C5E962
:101B900016468A61069A4A60079A8A60089ACA605D
:101BA0004FF080720F60CA61A9646B66F8BD00BF18
:101BB000ED07000038B504460D4605281AD8DFE8C1
:101BC00000F00319191315170D48FFF7DDF90EF092
:101BD00099FCAA6901460B48FFF7D6F92946204629
:101BE000BDE8384000F01CB80748EEE70748ECE7CE
:101BF0000748EAE701460748FFF7C6F9E7E700BFED
:101C00008414010022150100A4140100CA1401006B
:101C1000E4140100FF14010001460068FFF7CABF89
:101C2000052810B50CD00EF003FD60B10EF000FDDC
:101C30000C490D4B002808BF19460C48FFF7A4F9C2
:101C4000FFF796FDFCE70EF003FD0028EED1084CEF
:101C50000848A168FFF798F9A068BDE8104000F0B7
:101C60000BB800BF5E15010062150100731501007D
:101C7000382D00209315010038B505464FF020039C
:101C8000EFF3118483F311880EF03CFD0A4B9B683F
:101C9000AB420BD1094B5A68C2F3080212B9204675
:101CA000FFF7ACFD5A6842F080525A602046BDE80A
:101CB00038400EF0D9BA00BF382D002000ED00E00A
:101CC000202080F3118806484FF40061401880F30B
:101CD0000988022080F31488BFF36F8F00F006F8A4
:101CE000E03A002030BFFFF7FDBF00BF08B5084B4A
:101CF000084A23F07F039360BFF34F8FBFF36F8FCA
:101D00000DF090FF0DF098FFFFF76CFD0DF0B8FFA0
:101D10000000000000ED00E008B5FFF7E3FFBDE8BC
:101D20000840FFF7DDBC0000034B05225A60BFF3FB
:101D30004F8FBFF36F8F704790ED00E0BFF35F8F61
:101D4000014B00225A60704790ED00E0124910B537
:101D50000C68082C1CD8FFF7F1FF104849680022D6
:101D6000944201F10C0103D1FFF7DEFF002010BD0A
:101D7000826051F80C3C23F01F0343F0100313431F
:101D8000C36051F8043C43F0010303610132E7E70B
:101D90004FF0FF30EBE700BF2C11010090ED00E0A9
:101DA0000139034611F8012F0AB91A70704703F878
:101DB000012BF7E70138013910F8013F11F8012F25
:101DC000934202D1002BF7D11A46981A704710B5EA
:101DD0005AB10139841810F8012B11F8013FA042C3
:101DE00001D09A42F7D0D01A10BD1046FCE7F0B5EA
:101DF00081EA0004A50703460BD0013B0A44914247
:101E00001DD1F0BD002AFCD011F8014B03F8014BA5
:101E1000013A9C07F6D11D1F0C468F183E1B032E5E
:101E200008D894086FF0030505FB0422A40023449E
:101E30002144E2E754F8046B45F8046FEEE711F82B
:101E4000014B03F8014FDAE7F0B5C9B203469C072E
:101E50000FD141EA012444EA04441D469F187E1B29
:101E6000032E0CD8940803EB840413449C4209D13C
:101E7000F0BD002AFCD003F8011B013AE7E745F862
:101E8000044BECE704F8011BF0E74FF0FF3070471C
:101E9000014B1860704700BFE84400202DE9F8436B
:101EA0001D48DFF880800DF07BFE06461B480DF0D4
:101EB00077FE0024054654F8087073683A46D3F854
:101EC0000090002101233046C847726808EB0403E4
:101ED000D2F804905B683A46002130460834C8477F
:101EE000282CE8D10E4F0024E6596B683246D3F80F
:101EF0000080002101232846C0476A683B19D2F8B8
:101F000004805B683246002128460834C047402CD4
:101F1000EAD10020BDE8F883B8150100BF15010023
:101F2000F0150100C815010030B585B0044615460E
:101F300068460322FFF75BFF0D2200210DF103002D
:101F4000FFF782FF20466A4669460AF03DFB0446D9
:101F500020B9032269462846FFF749FF204605B00D
:101F600030BD13B50C4601AA0331FFF7DDFF48B9B8
:101F7000032201A92046FFF72AFFB0FA80F04009AA
:101F800002B010BD0020FBE770B5CD1C06460C4624
:101F9000284603210AF0FEFA60B9637903F03F0393
:101FA00043F040036371224629463046BDE8704045
:101FB000FFF7BABF70BD0000074A136833B9C168A4
:101FC00039B1016929B11060184670476FF04400BB
:101FD00070476FF015007047F82B002010B50446CD
:101FE00002480CF023FD00B1047510BD2C48002000
:101FF00008B5014603480CF019FD08B1012303752B
:1020000008BD00BF2C48002008B5034B01461868E6
:102010000CF02BFD002008BD88000020FFF7F4BF66
:10202000014B1B681B691847F82B0020044B054A1D
:102030001B6810600BB1DB6818476FF01200704727
:10204000F82B002088000020F7B51860C31D23F08E
:1020500003030E461A80013A94B205460422002179
:1020600006FB0400FFF7F0FE4FF6FF77013CA4B239
:10207000BC4201D103B0F0BD04FB06602B18042262
:10208000801B0DEB020128440193FFF7B0FEEDE742
:1020900073B5046806468CB1E31D23F003030422E4
:1020A00021460DEB02001D88FFF7A1FE019B23B125
:1020B000DA1D22F00302013D15803360204602B094
:1020C00070BD70B50C6806460D461CB1E31D23F0CB
:1020D00003031C88042229463046FFF788FEF21DC0
:1020E00022F00302631C13802E6070BD18B107300C
:1020F00020F003000088704702FB01007047401A7F
:1021000080B2B0FBF2F0704710B5114401384FF6C1
:10211000FF73013A92B29A4200D110BD11F8014DFD
:1021200000F8014FF5E70144884201D100207047D3
:1021300010F8013B002BF7D00120704710600860B9
:10214000704710B51468206014686160106010BD9D
:10215000884203D01AB1436813607047002070476B
:102160000B68834207D00AB1586810600BB11A6837
:102170000A60184670470023FBE700002DE9F0478E
:10218000114FDFF848900426013EF6B2FF2E19D019
:1021900033B24FEA830803EB43031D0104244FF0DD
:1021A0000C0A0AE01AFB04510A1D04EB08003A4429
:1021B000394409EBC000FFF7C1FF013CE4B2FF2C3A
:1021C000F0D1E1E7BDE8F0870C0100208C00002091
:1021D000F0B4124B05460F460C26302472B1614311
:1021E00006FB00142344597A187A814204BF013156
:1021F000197228463946F0BC0CF0D8BA4C4306FB9D
:10220000004423449C7ADA7AA24204D101329A72C1
:10221000F0BC0CF005BBF0BC704700BF0C01002007
:10222000F8B505460E461C468AB10123627820782F
:10223000801A10F0030729D003B3012F39D00132DF
:10224000D2B22270314628460CF0EAFA1CE00CF0BB
:10225000D5FA0028E9D0314628460CF0BBFA002810
:10226000E3D030230C22734302FB0533124A1A4495
:10227000937AD27A9B1A18BF0123D7E70232D2B2DF
:102280002270D4E9020398470020F8BD002BF8D053
:102290000132D2B222700423302212FB06320C2308
:1022A00013FB0523044A60681A442146FFF749FFDF
:1022B000C8E73846E9E700BF0C0100202DE9F04FE0
:1022C00000EB400389B01B014FF00008434E04931C
:1022D00005460424CDF80480013CE4B2FF2C0BD168
:1022E000019B002B72D0B8F1000F6FD142462946F6
:1022F00028460CF05BFA69E00DF1200B00230C2757
:102300004BF8043D4FF0300907FB04F309FB05309F
:1023100031185A46496830580293FFF719FF049B59
:1023200017FB0437F31982460393BAF1000F32D03A
:10233000079B1F785A78BF1A07F00307012F04D1B3
:10234000013A5A70D3E902029047079A13785278FB
:10235000DBB29A1A02F00302012A05930DD0029B08
:10236000039909FB0530304400224068FFF7F8FE6E
:10237000079A059BC2F804A05370029B09FB053322
:10238000F1185A464968F058FFF7E2FE012F8246DD
:10239000CBD1BCB9B0B930220C236A4303FB042271
:1023A0003244917AD07A884213D130226A4303FBB7
:1023B000042333441A7A597A91421CBF5A724FF05F
:1023C000010889E7294628460CF02AFA09B0BDE839
:1023D000F08FD17201220192E7E700BF0C010020CB
:1023E00010B5421E00200139C9B2FF2900D110BD2D
:1023F00012F8013F002BF6D05C1E01302340C0B222
:10240000F8E7F0B5427F0468064613460020FF2A2D
:1024100001D10020F0BD02EB820504EBC5078A4222
:10242000D7F808C014F83550604402D013462A4645
:10243000EDE7934200D175771BB203EB830304F8F9
:1024400033503B78FF2BE5D003EB830304EBC3044D
:10245000A3686344A360DDE730B5551A15F4000F97
:102460008368446909D125F07F421A44A2420ED9FB
:10247000121B00248260446130BD8A1A22F07F4220
:10248000934201D99A1AF1E72244D41A0022A41ADD
:102490000022EFE7034600221A709A6A5962084642
:1024A0000AB1D96A104770472DE9F047857F0123AB
:1024B0000446C3771DB9437FFF2B02D1C577BDE822
:1024C000F0870BF013FC6769667FD4F80080C71BA8
:1024D00027F07F47FF2E06D006EB860608EBC601E5
:1024E0008B689F4218D2A27AE37A934205D10133D6
:1024F000DBB2022B08BF0023E372E37A04EB830311
:102500000122DD60656A0023E377AC46234604219F
:102510000320BDE8F0476047FF1A1D448A784B78D6
:1025200018F836609B1ADBB2012BD3D1D1F80C908E
:10253000013A8A70B9F1000FCCD048696369CA8B3F
:10254000281A184420F07F400B69496AC847C1E740
:102550002DE9F04FC27F93B08346002A40F0B48348
:10256000436904930121837A8177C07A984200F00D
:102570008C800B44DBB2022B08BF00238BF80A309F
:102580000BEB83030191D3F80C80049B434423F0AD
:102590007F43CBF814309BF81D300393DBF80030F9
:1025A0000593DBF804300B939BF80930029300236A
:1025B00007934FF0FF0A029B013BDBB2FF2B029314
:1025C00066D19BF81D30039A9B1A18BF0123029312
:1025D000019BCBB1DBF8009000279BF81D50FF2D2D
:1025E0000BD02EB206EB860609EBC604A368434562
:1025F00040F23281A3EB0803A360DDE901230399D4
:10260000A94218BF13460293DBF800300893DBF8A9
:10261000043010939BF809300193019B013BDBB21E
:10262000FF2B019340F068819BF81D30039A934281
:10263000079B40F037834BB9DBF804309BF8094027
:102640000193013CE4B2FF2C40F09C8200238BF804
:102650001E30029B4BB19BF81D30FF2B40F0E182F6
:102660000BF02AFB08B9CBF818009BF81F30002BA1
:1026700000F02A83DBF824405B460122032104207A
:10268000A44613B0BDE8F04F60470192904682E740
:102690000B9B029A03EBC2077B680693F978BE781E
:1026A0008E4288D0069B387806EB460212019D18B0
:1026B000731CDBB2984208BF0023BB70069B9A5C78
:1026C000032AECD9697801EB81030A930A98059BE8
:1026D00003EBC004052A6378A078A3EB0003DBB208
:1026E0000AD84BB1042A0CD16A6852B9AA6842B917
:1026F000EA6832F07F4204D101212846FFF7CAFE82
:10270000CCE7012B40F09D805846FFF77AFE2B78EE
:10271000A060042B064640F08680DBF81430089356
:102720000BF0E4FA089B0990C31A23F07F4343445B
:102730009E4202469EBF6269921B9B18626896BFCA
:102740006361F31A0023002A49D0A989002946D0E1
:1027500001F1FF3C1FFA8CFCA5F80CC09A42B4F8BA
:102760001EE001D2F44502D3DFF8749231E0616AD1
:10277000994E9A488E19864281BF01F1E87101F5A0
:10278000D43101F5A5716162D4E908168CBF4FF010
:1027900001094FF00009761A91440EF1FF3E66627E
:1027A000A3EB0903A4F81EE0D8E7D4E908160E4409
:1027B00089498A48711881428EBF002101214E4407
:1027C00011440EF1010E8CBF666266620B44A4F8E0
:1027D0001EE0B4F81EE0F445E7D8A4F81CC0AA88AF
:1027E0001344A360EA88636913446361DDE9081256
:1027F0002046FFF731FEA2692B8913446A89A36141
:1028000093428CBF9B1A0023A361AB7B03B1E3709F
:10281000059B0A9A03F832A0637895F801A001336A
:102820006370002169E7A37863706B789BF81C20C4
:102830009A4201BFFF238BF81C300023CBF81830DD
:10284000EFE704215B46DBF8244001220846A0475D
:102850000123BE700793AEE6DBF818209342A8EB85
:1028600003081F4429BFFF23D31A8BF81C30002311
:10287000CBF81830A3691BB18BF81C50CBF818307B
:102880000022A26019F836308BF81D30D4F804C04D
:10289000BCF1000F2CD0A08BDFF840E1D4E9081385
:1028A0000B444D49591871459FBFA3F1E873A3F537
:1028B000D433A3F5A573636292BF019B63620023C7
:1028C000634410F1FF301A44E8D2049BA260DBF8A5
:1028D0001410DA192046FFF7BFFDA38BE383002312
:1028E000E37009F836A0637801336370AA4674E692
:1028F000A37863705546F9E7109B019A03EBC20376
:1029000004935B680A93049B93F80190BAF1FF0F5C
:1029100040D00FFA8AF303EB8303089AD04612F8EB
:1029200033A002EBC3040025DBF800300B93FF2338
:102930002370A28BE38B934240F280809B1A9BB260
:102940000C930FFA88F303EB8303DB001193C8E0C9
:1029500009EB49030A9A1B01D51809F101025FFA34
:1029600082F9049A12784A4508BF4FF000090A9A82
:10297000D35C032B0ED195F80180089B08EB8804EB
:1029800003EBC4046278A3789A4208D00121284658
:10299000FFF780FD049B9B784B45D9D13DE6EB6862
:1029A000DBF8141063602B692362AB8AA383AB69E5
:1029B000A361EB69E3602B6A23610026AB68A36027
:1029C00066616A682046FFF747FD01236662E68379
:1029D000E3704FF0FF0AA7E75A2B17FF592B177F19
:1029E000B6562EFE6068002800F0C780D4E90812B1
:1029F000B24B0A44B249D3188B429CBFA2F1E87291
:102A0000A2F5D432A3688BBF6262A2F5A572002240
:102A10006262034498BF01221344E28BA360013237
:102A2000E283626993424FF0000189BF9B1AD31A77
:102A3000A36061619CBF6361A16052E000237FE7F6
:102A4000B669091A46B9059FB84200D23E1A0993E1
:102A5000059612F83E3053E00693F8E730B200EBEB
:102A6000800002EBC0070E97BF680F97774509D229
:102A70000E9FBF69002F54D10F9EAEEB060E12F8C9
:102A800030604CE0FF264CE0069B98456AD0069BE0
:102A9000FF2BA7D01E4633B203EB83030593059AA1
:102AA0000B9B03EBC207FB8BBA8B934288BF9B1A2D
:102AB0007A688CBF9BB20023002A93D00C9A934271
:102AC00090D8FA78E3789A428CD231465846FFF78C
:102AD00098FCBB787B70059A0B9BB86003F832A01A
:102AE000B246119BDBF80020DBF81800059002EBE2
:102AF000030CFF209BF81D30DCF8081009930690AA
:102B0000FF2B06D003EB830E02EBCE06B0688142AA
:102B100096D8DCF818000D9001EB000E1E46FF2E33
:102B20009CD10D9828B105988142ADD3FF2E40F07D
:102B3000C0800998CCF80810834218BFBDF9240062
:102B40008CF8003016BF00EB80008BF81D8002F877
:102B50003080FF2B06D003EB830302EBC3039A689C
:102B6000511A9960A378013363700021002D3FF45E
:102B7000CDAE2846FFF78EFCC8E60121F6E701231B
:102B8000029359E5019B03EBC4056E686B78EA7804
:102B90009A423FF456AD03EB43031A01B318B25CFB
:102BA000012A24D0022A29D1D3E9019099F80020E2
:102BB000D3F80CE0DBF800C0DBF81410FF2A02D0D9
:102BC00007688F4223D09BF81D2001600021FF2A57
:102BD00009D002EB82080CEBC80ADAF808000144BD
:102BE000DAF81800D0B189F80020CEF800100022E1
:102BF0005A629A6A12B1D96A002090476B782A7893
:102C00000133DBB29A4208BF00236B70BEE702EBD0
:102C10008202DEF800101CF83220D8E71CF83820B9
:102C2000D5E7039BFF2B07D10BF060F804460BF0B0
:102C300035F808B9CBF814409BF81D30DBF80020BC
:102C4000204E03EB830302EBC3030A279D680BF0BE
:102C50004DF8DBF81440031B23F07F430333AB42F2
:102C60002CBFE418641924F07F448046DBF8283038
:102C7000204698470BF03AF8A0EB080020F07F4080
:102C8000A4EB0804033024F07F44A04207F1FF378F
:102C90007FF6EBAC002FDAD140F203413046FDF76E
:102CA0000DFDD4E7002B3FF46AAF00238BF81E30F4
:102CB000D1E4B0457FF4EFAE54E700BF5A2B17FFC5
:102CC000592B177F4016010013B0BDE8F08F00BFED
:102CD000F0B51C4E059F9DF81840DDF81CC02C2552
:102CE000454306EB050E72518EF808108EF8093038
:102CF000CEF80470013BDBB2FF2B13D104BB2C23B5
:102D000058433318089A1A62099A5A6218300A9A74
:102D10009A6232184FF6FF713450918020465C6100
:102D20005C81F0BD1AB207EBC201C1F804C017F80C
:102D3000322002EB4201A41A0CEB011CE4B2D9E7E9
:102D40000120EEE7CC010020074A2C2100FB0123E3
:102D500010B45C6A2CB1A44601220321022010BCED
:102D6000604710BC704700BFCC0100202DE9F04146
:102D7000224C2C2700FB07480DB2D8F8040000EBCA
:102D8000C50C10F835009CF80340661CF6B2B04242
:102D900098BF00269CF80100B0422DD0DCF804005A
:102DA00004EB4404250144194FF0030E00F805E03C
:102DB0006360069BA360079BE360089B23610A9BFB
:102DC000A361BDF82430A3820B9BE3610C9B2362BB
:102DD000022363620D9BA3620E9B6270E3628CF818
:102DE0000360D8E908350846984743460022042185
:102DF000A847606ABDE8F0810120FBE7CC01002014
:102E00002DE9F843224C2C2700FB07490DB2D9F8D5
:102E1000040000EBC50C10F835009CF80340661C5C
:102E2000F6B2B04298BF00269CF80100B0422DD007
:102E3000DCF8040004EB4404250144194FF00408B5
:102E400000F80580A380BDF82030E380BDF8243071
:102E50002381BDF828306381BDF82C30A3819DF813
:102E60003030A373022363620D9BA3620E9B6270DA
:102E7000E3628CF80360D9E90835084698474B4669
:102E800000224146A847606ABDE8F8830120FBE7BD
:102E9000CC0100202DE9F0411A4C2C2600FB0648FD
:102EA0000FB2D8F8040000EBC70C10F837009CF8FC
:102EB0000340651CEDB2A84298BF00259CF80100B4
:102EC000A8421CD0DCF8040004EB440424010719D8
:102ED0004FF0050E00F804E07A700222C7E90923DA
:102EE000069BFB628CF80350D8E9083408469847E3
:102EF000434600220421A047786ABDE8F081012002
:102F0000FBE700BFCC0100202DE9F0411C4C2C2731
:102F100000FB07480DB2D8F8040000EBC50C10F810
:102F200035009CF80340661CF6B2B04298BF0026FC
:102F30009CF80100B04221D0DCF804E004EB44042A
:102F400025010EEB050402200EF80500C4E901235B
:102F5000069BE360079BA362FF25089B6570606288
:102F6000E3628CF80360D8E9083508469847434681
:102F700000220421A847606ABDE8F0810120FBE738
:102F8000CC0100202DE9F0411A4C2C2600FB06480C
:102F90000FB2D8F8040000EBC70C10F837009CF80B
:102FA0000340651CEDB2A84298BF00259CF80100C3
:102FB000A8421CD0DCF8040004EB440424010719E7
:102FC0004FF0010E00F804E0FF2078700220C7E9FE
:102FD0000902FB628CF80350D8E908340846984788
:102FE000434600220421A047786ABDE8F081012011
:102FF000FBE700BFCC0100202DE9F041084C2C2557
:1030000005FB0043D3E9083706460846984706FB08
:103010000543BC4600220421BDE8F041604700BFE3
:10302000CC0100200AF062BE401A20F07F407047B9
:1030300008B50346012B08460ED833B119B1062254
:103040000649FEF7D4FE054807E019B106220449F7
:10305000FEF7CDFE024800E0002008BD2A02002055
:103060002402002070B506460D4606F015FA044607
:1030700010B10C24204670BD06F022FA10F0060FA5
:10308000F7D1062229461EB10248FEF7B0FEF1E74D
:103090000148FAE72A0200202402002000230370DE
:1030A0000B70704720BF40BF20BF7047F0B50D4B7D
:1030B00089B005460E4601AA03F118071868596839
:1030C000144603C40833BB422246F7D11B88238031
:1030D00008AB1D4415F81C0C831B5842584109B01D
:1030E000F0BD00BFDC10010008607047024B18689B
:1030F000436800211B6818473002002018B90B688C
:1031000043F000430B60704718B90B6823F000438D
:103110000B60704770B5031D451E00249D4201D110
:10312000204670BD15F8016F0022A018082AC0B211
:1031300001D10446F2E716F0010F03D00029F0D0C8
:103140000139C9B276080132EFE70000094B93F864
:10315000420193F8412190423BBF93F8412193F8FB
:10316000403193F84131C0182CBFC01A801AC0B248
:10317000704700BF3002002008B50146FFF7E6FFA8
:10318000884223BF044B93F84121D3F83C310020FF
:1031900028BF53F8220008BD3002002030B590F857
:1031A000743090F8751099425CD190F8C04090F856
:1031B000C130A34256D190F91D30002B25DBC48CC1
:1031C000828CA0F87C40C48FA0F87A2054437D22E2
:1031D00062434FF47A7492FBF4F2A0F87E2090F8E8
:1031E0007820012565F30102D2B2002342F00402E7
:1031F000013980F88850C0F8843080F8782080F851
:10320000765080F87510184630BD90F8C230D90657
:103210002AD490F850309A0603D5D0F8A4309B07F2
:1032200022D5C18C828CA0F8C810C18FA0F8C42010
:103230005143A0F8C6207D224A434FF47A7192FB95
:10324000F1F2A0F8CA2090F8C220002302F0F802A0
:1032500063F3C302013C80F8C33080F8C22080F8D9
:10326000C140D0E70120CFE70220CDE708B520B16B
:1032700041F2CA110348FDF721FA034B0022DA7428
:1032800008BD00BF9A1601003002002010B50C46A0
:1032900020B141F2C3110348FDF710FA024BE4B22A
:1032A000DC7410BD9A1601003002002010B50C46E7
:1032B00020B142F67D510548FDF700FA94F85030F0
:1032C0006FF3410384F8503010BD00BF9A1601001F
:1032D0002DE9F843224D95F8424195F8549195F81F
:1032E000403101348145E4B228BF814605F5A47719
:1032F000A34208BF002405F59878B9F1000F03D068
:1033000095F84131A34201D1BDE8F8833846FEF774
:10331000BFFE06460028F7D04046FEF7B9FE28B9A2
:1033200030461049BDE8F843FEF7CBBE066095F87D
:103330004221D5F83C3143F8220085F8424195F806
:1033400040310134E4B2A34208BF002495F854315F
:1033500009F1FF39013B85F854315FFA89F9CCE76F
:10336000300200207803002038B5334C94F8102147
:10337000002A5DD004F586734FF4AA71D4F80801D1
:10338000FEF762FE2D4B94F83A21B4F83811D4F8C8
:103390002C01FEF759FE94F8401194F81021284BA7
:1033A000D4F844010A440821FEF74EFE254BD4F818
:1033B000580102222421FEF747FE94F87421224B83
:1033C000B4F86811D4F86001013A92B2FEF73CFEFD
:1033D0001B48FEF75DFE054620B940F235211B482B
:1033E000FDF76CF91A4A2846111FFEF7A7FE94F85C
:1033F000293043F0380384F829304FF6FF73A4F8DE
:103400001A31A4F81C3142F21F53A4F81E311B23B9
:10341000A4F822314FF4A473A4F824310723A4F8AC
:103420002631A4F82831FF20BDE83840FFF750BF0F
:10343000C4F80C21A6E700BF300200206003002082
:10344000780300208C030020940300209A160100CA
:10345000800300202DE9F84F0C78944281460F46F6
:1034600090463DD01F4ED6F8703133F8343003808B
:1034700000254FF0020B06F5B27A22B2D6F87001A1
:10348000B9F800C000EBC20130F83220944520D1D9
:103490004868012820F003030AD9F3B1021D1CD0AB
:1034A0004279D2B1027902F00302013A012A14D81A
:1034B000012215444A60EDB213B15146FEF701FEF8
:1034C000013496F87421E4B2A24208BF00244445B6
:1034D000D3D13C702846BDE8F88FC1F804B0EBE7C3
:1034E0000025F7E73002002010B5094B93F81021B2
:1034F000824204460AD902464FF4AA71D3F8080161
:10350000FEF7FAFD10B1038CA34200D0002010BDDD
:10351000300200202DE9F04186B00223052805463F
:10352000884602930ED0062800F0A08040F2A280C8
:10353000073880B2FFF7D8FF002800F02581D0E9D6
:1035400000670FE0914BD3E9066702AB00930A4690
:103550008F4B03210020FFF79DFC022879D0029BAE
:10356000002B7AD1894CA37C23B142F26F71894838
:10357000FDF7A4F806AB0222A57443F8102D032131
:1035800000932A46824B0020FFF784FC022879D062
:10359000029B002B40F0EC80237CAB4203D0637C89
:1035A000AB4240F0E18006AB022243F80C2D002232
:1035B00000930321764B1046FFF76CFC02280CD1D8
:1035C000012211460320FEF703FE039B022B04D1C8
:1035D00042F2B3616F48FDF771F8039B002B40F096
:1035E000878002230493237C23B942F2BD6169489A
:1035F000FDF764F804AB002000930122644B2074B3
:103600000321FFF747FC02280CD1012211460320B9
:10361000FEF7DEFD049B022B04D142F2CC615D4833
:10362000FDF74CF8049A002A45D126F00046B7422F
:1036300037D9594B11460320FEF7F2FD002800F060
:10364000938042F2E0615348FDF738F88CE0FFF7D1
:1036500029FD029B022BFAD081E7029B012B81D02E
:1036600042F250714B48FDF729F87BE7474BD3E90D
:10367000346777E742F26A7146480026FDF71EF884
:1036800037466FE7637CAB4204D101221146032029
:10369000FEF79EFD029B022B7FF47AAFFFF702FD3F
:1036A000F8E73E4B11460320FEF7BAFD00285BD039
:1036B00042F2E761C7E7049B012B16D10022364B8B
:1036C00011460320FEF7ACFD20B142F2F061314813
:1036D000FCF7F4FF0022314B11460320FEF7A0FD5A
:1036E000002841D042F2F661ADE742F2F861AAE764
:1036F000039D012D45D1B8F1FF0F23D006AB022267
:1037000043F8042D032100934246214B0020FFF78C
:10371000C1FB02280CD12A4629460320FEF758FD9A
:10372000059B022B04D142F211711A48FCF7C6FF27
:10373000059B3BB1059B012B04D042F21571154846
:10374000FCF7BCFF237D7BB1154B04229A6000225D
:1037500011460320FEF764FD20B142F225710D48A9
:10376000FCF7ACFF237D4BB9A37C0BB9012302937B
:103770000023A374029806B0BDE8F081FFF792FC25
:10378000F0E742F22D715EE70120F4E730020020FD
:10379000E93000009A1601002C450020EC4500207D
:1037A0005C45002010B5C4B2231F012B04D941F29F
:1037B00071510948FCF782FF084A537D13B1043B5D
:1037C000012B06D80AF062FD28B9BDE810400AF0C6
:1037D0002BBD5475F9E710BD9A1601003002002088
:1037E000F8B590F83A50048E074605F007050E46E6
:1037F000284600210AF046FC97F8F8306A00DB06FC
:10380000E1B242F001020ED50431C9B208200AF03B
:10381000A5FC3246294607F1F9000AF0D9FEBDE8B9
:10382000F8400AF0CDBC08200AF098FC3046F6E7D4
:10383000F8B5134C94F8785194F874310135EDB221
:10384000AB4208BF002594F87731AB4207460E46DD
:1038500004D142F27E310B48FCF730FF94F8782116
:10386000D4F8703123F8327094F8782103EBC20356
:103870005E6084F87851BDE8F84007F00DB800BFED
:10388000300200209A1601002DE9F047254D06462A
:10389000A846002795F8753195F876219A4236D0DA
:1038A00095F87591D5F86CA1D5F808013AF839204A
:1038B0000AEBC9034FF4AA715C682760FEF71CFC91
:1038C00003463AF839001A8C824222D1D3F84821B3
:1038D00042B9D3F83C21C3F848411AB9C3F83C4176
:1038E000C3F84C21D3F84C2102B11460C3F84C4109
:1038F00098F8753198F874210133DBB2013E9A4291
:1039000008BF002316F0FF0688F87531C2D1BDE864
:10391000F087237967F3010323712146FFF788FFBE
:10392000E6E700BF3002002073B5012204461146CD
:103930000020FEF74DFC94F8202042F29B3300213A
:1039400007320093D2B23F4B0846FFF7A3FA30F09C
:10395000020304D042F29D313B48FCF7AFFE3B4DE1
:103960006B7D052B27D1238C2A7C07339A4222D1E9
:10397000002142F2AC3300930122324B29740846F5
:10398000FFF788FA30F0020304D042F2AE312E483D
:10399000FCF794FE002242F2B33300931146294B08
:1039A0001046FFF777FA30F0020304D042F2B53147
:1039B0002548FCF783FED4F83C11D4F840319942F5
:1039C00003D0D4F84831994201D1214E12E00B794D
:1039D0006FF301030B710B68C4F83C31208CFFF7C7
:1039E00027FFE8E70368C4F83C31C4F840313146AA
:1039F000FEF767FBD4F83C0118B1D4F8483198427F
:103A0000F0D10023C4F84031C4F84431D4F83C115B
:103A100051B94FF6FF732384D5F88831A34208BF0C
:103A2000C5F8881102B070BD0B796FF301030B71FB
:103A30000B68C4F83C31C4F84831208CFFF7F8FE1D
:103A4000E4E700BF114400009A1601003002002094
:103A50008C030020F8B50F4690F83810C58DC1F3DF
:103A6000C2040646C90920460AF00CFB96F8F83055
:103A700062009B06E9B242F001020DD50431C9B2E1
:103A800008200AF06BFB394606F58D700AF0EEFD52
:103A9000BDE8F8400AF09ABB08200AF05FFB384600
:103AA000F6E70000262810B504460BD027280BD0D7
:103AB00025280BD102200AF021FB2046BDE810404A
:103AC0000AF022BB1A20F6E75020F4E70A2802D8B1
:103AD00002304000EFE7272801D80330F9E74FF420
:103AE000B7510248FCF7EAFDE7E700BF9A1601006C
:103AF00070B5334C94F8793094F87A209A4227D0F4
:103B00000133DBB2022B08BF002384F87930012295
:103B100094F8790094F8C9302B21272515FB00155E
:103B200094F8CA10994204EB050613D00133DBB2B6
:103B3000022B08BF002384F8C93094F8C90027235A
:103B400003FB00400622B11C7D30FEF750F903E074
:103B50000022DDE7002AF0D130460AF037FB635D32
:103B600003F00F03022B22D0072B20D00223962034
:103B700063750AF051FC00200AF0B0FB94F828307D
:103B8000C3F30202D3B219460020CE0700F10105AB
:103B900012D5013B134094F82820C0B263F302020F
:103BA00084F828202530BDE87040FFF77BBF032351
:103BB00063750AF0A9FBE1E749082846E5E700BF7D
:103BC00030020020000000002DE9F04F8FB0924637
:103BD0000493D0E90032002B8046099180F2B68030
:103BE000816823F000438A422CBF9A1A5A1A059220
:103BF000D8F80C2000243D32CDE90B44FF27D31820
:103C000007938DF82970ADF82A400697A146A34680
:103C1000254602230D930DAB02937B4B01930BAB17
:103C200000930DF129020CAB01210020FFF76CF984
:103C3000022800F094800D9B23B141F26E4173483D
:103C4000FCF73CFD9DF82930FF2B64D0FF2F07D0F7
:103C50000C9B4B4504D041F277416C48FCF72EFD9C
:103C60009DF82920052A51D9694890F81031073369
:103C70009A424BDA062A00F09F80069BFF2B4AD11E
:103C8000073A92B24FF4AA71D0F80801FEF734FA5D
:103C900080453BD0099B1BB990F91D30002B35DBCB
:103CA000059B0B9E1E44D0E90032002B5BDA816835
:103CB00023F000438A422CBFB6187618F61AC26861
:103CC00002F13D094B440893DAF80030B34216D2B2
:103CD0009D4238BF1D46079B0BEB0307189B1B78C3
:103CE000A34205D929463046FFF79EF9B8423ED295
:103CF000BDF82A30049ACAF8005093420BD2DDF87E
:103D000030909DF82970DDF820B03546189B1B785F
:103D1000A3423FF67EAF9DF82930FF2B11D1DAF890
:103D20000030DFF8F08036A7D7E900679D4238BF42
:103D30001D464FF00709189B1B78A3423ED8CAF8CE
:103D40000050189B1C700FB0BDE8F08F934238BF35
:103D5000134600224BE701210020FFF74DF90D9B90
:103D6000022BF8D067E7934238BF1346A7E7294AEA
:103D700005EB0B03A3FB0201072202FB031120A3A7
:103D8000D3E90023FCF70CFA40F2E243B0FBF3F076
:103D9000049B80B29842ADF82A000BD2199B0222F4
:103DA00003EB44000DF12A010134FEF720F8E4B2E0
:103DB000283593E700259BE70692A7E705EB0B0361
:103DC000A3FB080109FB031132463B46FCF7E8F967
:103DD00040F2E243B0FBF3F0049B80B29842ADF8AE
:103DE0002A000BD2199B022203EB44000DF12A0199
:103DF0000134FDF7FCFFE4B228359CE700259EE77F
:103E000000CA9A3B00000000E93000009A16010049
:103E1000300200208D49FD1A1FB5002303930623AD
:103E20008DF80B3090F91D30D0F8DC10002BBEBFA0
:103E30000246036F42F8E43F01910DF10B0100913E
:103E4000A8BF03AAB0F8C6300021FFF7BDFE05B039
:103E50005DF804FB000000002DE9F043B0F8D070DD
:103E600089B0044642480623A7FB00018DF80D30B7
:103E700040F22313002503FB071105AE3AA3D3E953
:103E800000230595C6E90155FCF78AF908AA0DF14A
:103E90000D0142F8100DB4F8C630009101960121D1
:103EA0002046FFF791FE04F1D007A8464FF6FF79B0
:103EB000022239460DF10E00FDF799FF9DF80D0025
:103EC000BDF80E200023D9B2884215D80135062D41
:103ED00007F10207ECD1D4F88C00B8F1000F15D12E
:103EE000BDF8142040F2E2435343C4F88430022268
:103EF0003146FDF77CFF26E04A4505D036F8131021
:103F0000914223D04FF001080133DCE794F874307C
:103F100084F8753094F8C03084F8C130154B002215
:103F2000C3F8882110F8053C43F0030300F8053C72
:103F3000032300F8043C112300F8023C0F2300F88F
:103F4000013C2023037009B0BDE8F08340F2E24356
:103F50005343D4F88C00C4F8843002220DF10E01D2
:103F6000C7E700BFAFF300808D49FD1A07000000CE
:103F70000054CE09300200202DE9F04F8BB0002410
:103F8000FF25DFF818918DF81F50804693461F4695
:103F900001F1040A1C60089426460223099309AB28
:103FA00002933B4B019308AB00930DF11F025B465C
:103FB00041460020FEF7A8FF02283BD0099B23B111
:103FC00041F2B3313348FCF779FB9DF81F20FF2AFB
:103FD00055D0062AE1D999F8103107339A42DCDA34
:103FE000073A92B24FF4AA71D9F80801FEF784F8A3
:103FF0000028D2D090F91D30002BCEDBD0E9003C58
:10400000002B089A1ADA816823F000438C452CBFF4
:1040100062445218D21AC168FF2D01F104010B4409
:1040200010D19DF81F501C461646B6E741460020A9
:10403000FEF7E2FF099B022BF8D0BFE7634538BFCC
:104040006346E8E73146104605930492FEF7ECFF1D
:1040500004EB0A018842DDE90423E2D90E48344426
:10406000A4FB0001072303FB041107A3D3E90023EA
:10407000FCF796F8803038600BB0BDE8F08FFF2D6C
:10408000ECD1F9E7AFF3008000CA9A3B00000000D2
:10409000E93000009A1601008D49FD1A3002002017
:1040A00073B5164602AA1C46054642F8046D273130
:1040B0000120FFF761FF23681BB3019B9B1B1B02C1
:1040C00004D541F207411448FCF7F8FA314601984B
:1040D000FEF7AAFF024611480723A2FB000103FBDB
:1040E00002110BA3D3E90023FCF75AF82368184404
:1040F0000028206005DB40F2E240684323688342E9
:1041000001D802B070BD1B1A2360F7E7AFF300803F
:1041100000CA9A3B000000009A1601008D49FD1A62
:1041200013B500F184030446D0F89020C168808C58
:10413000FFF7B6FF02A9D4F88430D4F88C0040F21F
:10414000E242B3FBF2F3022221F8023DFDF74FFEFB
:1041500002B010BD10B4054C024604F58273D4F8C9
:10416000FC10B4F8F40010BCFFF79ABF3002002036
:1041700070B504780A78C4F38013B3EBD21F19D159
:1041800004F00F04012C00F1020501F1080608D02B
:10419000062231462846FDF71AFEB0FA80F04009A3
:1041A00070BD062231462846FDF711FE0028EFD1EA
:1041B0002046F5E70020F3E710B5174C94F841319D
:1041C00094F842219A4204D142F2C6211348FCF7E6
:1041D00075FA94F84121D4F83C3153F8221094F840
:1041E000783108680B7094F8413194F8402101331C
:1041F000DBB29A4208BF0023094A84F84131FDF737
:10420000A0FF20B942F2DA210448FCF757FABDE8D2
:10421000104006F041BB00BF300200209A1601009A
:104220008003002010B50120FEF7A6FF044620B948
:1042300041F668010948FCF741FA4FF6FF73E38045
:104240000623237104F108001D220021FDF7FCFD67
:104250003C232372BDE81040FFF7AEBF9A16010061
:10426000D0F8B43070B504460E4600F1B40523B959
:1042700042F2F9311048FCF721FA238CA4F8BA3045
:104280000E4A84F8BC60072384F8B83092F878317D
:10429000D4F8B40084F8B43002F5A8722946FDF7CA
:1042A00050FF20B942F209410348FCF707FABDE884
:1042B000704006F0F1BA00BF9A16010030020020EB
:1042C0002DE9F0478246087801F108080D46C0093B
:1042D000414691461E4609F0D1F80446D8B91C4F14
:1042E000BAF1000F0ED12B7897F8E120DB09B3EB80
:1042F000D21F13D1062241461648FDF768FD68B962
:10430000012012E097F8E230DB07ECD5484608F0D0
:1043100047FE0028E7D02046BDE8F08797F8E10087
:10432000C0F3011010F0020001D10446F3E795F943
:104330000030002B09DA6B7B03F0C003402B04D163
:10434000002EDDD001203070EFE70020EDE700BF48
:1043500030020020140300202DE9F04180460320A4
:104360000F461646FEF708FF044688B34FF6FF7364
:10437000C380184B93F8E1305A0725D0C3F30203EA
:10438000DAB2012A1DD0042A1CD040F2BE411248E4
:10439000FCF794F904F10805B8F1000F16D009F004
:1043A000CBFF00F07F00637A2B449870637A2B4434
:1043B000DF70637A1D442E71FFF7FEFE0020BDE81A
:1043C000F08103232371E5E70223FBE77F20EAE77F
:1043D0000120F4E7300200209A1601000B4A92F8FF
:1043E000803192F8811199420ED192F8803102EB1E
:1043F0004303A3F87A0192F880310133DBB2032B37
:1044000008BF002382F88031704700BF30020020CF
:1044100020B141F27B110248FCF750B9704700BF50
:104420009A16010001280A4B0AD19A7C052A02D16A
:1044300000229A74704741F294110648FCF73EB985
:104440001B7C052B02D141F29B11F6E7704700BFA0
:10445000300200209A16010001280A4B0AD19A7CEA
:10446000062A02D100229A74704741F2AD11064823
:10447000FCF724B91B7C062B02D141F2B411F6E7FC
:10448000704700BF300200209A16010040B1054B72
:104490009B7C052B04D041F283110348FCF70EB935
:1044A000704700BF300200209A16010060B1074B30
:1044B0009A7CC9B28A4207D0DB7C8B4204D041F29D
:1044C000BE110348FCF7FAB8704700BF3002002065
:1044D0009A160100044B5B7D23B10121002208469E
:1044E000FDF776BE704700BF30020020062810B5E9
:1044F0000C460AD9094BC21F92B24FF4AA71D3F8E5
:104500000801FDF7F9FD206010BD052804D006283C
:10451000034818BF0020F7E70248F5E73002002003
:10452000000300204802002008B50A4B00221A7040
:10453000094BA3F11001012818BF0B461146FDF7E6
:104540006FFE30B141F285210448BDE80840FCF718
:10455000B5B808BD54040020CC4500209A160100CF
:10456000002208B51146064B1046FDF759FE30B142
:1045700041F2F8110348BDE80840FCF79FB808BDB8
:10458000FC4400209A160100002208B51146064B93
:104590001046FDF745FE30B141F22F210348BDE83A
:1045A0000840FCF78BB808BD9C4500209A16010016
:1045B00010B5094C237823B941F2DC110748FCF708
:1045C0007DF820780138C0B2207018B9BDE81040DD
:1045D00006F060B910BD00BFF00300209A1601007C
:1045E00038B1054A1378591C117023B9012006F01F
:1045F00051B9FFF7DDBF7047F0030020FFF7D8BFC8
:104600001FB5544C48B1A37C052B04D041F60111D1
:104610005148FCF753F804B010BD237C052B02D0A1
:10462000637C052B7AD104AB022243F8082D0022CB
:1046300000930121494B1046FEF72CFC022814D0B0
:10464000029BFBB10298012840F08180237D002B62
:1046500064D0434B04229A6000221146FDF7E0FD2E
:1046600000285BD041F6EA0155E0012211461046D0
:10467000FDF7AEFD029B022BE2D101210020FEF7E7
:10468000BBFCF7E702230393237C23B941F6960191
:104690003148FCF713F803AB0122002000931146C8
:1046A0002E4B2074FEF7F6FB022819D0039A22B392
:1046B0000398012848D100222A4B1146FDF7B0FD8E
:1046C00020B141F6D0012448FBF7F8FF0022264B29
:1046D00011460120FDF7A4FD00B341F6D6011AE012
:1046E000012211461046FDF773FD039B022BDDD11D
:1046F00001210020FEF780FCF7E7A369E16923F0C0
:1047000000438B4216D2174B11460120FDF788FD5E
:1047100020B14FF4C6511048FBF7D0FF0022134BD5
:1047200011460120FDF77CFD00283FF474AF41F6EF
:1047300010116DE70C4B11460120FDF771FD0028AB
:10474000ECD041F6C701E6E741F6D801E3E741F6D0
:10475000F201E0E7300200209A160100E930000083
:104760004C4500201C450020DC450020EC44002086
:1047700030B50468002C89B01FDAD0E9013524F087
:1047800000449D4234BFE41A641B0D4B0593A4B250
:1047900000230690CDE90333CDE901431846009488
:1047A000FEF72EFB30F0020307D0064841F2B72196
:1047B00009B0BDE83040FBF781BF09B030BD00BF94
:1047C000093100009A16010037B502AD104B45F8CB
:1047D000043D044609F03CFC002009F081FC0D4832
:1047E00009F000FC0121204609F04CFC284609F0A4
:1047F0009DFC620002F0FE022521082009F0AEFCBB
:10480000054940F25B6009F04BFD03B030BD00BFCD
:10481000D6BE898EE97A00005555550008B5084B7B
:104820000022986011461046FDF7FAFC30B141F2C3
:1048300095510448BDE80840FBF740BF08BD00BFE4
:104840003C4500209A1601002DE9F04F90468FB0AC
:10485000D8F800401A9A0C929B461B9A0B91002C98
:104860008146189B9DF864A00D92DBF8005003DA96
:10487000AB4238BF2B461C46AC425A4F40F28380B5
:1048800041F2C253CDE90773574B0021CDE9041320
:10489000631B009306914B46CDE902110191012261
:1048A0000846FEF763FA30F0020304D041F2C45127
:1048B0004E48FBF703FF00231A4619461846FFF738
:1048C00063FE4B4E0B9BF36041F2EF53CDE9077350
:1048D0000D9B069300220C9B0593CDE903224B46CA
:1048E000CDE90122009411461046FEF73FFA30F060
:1048F000020304D041F2F1513C48FBF7DFFE0520F2
:10490000FFF78CFFD6F88431AB4228D0CBF80030CB
:10491000D8F80030002BBCBF23F00043C8F80030AB
:10492000D8F80020D6F884118A4238BF0A4641F2EE
:104930001D61A3B292B2CDE905710021CDE9012339
:104940000092CDE9031152460846FEF759FA30F0BD
:10495000020304D041F21F612448FBF7AFFEFF20A1
:10496000FEF792FF234B012211460020C3F808A056
:10497000FDF756FC90B31D4841F232610FB0BDE81F
:10498000F04FFBF79BBE22D200231A461946184669
:10499000FFF7E6FD41F2D753CDE90773164B00212F
:1049A0002C1BCDE9041306914B46CDE90211CDE94C
:1049B000004101220846FEF7D9F930F0020304D085
:1049C00041F2D9510948FBF779FE2C4679E70023DB
:1049D0001A4619461846FFF7C3FD6CE70FB0BDE84D
:1049E000F08F00BF11440000614500009A160100DD
:1049F00030020020FC450020894500007FB50D4CA9
:104A0000237C05460E4623B141F2A7710A48FBF705
:104A100055FE00220392094A0523CDE90132237491
:104A2000236A0093064B31461A1F2846FFF70CFFF6
:104A300004B070BD300200209A1601004D4C0000F9
:104A40004C0200207FB51F4C237C05460E4623B147
:104A500041F633111C48FBF731FE002203921B4A3A
:104A60000623CDE901322374D4F8D8300093184BD3
:104A700031461A1F2846FFF7E7FED4F80031F3B19C
:104A8000D4F8D030002B0ADAD4E9352123F00043E2
:104A900091422CBFC3EB0103C3EB02031D440D4B3A
:104AA0000122114600209D60FDF7BAFB38B106488F
:104AB00041F65A1104B0BDE87040FBF7FFBD04B0E9
:104AC00070BD00BF300200209A160100294D000081
:104AD000040300206C45002007B50520FFF79EFE6B
:104AE00041F62613002100930522094B0846FEF7E4
:104AF000D1F930F0020307D0064841F6281103B07F
:104B00005DF804EBFBF7DABD03B05DF804FB00BF12
:104B1000014600009A160100436810B45C681CB19D
:104B2000A446002310BC60476FF0220010BC704701
:104B30000C4B1A7810B58AB901220B481A700BF089
:104B40002FF8044620B941F247210848FBF7B6FD8B
:104B5000636801211B682046984700B910BDFEF725
:104B6000A1FAF5E7BC030020841101009A160100A8
:104B7000024B1868436800215B6818473002002028
:104B8000F0B4484003274FEA102C082600240CF00C
:104B90000105013E45EA440516F0FF06ECB24FEA76
:104BA0005C0CF4D125022DB2C0B24FF0080C344693
:104BB00000F0010646EA44040CF1FF3616F0FF0C43
:104BC000E4B24FEA5000F3D12C4304EB0414013F4C
:104BD0000C4417F0FF07A0B2D5D125244140B1FB0A
:104BE000F4F004FB1010C0B2C40800F00705145D17
:104BF0002C41E40705D45943090C1046F0BCFEF7DC
:104C000089BAF0BC7047000070B514460E460546E0
:104C1000FEF708FA2146FEF707FAC41C092C11D941
:104C2000094B1B7813B10020FFF77EFC32460021B0
:104C30002846FFF79DFDAB681C44262C00D8AC60CD
:104C4000012000E0002070BD5404002070B5324CFB
:104C5000237D054623B141F60A013048FBF72EFDBE
:104C6000237C052B04D041F60B012C48FBF726FDD5
:104C700094F82900A56000230126267500F007009E
:104C8000237405236374FFF79FFD94F8293094F88B
:104C90002820C3F3C20363F3020284F82820FEF73E
:104CA00027FF08F00BFC94F8293000B313F0C00F75
:104CB00014BF3046002008F005FA821C41780078C5
:104CC00009F052FBE26805F10901012009F0B0FB8F
:104CD00009F05EFC2A4605211148FFF795FF0346BF
:104CE00050B104236375BDE8704009F09DBA13F01C
:104CF000C00FE7D03046DEE70A4A0146FEF742F928
:104D000030F0020306D041F65A010448BDE8704075
:104D1000FBF7D4BC70BD00BF300200209A16010022
:104D200048020020D5440000F0B55C4C237D8DB0D6
:104D3000054623B141F66D115948FBF7BFFC237CB2
:104D4000062B04D041F66E115548FBF7B7FC022341
:104D500023750123002663750623267494F8E10069
:104D6000637494F8E030A56066F3410300F0070037
:104D700084F8E030FFF728FD94F8E030C3F38100B9
:104D8000421C62F38303253084F8E030FEF78AFE8C
:104D900094F8E03003F00C020C2A08BF66F383039A
:104DA0004FF0960008BF84F8E03009F035FB00238F
:104DB00019461A46184609F09DFAD4F83C3194F881
:104DC000412153F82200083009F0FAF909F0AAFA53
:104DD00008F074FB94F8E13040B3C3F3001008F01E
:104DE00071F906460DF12F0008F0EEF871780746CC
:104DF000B21C307809F0B8FA39469DF82F0009F056
:104E000083FCE26805F10901002009F011FB09F0BB
:104E1000BFFB06212A462348FFF7F6FE014688B16C
:104E20000423637509F000FA0DB0F0BD13F0300FE4
:104E3000E7D0012008F046F9821C4178007809F09B
:104E400093FADEE741F6C9130893174B0793174B04
:104E50000190CDE90403D4F8F03004220933009323
:104E600006922B46CDE90200FDF780FF30F00203E9
:104E700004D041F6CC110A48FBF720FC0023194668
:104E800018460B4AFEF77EF830F00203CCD041F60C
:104E9000D5110348FBF712FCC6E700BF3002002023
:104EA0009A1601000003002011440000A5500000E4
:104EB000D544000010B5044609F0CAF8002009F0F6
:104EC0000FF90A4809F08EF804F1100009F02EF9E4
:104ED000637DA17D1B0243EA0143217D40F25B60BB
:104EE0001943BDE8104009F0DBB900BFE97A0000C2
:104EF0002DE9F041684D1C462B7D074623B142F257
:104F000056016648FBF7DAFB238C2A7C07339A426A
:104F100004D042F259016148FBF7D0FB03232B7503
:104F200001236B7594F82030C5F81441002607332F
:104F3000A5F81861DBB22E746B74238D638520464F
:104F40002685AF60FFF7B6FF962009F065FA94F862
:104F5000382094F83A00D3093146C2F3C20200F077
:104F6000070009F0C7F995F84121D5F83C3153F80D
:104F7000221020460831FEF733FC637F580604F107
:104F8000170259D5608CE18B013803F03F0380B2E2
:104F9000FFF7F6FDFEF786FDD4E917231344002240
:104FA000E265A26D2366934288BF2266D4E9192385
:104FB00000261344A366EA68666607F109013046D5
:104FC00009F036FA804609F0B7FA304609F0CEFA11
:104FD000A36E206E03F1500606EB400694F83A00EB
:104FE000012100F0070009F002F94644064494F854
:104FF0003A0000F0070002283ED004280CBF4FF40E
:10500000BC73282301211E4409F0F3F8304409F051
:1050100087FA94F8201007313A46C9B22046FFF7C4
:10502000F3FD034650B304236B7509F0FDF802202D
:10503000BDE8F041FEF728BC618DA67F01FB066646
:10504000E17F25200E4496FBF0F100FB1166F0B2E3
:10505000C108E077515C06F0070641FA06F6F10751
:1050600003F03F0396D4B0FBF3F103FB1101C9B287
:105070001046FEF74FF88DE71823C3E7084A0146AC
:10508000FDF780FF30F00203D1D042F2DD0103488A
:10509000FBF714FBCBE700BF300200209A1601009B
:1050A000D5440000084A08B5936013460022114613
:1050B0001046FDF7B5F830B141F295510348BDE80F
:1050C0000840FBF7FBBA08BD3C4500209A160100DA
:1050D00010B590F8F840D0F8402114F0800F18D1A6
:1050E000D0F83C31ABB1240713D4D0F84841A342E7
:1050F00004BF1C68C0F8484192B91A680A60196078
:10510000C0F84011C0F844110B680BB9C0F84C113D
:1051100010BD2AB9D0F83C310B60C0F83C11EFE764
:10512000D0F844311A680A601960EBE710B490F8BF
:10513000F84024070A460FD5D0F8401131B9D0F80D
:105140003C111160C0F83C2110BC7047D0F84431CC
:10515000196811601A60F7E710BCFFF7B9BF0000CB
:10516000F8B5214F054607F5AE700E46FCF790FFE7
:105170000446B0B333797179D7F8142143F07F43F3
:1051800043F47E0343F4435343F0100343EA012303
:10519000B17943EA0143D2F8A410C1F310010B40E6
:1051A000C2F8A43092F8503043F0200382F8503017
:1051B000037943F003030371082209234371C37188
:1051C00000211044FCF740FED5F8A43023721A0ADF
:1051D0001B0C28466272A3722146FFF7A7FF00202E
:1051E000F8BD0120FCE700BF3002002090F8F83045
:1051F00043F0200380F8F8300B7843F003030B7082
:1052000001234B700623CB700020704770B5044615
:105210000B480E461546FCF73BFF78B10379067242
:1052200043F003030371032343711123C3714572D8
:1052300001462046FFF74CFF002070BD0120FCE72F
:105240008C030020000000002DE9F04FCC4D8FB002
:105250001C462B7C0A918146174623B141F6857185
:10526000C848FBF72BFA94F820300733DBB22B74D5
:1052700094F91D30002B09DA636DE26D07FB0333EF
:105280001344A26DE365934288BFE265228D94F8D2
:1052900074301744628CBFB22785174494F8752088
:1052A0009A42BFB240F0AF8194F8F8305E0700F147
:1052B000988294F8C12094F8C0309A4200F0968009
:1052C0000520FFF7ABFAD5F8883113B19C4240F0C6
:1052D0008D8094F8C23003F00703052B00F24C8157
:1052E000DFE813F0060065001E01840084008400DE
:1052F000A548FCF7CDFE0646002877D094F8C230CA
:10530000042262F3020384F8C230037943F00303FA
:105310000371182343710F23C371B4F8C4300381A0
:10532000B4F8C6304381B4F8C8308381B4F8CA30C9
:10533000C38100230374C37403754FF0FF334375B7
:105340008375C375037643768376C3760377437795
:105350008377A0F8117001462046FFF7B9FE226856
:10536000B4F84230C5F88841002AA4F84430C4F8A3
:10537000E0900BDAD4E9011322F000428B422CBFFB
:105380004B4409EB01039B1AC4F8E03013367F4B02
:10539000C4F8DC600122114600209C60FCF740FF4D
:1053A00020B341F6F5417748FBF788F91EE094F801
:1053B000C36096B37448FCF76BFE0146B0B1037945
:1053C00043F0030303711123C371032343710F23BC
:1053D000037294F8C33043722046FFF779FE94F8C5
:1053E000C03084F8C1300023C5F8883194F8F52026
:1053F00094F8F4309A4200F0FF800520FFF70EFA8F
:1054000094F8F63003F00302032A00F26E81DFE81D
:1054100012F0BF00F300F3000D0194F91D30002BD2
:105420003BDB94F8741094F875308B42DED194F81D
:10543000C230C4F88460052262F3020394F8CC20E1
:1054400084F8C230012384F88830B4F8C63022B121
:1054500093FBF2F3013313FB02F3A4F87A30B4F8B0
:10546000C830A4F87C30B4F8CA30A4F87E3094F880
:105470007830022262F3010394F8C22082F008021D
:10548000C2F3C00262F3820384F878300139012349
:1054900084F8763084F87510A8E73B48FCF7F8FDEF
:1054A00001460028A2D0037943F0030303711823B7
:1054B00043711023C371B4F8C4300381B4F8C6300B
:1054C0004381B4F8C8308381B4F8CA30C38194F8FA
:1054D000CC300374B4F8CE30A0F81130B4F8D0302A
:1054E000A0F81330B4F8D230A0F81530B4F8D430A6
:1054F000A0F81730B4F8D630A0F81930B4F8D83086
:10550000A0F81B30B4F8DA30A0F81D302046FFF7C1
:10551000DFFD94F8C03084F8C130C5F8886165E7D4
:1055200094F8F83018073FF561AF0220FDF724FE2C
:1055300000283FF45BAF94F8C230032262F3020309
:1055400084F8C230238CC38001230371037A134390
:105550000372182343720F23C372B4F8C4308381DB
:10556000B4F8C630C381B4F8C8300382B4F8CA3086
:105570004382FEF721FE39E741F6AE5113E700BF43
:10558000300200209A1601008C0300208C45002078
:10559000B348FCF77DFD014670B394F8F63094F8FB
:1055A0003900012262F3010384F8F630DBB2C3F361
:1055B0008206C3F3421363F3C50094F8382084F8DD
:1055C000390094F8F70066F30202C0F3000060F3BC
:1055D000861284F838200A794B7242F003020A716D
:1055E00003224A711622CA710E722046FFF770FD1F
:1055F000B4F84230A4F8443094F8752094F874302C
:105600009A4200F0EE800520FFF708F994F8763012
:10561000013B072B00F2E385DFE813F06D00E302A6
:1056200045035C04BA04E10519052D0594F8F4203E
:1056300084F8F520C3F38202910744D5022262F375
:10564000840384F8F63094F8F6305A09900743D56D
:10565000022262F3471384F8F63094F8F62094F8A7
:105660003830C2F38201C3F3C2038B4294F878301E
:1056700014BF61F384036FF3840384F8783094F8E3
:105680003A30520903F00703934294F8783014BF7C
:1056900062F347136FF3471384F8783094F8783047
:1056A00094F8F72043F00103C2F3400262F3410390
:1056B00084F87830082384F8763094F87530013B0C
:1056C00084F8753098E7D60701D50122B7E712F0C4
:1056D000040218BF0422B2E7D10701D50122B8E7BE
:1056E00012F0040218BF0422B3E741F60E715D48C0
:1056F000FAF7E4FF80E7D5F888310BB9C5F888419F
:1057000094F8783013F0030300F0B4805448FCF7A9
:10571000BFFC0646002864D094F8783003F00303F9
:10572000012B09D0022B00F0988041F652214D4800
:10573000FAF7C4FF002200E04B4A94F87830317940
:105740006FF3010384F87830E38C06333B449BB25B
:1057500041F00301A4F8803031710C2171710021F6
:10576000F17194F88810317240F2E240D4F884105C
:10577000B1FBF0F1A6F80910B4F87A10A6F80B10F6
:10578000B4F87C10A6F80D10B4F87E10A6F80F102F
:105790002168A6F811300029C4F890900BDAD4E9FA
:1057A000010321F0004183422CBF4B4409EB00036D
:1057B0005B1AC4F8903006F10903C4F88C302B4B07
:1057C000C3E90242012211460020FCF729FD20B165
:1057D00041F61A212348FAF771FF31462046FFF7B8
:1057E00077FC94F8B12094F8B0309A421ED005208E
:1057F000FFF714F81A48FCF74BFC0146B0B194F8D7
:10580000B03084F8B130037943F00303037102230D
:105810004371C37194F8B23003722046FFF758FC0D
:10582000E38F012B98BF0133A4F8443094F8E920AA
:1058300094F8E8309A4200F015850520FEF7EEFF57
:1058400094F8EA3003F00303032B00F2E985DFE864
:1058500013F0C904090509052505054A6DE700BFD0
:105860008C0300209A160100214100007C45002095
:10587000593E0000B4F88080A7EB08081FFA88F8AA
:1058800018F4004FADD194F8742084F8752094F882
:10589000C01094F8C1208A4209D094F8C22002F0C6
:1058A0000702052A04BF84F8C110A4F84430D5F8D3
:1058B00088210023944208BFC5F888312B74A28C3C
:1058C000B4F87A309A4214D1B4F87C10E38C99423F
:1058D0000FD140F2E2435A43B4F87E3042F21071E5
:1058E00001FB0323013B93FBF2F3E28F9BB29A424D
:1058F0001DD00220FDF740FC064620B941F68E215E
:10590000CD48FAF7DBFE238CF380082333710023A4
:105910003372B4F87A30A6F80930B4F87C30A6F8BF
:105920000B30B4F87E30A6F80D30FEF745FCD4E914
:105930000037002B0ADAA66823F00043B7422CBFD9
:1059400009EB07064E442360A6EB0309A38CB4F8C9
:105950007AB0BA4913FB08F39BB2B3FBFBF21FFA10
:1059600082FA1BFB0AF080B2834280F01581C01AD4
:105970000246C317CDE90A230B9B40F22312424390
:1059800001FB0323A0FB01011944A9A3D3E90023D0
:10599000FAF706FC20F07F4000EB0906238DA3EB0D
:1059A00008035344238523689F4238BF1F46D4F819
:1059B00084300A9394F91D300D9740F2E249002B90
:1059C00009FB0BF780F2FE80E26D636D9C4903FBDF
:1059D000182395F820219B4D31F8128094F850201F
:1059E000C2F3820231F8122094F88810904407FB29
:1059F00008F808F57428944A09FB01F108F23F28D9
:105A0000B8FBF2F87A0808FB0AF0963A034461669C
:105A10000021C4F85480A2652167934294BFE365D6
:105A2000E265A0FB050182A3D3E90023FAF7B8FBE6
:105A30000A9B361AB3FBF9F009FB00F0A0FB050145
:105A40007BA3D3E90023FAF7ABFBA7EB080820F010
:105A50007F45B4F87E30B4F87C20E28442F21071C5
:105A600001FB0373013BB3FBF7F3E387774BA4F828
:105A700024B03B44B3FBF7F3A4F84230744B3B44EF
:105A8000B3FBF7F7931DB9B29942C4BFC2F57F4388
:105A9000FA33A4F84A10C8BFC91894F87830C8BFC0
:105AA00089B213F0040308BFA4F84030A4F84610EC
:105AB0000020012108F08EFE0022012182461046BE
:105AC000FCF786FB94F82070624B0737FFB2002189
:105AD00000973A460846FDF7DDF930F0020304D09E
:105AE00041F617315448FAF7E9FD564BA8FB0389F4
:105AF00040464FA3D3E900234946FAF751FB002360
:105B000020F07F42CDE90A230A99534A07234B43E9
:105B10000B9902FB01330A99A1FB02121A4420F0EF
:105B20007F4B0846B8EB0000114669EB01014FF4CA
:105B30007A720023FAF734FBE3680D9A94F91DC0DA
:105B4000464908971A441346454A32EA2C0228BFB0
:105B50000A464449CDE906410021CDE90432CDE9A8
:105B600002013346CDE9005B3A460846FDF7FEF8F0
:105B700030F0020304D041F625312F48FAF79EFD9C
:105B8000BAF1000F00F087830122114600200FB008
:105B9000BDE8F04FFCF71CBB0BFB123082B20023B8
:105BA000CDE90A230A9B0A9AA3FB010140F22313C1
:105BB00003FB02111EA3D3E90023FAF7F1FAA9EBC4
:105BC0000006EBE60A9908461E4919A3D3E900230B
:105BD000A0FB0101FAF7E4FA20F07F40451CB8462B
:105BE00037E794F87830002B40D01F48FCF750FA84
:105BF000064600283FF4F5AD002384F87830E38CA6
:105C000006333B44A4F87E30037943F00303037169
:105C1000082343710123C371052204F1790108307F
:105C2000FCF7E5F8B4F87E30A6F80D30D5E500BFF6
:105C30008D49FD1A070000009A1601000054CE0994
:105C40008A16010000CA9A3B40420F00FF596202C7
:105C50007FC3C9018D3200008D49FD1A39640000EF
:105C60003D6400006D3200008C030020B4F87E30EB
:105C7000FB1A1E043FF5B5AD94F8743084F8753006
:105C800004F11706052204F179013046FCF7AFF85C
:105C900005213046FCF7A4FB637F60F305036377BF
:105CA000012323779DE594F87880B8F1000F7FF405
:105CB00098ADE048FCF7ECF9064600283FF491ADBA
:105CC00094F91D30002B00F1040A4DDB04F1F90BAF
:105CD0005B46424604F1940104F1840008F040F868
:105CE0001022594604F58D70FCF781F804F589718E
:105CF000082204F23310FCF77AF894F8113184F892
:105D0000098168F3000384F8113194F8323184F882
:105D10000A8143F0010384F8323194F8F83084F8B2
:105D20000B8143F0100384F80C8184F80D8184F812
:105D30000E8184F80F8184F81081A4F82A81A4F8D8
:105D40002C81A4F82E81A4F8308184F8F8305146D3
:105D50002046FFF74BFA31462046FFF7B9F994F891
:105D6000743084F875303CE594F8F83003F048035B
:105D7000082B00F09F8094F87980B8F1000F20D0B4
:105D8000037943F00303037194F85030980612D559
:105D9000D4F8A43059070ED51123F37103233372BD
:105DA00086F80980022373717379013373710023BC
:105DB00084F87930CFE70D23F37186F8088001234A
:105DC000F1E79C48FCF764F9824600286DD003791E
:105DD00043F0030303710D2343714FF0040B00F1F3
:105DE0000803194680F807B00C2268680D93FEF787
:105DF00093FE0D9B0822194604F19C00FBF7F7FF68
:105E00005A460AF1100104F58B70FBF7F0FF51467A
:105E1000204604F1F90AFFF75BF95346424604F1C4
:105E2000940104F1840007F09BFF1022514604F511
:105E30008D70FBF7DCFF082204F5897104F2331042
:105E4000FBF7D5FF94F8113184F8098143F0010381
:105E500084F8113194F8323184F80A8168F3000330
:105E600084F8323194F8F83084F80B8143F0100351
:105E700084F8F830337984F80C8143F0030384F814
:105E80000D8184F80E8184F80F8184F81081A4F8C4
:105E90002A81A4F82C81A4F82E81A4F830813371D2
:105EA000012373710523F37155E762493046FCF70E
:105EB00008F996E45146D5F81401FFF797F9D5F89B
:105EC000142192F8F83068F3820368F3C30382F870
:105ED000F83040E794F8501011F0200828D094F8DA
:105EE000743084F875300220FDF746F9064620B973
:105EF00041F61C415048FAF7E1FB238CF380012363
:105F00003371337A43F00303337209237372F372EC
:105F10000822002106F10C00FBF796FFD4F8A4300C
:105F200033731A0A1B0C7273B373FEF745F958E406
:105F30004048FCF7ADF8064600283FF452AC94F810
:105F4000743084F875303D4BC4F8A430037943F0C5
:105F5000030303710923437194F91D30002BB4BF6F
:105F60000E2308230822C37141461044FBF76CFF3F
:105F7000D4F8A43033721A0A1B0C7272B372314611
:105F80002046FFF7A5F8B4F84230A4F8443028E4DE
:105F900094F8A830DA0724D42648FCF779F80146AB
:105FA00000283FF41EAC94F8743084F8753094F8EF
:105FB000A83043F0010384F8A830037943F00303C9
:105FC0000371062343710C23C371092303726FF01D
:105FD0000E034372052383724FF0FF33C3720373C2
:105FE000CEE79B072CD594F8743084F875300220E6
:105FF000FDF7C2F8064620B941F68D410E48FAF782
:106000005DFB238CF38001233371337A43F0030368
:106010003372062373720C23F37294F8A93033732E
:10602000B4F8AA30A6F80D30B4F8AC30A6F80F30AA
:106030007BE700BF8C0300209A160100FF49010096
:1060400041F6A541CA48FAF739FBFFF7CABBC94870
:10605000FCF71EF8014600283FF4C3AB94F87430F7
:1060600084F87530037943F003030371012343710E
:106070001223C37184E794F87820D60758D5BD4819
:10608000FCF706F8064600283FF4ABAB94F87830EE
:106090006FF3000384F87830DBB2C3F3820252EA74
:1060A00053123FD194F8741084F875109807A4F82F
:1060B0007A2020D50220FDF75FF8804620B941F60E
:1060C0003271AB48FAF7FAFA238CA8F806300C23A1
:1060D00088F80430002388F8083094F83830C3F387
:1060E000C20388F8093094F83A30C3F3020388F801
:1060F0000A30FEF761F8337943F003033371052367
:1061000073711823F37194F87830C3F382033372F8
:1061100094F87830C3F342137372B4F87A30738111
:10612000FFF75BBBE38C06333B44A4F87A30E2E72D
:10613000B4F87A30FB1A19043FF553AB94F8743075
:1061400084F8753012F01C0F94F8383094F83A1037
:1061500018BFC2F38206C3F3C2001CBF66F3C503B7
:1061600084F8383012F0E00F1FBF94F83A30560927
:1061700066F3020384F83A3094F83830C3F380169B
:1061800066F3C713920701F0070184F838300BD487
:10619000DBB2C3F3C203834206D194F83A3003F072
:1061A00007038B423FF41DAB0220FCF7E5FF0646D8
:1061B00020B941F670716E48FAF780FA238CF380AB
:1061C0000C2333710023337294F83830C3F3C203C5
:1061D000737294F83A30C3F30203B372A5E641F642
:1061E000EB712FE7FCF7B2FF0646D5F83001FBF75D
:1061F0007DFF0644B6B2FF2E04D941F6DE515C485D
:10620000FAF75CFA95F83A31B3422BD15948FBF7CB
:106210003FFF014630B394F8EA30B4F8F2006086EC
:10622000012262F30103B4F8EE20A28584F8EA307B
:106230000B79C88143F003030B7109234B711423BD
:10624000CB711B230B7200234B726FF06F038B72A9
:106250000A23CB728A812046FEF73AFFB4F8423017
:10626000A4F8443094F8203094F91D504248434932
:10627000A268073331EA250128BF0146DBB2CDE928
:106280000023CDE90214231D22460A99484601370E
:10629000FEF7DAFA67840FB0BDE8F08FFCF756FF1F
:1062A0000646D5F83001FBF721FF0644B6B2FF2EB3
:1062B00004D941F61F612E48FAF700FA95F83A31F1
:1062C000B34204D041F625612948FAF7F7F994F86A
:1062D000E83084F8E93094F8EA30D5F80C016FF32F
:1062E000820384F8EA300023A4F84430B4F8EC3098
:1062F0002386B4F8F030E386FBF7F8FED5F8CC300F
:106300000BB1013080B2D5F800310BB1013080B251
:10631000268E95F810310E36013026F0030698428D
:10632000B6B278D0B5F83831B34274D30220FCF756
:1063300023FF054620B941F686610D48FAF7BEF9FC
:10634000238CEB8001232B712B7A43F003032B72F8
:1063500009236B721523EB72238EAB81E38D2B82A5
:10636000E38EEB81A38E6B82FDF726FF7AE700BFF9
:106370009A1601008C030020F14E00008D6700008A
:106380000BB995F84031013B85F8423195F842212F
:10639000D5F83C3153F8223041461868FBF791FE9E
:1063A00095F8403195F85421013B9A4204DB41F6BF
:1063B0005F615046FAF782F995F85431013385F858
:1063C000543195F8423195F841219342D8D1238E2A
:1063D000292B9ABF3423A5F83831A5F83861B5F8D0
:1063E0003631B5F83821B3FBF2F3DBB285F83A3138
:1063F00023B941F676610D48FAF760F9D5F82C011A
:106400000B4B95F83A21B5F83811FBF71DFE042027
:10641000FCF75EFF8AE7DFF81C80DFF810A0D0E70A
:1064200041F6A8610148FAF749F91BE79A160100FD
:106430006003002078030020FEF706BFFEF704BFCC
:106440002DE9F04190F8F8E01EF0800F04460E466A
:106450000DD1D0F83C1151B11EF0080FD0F840C159
:1064600003D190F8EA305B0723D5614521D094F839
:10647000F83043F0800384F8F83007F027FF037802
:10648000012262F3010300224270D4F83C21037020
:10649000DBB25AB143F01003037003786FF3471374
:1064A0000370002383703060BDE8F08162F3041351
:1064B000F2E794F8512194F850310D1DA81813B942
:1064C000437884F8503122B1AB5C012767F30103B4
:1064D000AB5494F8507194F83980BF1AFFB24770EA
:1064E000AB5C6FF30413AB5408F00708B8F1020F6C
:1064F000A38E29D0B8F1040F29D0DB080A3B9BB248
:106500001EF0200F18BF043BB4F82EE018BF9BB25A
:10651000734528BF73469F4281BF4370AB5C43F015
:106520001003AB540B681BB1AB5C43F01003AB54CE
:10653000BCF1000FB1D1D4F8483199421CBFC4F866
:106540004411C4F84011A8E79B080B3BD7E794F827
:1065500038805FEAD81815BFA3F51473A3F5D77375
:106560009B111B11023BCAE72DE9F0418EB00223BB
:1065700009930023CDE90A33FF227D4E7D4F7E4DE6
:106580008DF8232004460C9309ABCDE901630CABD5
:1065900000930DF123020DAB01210020FCF7B4FCA8
:1065A000022826D0099B23B141F20D313846FAF773
:1065B00085F89DF82330FF2B04D095F81021073281
:1065C0009342E1DA5A1FD2B2F92A6C4F05D86A4ACF
:1065D00092F81021073293420FDB3B7813B1012070
:1065E000FDF7A2FF0EB0BDE8F08101210020FCF70D
:1065F00003FD099B022BF8D0D4E70AA9E0B2FDF70E
:1066000075FF054620B941F21D315A48FAF756F890
:10661000D5E90034002BB8BFAB689DF823009C423D
:1066200038BF1C46EB680BA91C44FDF75FFF05460D
:1066300020B941F22B314F48FAF740F8D5E901363D
:106640002A689E4238BF1E46002A09DA0C9B22F0B7
:106650000042921B9A4235BF9A1A00230C920C9367
:106660000C993A7804F131038B420AD212B101201D
:10667000FDF75AFF9DF8232001212846FEF778F800
:10668000B0E75AB901203E4B38701146FBF7C8FD00
:1066900020B141F266213748FAF710F82B68002B39
:1066A00019DBB34217D99B1B00209BB235490591DA
:1066B000CDE901039DF823200695CDE90300009064
:1066C0000121FCF79DFB30F0020304D041F25D3163
:1066D0002848F9F7F3FF0A9E002E83D00B9D002D6A
:1066E00080D0B38CAA8C9A427FF47CAF264897B2B4
:1066F000A7FB000140F2231303FB07111AA3D3E900
:106700000023F9F74DFD0C9B20F07F4000229842BA
:1067100018D302B10C9396F91D1095F91D2000298C
:1067200013DA002AFFF65EAF14349C427FF65AAFAC
:106730003046FCF733FD02287FF454AF0B98FCF78A
:106740002DFD4FE71B1A0122E1E7002ABFF64AAFF1
:1067500014349C427FF646AF2846FCF71FFD022802
:106760007FF440AF0A98EAE78D49FD1A0700000060
:10677000E93000009A160100300200205404002085
:10678000AC450020FD3000000054CE09F7B5504D57
:106790001C462B7D074623B142F2FE014D48F9F716
:1067A0008DFF238C2A7C07339A4204D042F20111D8
:1067B0004848F9F783FF04232B7594F82030C5F877
:1067C000144100220733A5F81821DBB22A746B7438
:1067D000238D6385022022856875AF60FDF754F82C
:1067E00001A92046FFF72CFE019994F8F8200B78B8
:1067F000C2F3000262F3C30394F8F820C2F340022C
:1068000062F382030B702046FEF754FB962007F0DC
:1068100003FE94F83A0000F0070007F05FFD204601
:106820000199FDF717F9637F580604F1170221D586
:10683000608CE18B013803F03F0380B2FEF7A0F9D2
:10684000FDF730F9EA6807F10901012007F0F0FDD2
:1068500007F09EFE94F8201007313A46C9B2204650
:10686000FEF7D2F9034628B304236B7507F0DCFC6E
:1068700003B0F0BD618DA67F01FB0666E17F252098
:106880000E4496FBF0F100FB1166F0B2C108E07710
:10689000515C06F0070641FA06F6F10703F03F03E4
:1068A000CED4B0FBF3F103FB1101C9B21046FCF7E3
:1068B00031FCC5E7084A0146FCF764FB30F00203EF
:1068C000D6D042F2AE110348F9F7F8FED0E700BF88
:1068D000300200209A160100D54400002DE9F04F47
:1068E000C67A85B004460D4600F10807192E01F25C
:1068F000D780DFE816F01A007E00BB00C900F70061
:106900001F014401C5058A01AF01DA010302350206
:106910009E02A001B6022604AE049A05B4054C06F8
:106920004C062407E0071708A108C84ED6F81451F2
:1069300095F91D30002B81F2B380417A0020FCF7DD
:10694000B5FB002801F0AC80B4F815106B8CCB1AA5
:106950001A0400F1898095F8743095F875209A42F0
:1069600042D1D6F888210AB9C6F88851227B85F829
:106970008820B4F80D0040F2E2424243C5F884207A
:10698000207CE27B42EA0022A5F87A20A07C627C8F
:1069900042EA0022A5F87C20E27C207DA5F8801048
:1069A00042EA0022A5F87E2095F8782002F0FC0249
:1069B0006FF38202013B85F87820012285F876206A
:1069C00085F8753095F8C02095F8C130934207D00E
:1069D00095F8C23003F00703042B01D185F8C120DC
:1069E0000020A5F844003CE02A2385F8B3300020BD
:1069F00037E0964BD3F8145195F91D30002B81F2F6
:106A00004F80417A0120FCF751FB002801F04880BB
:106A1000B4F811306A8C9B1A1B0425D495F87420A5
:106A200095F875309A4204D042F281418848F9F7CE
:106A300045FE052204F10C0105F17900FBF7D7F9B9
:106A4000637CA27C002043EA0223A5F87E3085F80F
:106A50007800022385F8763095F87530013B85F88B
:106A6000753005B0BDE8F08F2823BEE7417A0220DB
:106A7000FCF71CFB002801F01380744B227BD3F839
:106A8000143183F8B320B2E7704ED6F8147197F939
:106A90001D30002B81F20480417A0320FCF706FBB5
:106AA000002800F0FD87082204F1160107F1940088
:106AB000FBF79DF9D6F81401042204F11E0100F53C
:106AC0008970FBF794F9D6F8143193F8F82042F066
:106AD000040283F8F820B3F84220A3F844200123ED
:106AE0002B7084E7594DD5F8146196F91D30002BB1
:106AF000C0F2D687417A0420FCF7D8FA002800F0CB
:106B0000CF87082204F10C0106F19C00FBF76FF916
:106B1000D5F81401042204F1140100F58B70FBF781
:106B200066F9D5F8142192F8F83043F0040382F89E
:106B3000F8305CE7454DD5F8142192F8740092F8CE
:106B40007510884208D092F87630032B04D040F6B6
:106B5000E7113F48F9F7B2FDD5F8145195F91D300A
:106B6000002BC0F29D87617A0520FCF79FFA002870
:106B700000F09687002085F8780003236AE7417AC1
:106B80000620FCF793FA002800F08A872F4E327D0A
:106B9000D6F81431032A2FD193F8741093F8752086
:106BA000914208D093F87630032B04D04FF4206143
:106BB0002748F9F783FDD6F81431002283F87820AE
:106BC000032283F8762093F87520013A83F8752024
:106BD000D6F8142192F8F8305F0641BF6FF38613A0
:106BE00082F8F8300923237101232B70D6F8143171
:106BF0000020A3F8440034E793F8F82002F0FB02E9
:106C00006FF3C30283F8F820E2E7104BD3F8145176
:106C100095F91D30002B80F24387417A0820FCF75C
:106C200045FA002800F03C873946284605B0BDE803
:106C3000F04FFEF795BA054BD3F8145195F91D3076
:106C4000002BC0F22D87417A0E20E8E730020020A9
:106C50009A160100417A0920FCF728FA002800F072
:106C60001F87237B617BB34843F07F4343F47E035C
:106C700043F4435343F01003D0F8142143EA0123B3
:106C8000A17B43EA0143D2F8A410C1F310010B40E9
:106C9000C2F8A43092F8503043F0200382F850300C
:106CA00001232B70D0F81431A2E7A24ED6F814516C
:106CB00095F91D30002B80F2F386417A0A20FCF70B
:106CC000F5F9002800F0EC8606F5AE70FBF7E0F968
:106CD000014608B90120C4E695F8F83043F04403B2
:106CE0006FF3041385F8F830037943F0030303715D
:106CF000012343710B23C371284627E0417A0B20FF
:106D0000FCF7D4F9002800F0CB868A48D0F814416B
:106D100094F91D30002B1CDB00F5AE70FBF7B8F9C1
:106D200001460028D6D094F8F83003F0DF0343F092
:106D300004036FF3041384F8F830037943F003037A
:106D40000371012343710B23CB712046FEF7C0F979
:106D50004DE694F8F8306FF3451384F8F83046E6C2
:106D6000417A0C20FCF7A2F9002800F099867148BE
:106D7000D0F8146196F8A83013F0010750D100F54F
:106D8000AE70FBF785F901460028A3D096F8A8302D
:106D900043F0010386F8A830037943F0030303713D
:106DA000062343710C23C371092303726FF00E0392
:106DB0004372052383724FF0FF33C372037330466F
:106DC000FEF7B4F996F8F83043F0800386F8F8300F
:106DD00007F07CFA03784770012262F30103D6F8CA
:106DE0003C210370DBB2C2B143F010030370237B7C
:106DF00086F8A930A27B637B43EA0223A6F8AA3077
:106E0000E37B227C43EA0223A6F8AC3096F8A83054
:106E100043F0020386F8A830E9E562F30413E5E7DE
:106E200013F002037FF4E3ADA6F8443001232B7086
:106E3000DDE7417A0D20FCF739F9002800F03086B3
:106E40003C4BD3F8142192F8F83003F0FB036FF3B6
:106E5000C303002082F8F830A2F8440001232B700D
:106E6000FFE5417A0F20FCF721F9002800F0188691
:106E7000304AD2F88831D2F8140143B1834206D0A7
:106E800020220F2105B0BDE8F04FFEF7BFB990F901
:106E90001D6090F8C01090F8C130002EC0F2B6808E
:106EA000994209D090F8C23013F0070302D0043B96
:106EB000012B01D82322E4E790F8741090F8753084
:106EC000994203D090F87630032B05D190F8F41056
:106ED00090F8F530994201D02A22D2E7B4F80C900C
:106EE0001FFA89F3052B22D9B4F80E801FFA88F116
:106EF000B1F5486F1BD88B4219D8B4F810E01FFACF
:106F00008EF6B6F5FA7F12D2B4F812C01FFA8CF3DF
:106F1000A3F10A07BFB240F6764A574507D806FBE9
:106F20000117B7EB830F02DA277DB94204D21E2284
:106F3000A7E700BF30020020A0F8C490A0F8C680E8
:106F4000A0F8C8E0A0F8CAC080F8CC7094F816C0C9
:106F5000677D47EA0C27A0F8CE7094F818C0E77D4B
:106F600047EA0C27A0F8D07094F81AC0677E47EA69
:106F70000C27A0F8D27094F81CC0E77E47EA0C27D3
:106F8000A0F8D47094F81EC0677F47EA0C27A0F8D9
:106F9000D670E77F94F820C047EA0C27A0F8D87095
:106FA00094F8217094F8224047EA0424A0F8DA40CB
:106FB000848C8C4211D1C48CB4420ED140F2E24494
:106FC000614342F2107404FB0313013B93FBF1F3A2
:106FD000C18F9BB2994200F0A58090F8F8301C0751
:106FE00040F19A8090F8C230022161F3020380F8E8
:106FF000C23090F8C130013B80F8C130D2F88831FE
:10700000002B7FF4F4ACC2F88801F0E4994204D07C
:1070100090F8C230990740F08E80B4F80C901FFAB7
:1070200089F3052B83D9B4F80E801FFA88F1B1F5E6
:10703000486F3FF67CAF8B423FF679AFB4F810E073
:107040001FFA8EF6B6F5FA7FBFF471AFB4F812C02E
:107050001FFA8CF3A3F10A07BFB240F6764A5745F0
:107060003FF665AF06FB0117B7EB830FBFF65FAFC7
:10707000277DB942FFF45BAFA0F8C490A0F8C680AA
:10708000A0F8C8E0A0F8CAC080F8CC7094F816C088
:10709000677D47EA0C27A0F8CE7094F818C0E77D0A
:1070A00047EA0C27A0F8D07094F81AC0677E47EA28
:1070B0000C27A0F8D27094F81CC0E77E47EA0C2792
:1070C000A0F8D47094F81EC0677F47EA0C27A0F898
:1070D000D670E77F94F820C047EA0C27A0F8D87054
:1070E00094F8217094F8224047EA0424A0F8DA408A
:1070F000848C8C4210D1C18CB1420DD140F2E2415E
:10710000614342F2107404FB0313013B93FBF1F360
:10711000C18F9BB2994205D001232B7090F8C230E9
:10712000032162E7002380F8C33090F8C2300121C8
:1071300003F0F70359E740F65231CF48F9F7BEFAAA
:1071400055E4CE4BD3F8145195F91D30002BC0F205
:10715000A784417A1020FBF7A9FF002800F0A08443
:1071600095F8C02095F8C1309A423FF440AC95F8AC
:10717000C23003F00703042B7FF439ACB4F80CE001
:107180001FFA8EF2052A1ED9B4F80EC01FFA8CF32E
:10719000B3F5486F17D89A4215D8278ABAB2B2F514
:1071A000FA7F10D2668AB0B2A0F10A0189B240F625
:1071B0007648414507D802FB0332B2EB800F02DA72
:1071C000227D934203D21E22102128465AE6002037
:1071D000A5F84400A5F8C4E0A5F8C6C0A5F8C87095
:1071E000A5F8CA6085F8CC20A27D637D43EA02231E
:1071F000A5F8CE30227EE37D43EA0223A5F8D03005
:10720000A27E637E43EA0223A5F8D230227FE37E8A
:1072100043EA0223A5F8D430A27F637F43EA022326
:10722000A5F8D63094F82020E37F43EA0223A5F89E
:10723000D83094F8222094F8213043EA0223A5F8AC
:10724000DA3095F8C230012262F3020385F8C230C9
:1072500007E4417A1120FBF729FF002800F0208481
:10726000864F237BD7F8146196F8F41096F8F52032
:107270008A4227D0162B7FF4BAAB627B232A0ED02A
:1072800096F8383086F8F51096F83910C3F3C20333
:1072900063F30201002386F83910A6F8443096F80B
:1072A000F7309B077FF5A3AB0C232272237196F86E
:1072B0003830C3F3C203637296F83A30C3F3020363
:1072C000A3720CE496F8C11096F8C020914278D0D1
:1072D0000F2B7FF48CAB96F91D20637B002A3ADBE1
:1072E0001A2B38D196F8742096F875309A4204D04B
:1072F0004FF4F3616048F9F7E1F996F8C2300522DE
:1073000062F30203B6F8C620A6F87A20B6F8C820C1
:10731000A6F87C20B6F8CA20A6F87E2096F8782039
:1073200086F8C230012183F00803C3F3C00361F380
:10733000010263F3820296F8753086F88810002007
:10734000013BC6F8840086F8782086F8761086F827
:107350007530FFF786BB232B18D0D7F88831B3429E
:1073600004D04FF4F6614448F9F7A8F90023C7F8B0
:107370008831A6F8443096F91D3096F8C02086F87A
:10738000C120002BBCBFD6F8E430336796F8C2307A
:107390001F077FF52CAB08232371637B2372F28CCC
:1073A000B38CA4F80B20F28FA4F809305A437D2344
:1073B00053434FF47A7293FBF2F3A4F80D30FFF7C6
:1073C0008EBB96F8E82096F8E91091421AD0142B5B
:1073D0007FF40DAB96F8EA3086F8E9206FF382036C
:1073E00086F8EA3000200923A6F8440063721523CA
:1073F000E372338EA381F38D2382F38EE381B38E08
:1074000063822BE5032B7FF4F2AA96F8F83003F0A1
:10741000FB036FF3C303002086F8F830A6F844009E
:107420000D23E372637B237318E5417A1220FBF787
:107430003DFE002800F034831048D0F8144100F5D8
:10744000AE70FAF725FE014600283FF443AC0379FD
:1074500043F00303037101234371132374E4417A5E
:107460001320FBF723FE002800F01A83034BD3F808
:107470001431FFF7BDBB00BF9A1601003002002097
:10748000417A0720FBF712FE002800F00983C34F62
:10749000D7F8146196F8C12096F8C0309A423FD0D0
:1074A00096F8C23043F0100386F8C23096F91D30CA
:1074B000002B09DB96F8742096F875309A423FF459
:1074C0001CAF40F6BF3115E7D7F88831B34204D07E
:1074D00040F6D631B248F9F7F1F80023C7F8883101
:1074E00096F8C03086F8C13096F8C23018077FF59C
:1074F0007EAA082323711A232372F28CB38CA4F87A
:107500000B20F28FA4F809305A437D2353434FF4E4
:107510007A7293FBF2F3A4F80D3001232B7032E062
:1075200096F8E83096F8E9209A4208D086F8E930D3
:1075300096F8EA306FF3820386F8EA30EDE796F8C2
:10754000F43096F8F5209A421AD086F8F53096F87D
:10755000383096F83920C3F3C20363F3020286F889
:10756000392096F8F72091070DD50C2222710022C0
:107570002272637296F83A30C3F30203A372CCE727
:10758000237B122BC9D1D7F81431FFF731BB417AD5
:107590001420FBF78BFD002800F08282142E40F0AF
:1075A00088808048FAF774FD064600283FF492ABC5
:1075B0007A4FE07AD7F8141191F8E8C091F8E9E031
:1075C0000B8E0093E645CB8D01938A8ECB8EBA4607
:1075D00071D1142840F0AF80A0891A2840F284802D
:1075E0008F8D874228BF0746208A1A28009898BFA7
:1075F0008346E08988BF4FF01B0BB0F5A47F75D39D
:10760000B1F83280804528BF8046B4F81290B9F5B1
:10761000A47F6DD3B9F5296F28BF4FF4296900986D
:10762000584567D0FBF792FD0446DAF83001FAF7C7
:107630005DFD0444A4B2FF2C04D940F6D2015848A1
:10764000F9F73CF89AF83A31A34240F04082DAF870
:10765000143193F8E820DF85013A83F8E92093F8A4
:10766000EA20A3F8ECB042F00302A3F8EE70A3F80E
:107670003480A3F8F090A3F8F28083F8EA20032383
:107680008AF81530002E3FF4B2A93379DAF81401E4
:10769000A6F808B043F0030333710923737115236F
:1076A000F371B781A6F80A90A6F80E803146FFF76D
:1076B0004DBB00267CE791F8EA7007F00307012F25
:1076C00087D9022F37D11438012885D940F62711E0
:1076D0003348CDE90232F8F7F1FF039A029B904656
:1076E0009946DDE900B7CDE7019F7DE790468CE73D
:1076F000994694E791F8EA0081F8E9C06FF38200B7
:1077000081F8EA000020A1F844000198B84203D1B2
:10771000424501D14B45B5D00123CF85A1F8369024
:10772000A1F83480A4F80CB02782A4F80E90A4F835
:1077300012802B70A6E71528C8D19046D0E7417A71
:107740001620FBF7B3FC002800F0AA811348037D44
:10775000D0F81451042B5CD195F8F53095F8F4105D
:107760008B4209D095F8F62002F00302013A022A72
:1077700002D82322162128E595F8740095F8752083
:10778000904203D095F87620032A05D195F8C000E1
:1077900095F8C120904207D02A22EBE73002002062
:1077A0009A1601008C03002095F8F6208B4242F0D7
:1077B000030285F8F62018D1013B85F8F53095F8DD
:1077C000F73095F838206FF3410385F8F73095F8D6
:1077D000F630C2F3020262F3840395F83920C2F353
:1077E000C20262F3471385F8F63095F8F630627BF3
:1077F000C3F382010A4062F3840385F8F630227BEA
:10780000DBB202EA531262F3471385F8F630FFF752
:10781000EEB800F5AE70FAF73BFC014600283FF4E5
:1078200059AA95F8F63095F8F5C095F83800022277
:1078300062F3010385F8F63095F8392095F8F430B5
:10784000C0F30200C2F3C2026345C7B2D6B214D17C
:10785000013B85F8F53095F8F7306FF3410385F873
:10786000F73095F8F63067F3840366F3471385F82D
:10787000F630B5F84230A5F8443095F8F630667B1E
:10788000C3F382073E4066F3840385F8F630247B19
:10789000DBB204EA531464F3471385F8F6300B792E
:1078A000087243F003030B7103234B711723CB7151
:1078B0004A72FFF721BA8A4ED6F8145195F91D3055
:1078C000002BC0F2ED80417A1720FBF7EFFB002878
:1078D00000F0E680337D042B7FF489A895F8F5202D
:1078E00095F8F4309A423FF482A895F8F63003F008
:1078F0000302022A7FF47BA843F0030385F8F630E5
:10790000627BC3F382010A4062F3840385F8F63098
:10791000227BDBB202EA531262F3471385F8F6309A
:10792000FFF75EB86E4BD3F8146196F91D30002B4B
:1079300080F2B680417A1820FBF7B8FB002800F0EF
:10794000AF80277B627B47EA020010F0070025D159
:1079500096F8F42096F8F53093423FF448A896F84C
:10796000F63003F00303022B7FF441A896F8F730BA
:1079700086F8F5209A07A6F844007FF538A80C236E
:107980002072237196F83830C3F3C203637296F8FD
:107990003A30C3F30203A372FFF760BAE089738C35
:1079A000C31A1B0441D496F8741096F875308B42B4
:1079B00040D196F8F44096F8F530A34214D096F8EA
:1079C000F63003F00303022B0ED196F8F73086F859
:1079D000F54096F87840C3F3400363F34104002375
:1079E00086F87840A6F8443096F87830A6F87A0001
:1079F00002F0070262F3840367F347136FF3000397
:107A000086F878300820013903F01C0386F87600E8
:107A100086F87510002B3EF4EAAF96F8393062F321
:107A2000020386F83930FEF7E2BF282386F8B33028
:107A3000FEF7DDBF2A23F9E7294ED6F8145195F950
:107A40001D30002B2CDB417A1920FBF72FFB38B3BC
:107A500095F8383095F83A20C3F3C203C2F3020216
:107A60001343227B13423EF4C2AF95F8742095F87D
:107A700075309A427EF4BBAF052206F58D7105F193
:107A80007900FAF7B4F9012385F87830022385F8F4
:107A9000763095F87530013B85F87530FEF7A7BF55
:107AA0000F48E47AD0F8145100F5AE70FAF7F0FA06
:107AB000014600283FF40EA90379047243F0030342
:107AC0000371022343710723C371FFF715B9002E19
:107AD0003FF400A903493046FAF7F3FAFFF7FAB882
:107AE000300200208C0300202DE9F04F95B006F005
:107AF000C3FBC6B266B306F0DFFBC7B206F060FC9C
:107B00005FFA80F906F066FC5FFA80F806F03AFE4C
:107B10005FFA80FA06F024FE5FFA80FB06F01AFC9A
:107B2000C5B2B44C06F092FB06F066FC06F040FCD1
:107B300006F01CFE06F006FC637D052B01F2C583F2
:107B4000DFE813F07D00D0000E00BD09BD09BD09BE
:107B50004FF0FF0B3546B246B1463746D846E0E710
:107B60000123637506F022FD0546962006F054FCBD
:107B7000237D013B032B00F2AF80DFE803F0022FEF
:107B8000636300231A461946184606F0B3FB06F055
:107B9000A1FB06F015FB06F065FB20B140F28F213A
:107BA0009548F8F78BFD05F089FC38B112A805F06F
:107BB0000BFA01469DF8480006F0A6FD0021084694
:107BC00006F017FBC33500210544084606F00DFBFF
:107BD000281A06F0A5FC06F0DBFC30E000231A466C
:107BE0001946184606F086FB94F84121D4F83C313A
:107BF00053F82200083006F0E3FA06F033FB20B118
:107C000040F2B6217C48F8F759FD05F057FC38B131
:107C100012A805F0D9F901469DF8480006F074FD58
:107C20000021084606F0E5FAC33500210544084660
:107C300006F0DBFA281A06F073FC06F073FB15B0A9
:107C4000BDE8F08FD4F8143193F8382093F83A0057
:107C50000021D30900F00700C2F3C20206F04AFB7C
:107C600094F84121D4F83C31D4F8140153F822108F
:107C70000831FBF7B5FD06F0F5FA20B140F2DE2140
:107C80005D48F8F71BFDD4F8143193F83A00012150
:107C900000F0070006F0ADFAD4F8142192F83A305B
:107CA00003F007039B35022B054413D0042B0CBFB4
:107CB0004FF4BC702820054492F83800C109C0F385
:107CC000C20006F092FA281A06F02AFC0120FBF7FF
:107CD000DBFDB4E71820EEE740F215314648F8F72F
:107CE000EDFCACE726B90323637506F09DFAA6E721
:107CF000237D013B032B01F2DE80DFE813F004005B
:107D00009902C105C105002FEDD0BAF1000F39D09D
:107D1000584605F091F98DF8480006F0DBFA94F822
:107D20007920064627212B23007811FB02330A9382
:107D3000E51800F00F03032B0AD173780C2B07D141
:107D400094F829305F061FD594F82930580647D497
:107D5000307800F00F03052BC5D17378222BC2D1E8
:107D60000A9BE35C03F00F03012B40F01B82B71C5E
:107D700012AA3946C0F3801005F044FB00283DD11B
:107D800000204BE0FF20C6E712AAB11CC0F3801010
:107D900005F038FB0028D7D00A9B3278E35CC3F3A8
:107DA0008013B3EBD21FD3D1062206F10801A81C21
:107DB000FAF70DF80028CBD10323637506F0A4FA77
:107DC00094F8C900272303FB00407B3006F0FEF93E
:107DD00006F048FA00283FF432AF40F2BB317DE7AD
:107DE000B9F1000FD8D19DF8480005F04FF90028EF
:107DF000D2D1ADE7300200209A1601003146284664
:107E0000FCF7B6F90028BBD09DF84830FF2B00F0F6
:107E1000B68194F82A00C11A4842484100F0010096
:107E200000283FF460AF94F8823133B194F8803188
:107E300094F881219A427FF456AFD4F8CC30002BCD
:107E40003FF451AF0420FBF797F9074600283FF4B1
:107E50004AAF4FF0040984F8159006F0E5F9D4F81C
:107E6000CC50D4F8081100234FF4AA722846C4F865
:107E7000CC30FAF744F905F1100A2884032206F100
:107E8000120105F11400F9F7B2FF05F117084A468F
:107E900006F10E015046F9F7AAFF052206F11E0170
:107EA0004046F9F7A4FF05214046FAF799FA6B7F9F
:107EB00060F305036B7796F82330C3F30403AB77C5
:107EC000338BAB8440F2E24808FB03F8F27EB37ECA
:107ED00043EA022351464A46EB8405F16C00F9F768
:107EE00086FFB38BE98C42F2107202FB0383013BE5
:107EF000B3FBF8F3EB87C44B4344B3FBF8F3A5F8AB
:107F00004230C24B881D4344B3FBF8F39AB282421D
:107F10001346C4BFC1F57F43FA33A5F84A20C4BF56
:107F2000D21892B22B8CA5F846203146FB80012254
:107F300000233B727A7211F8082B0C934FF006095C
:107F4000C2F3C012FA7587F804904A4607F1180088
:107F5000F9F74DFF9DF8480007F10B03FF280B933D
:107F600007F1110B06F1020A0C9B00F03A810B9A03
:107F700007F10A0105F01CFABB7A0233BB724A46CC
:107F800051465846F9F733FF338BFB83738B3B84A1
:107F9000B38B7B8496F82330C3F3421387F82430E5
:107FA000288CFCF71BFAFCF707F90320FBF7E4F831
:107FB000074620B940F23E419548F8F77FFB2B8CED
:107FC000FB800B233B71337813F020030ED06A7CC7
:107FD0002B7CE97C43EA0223AA7C42EA0122697FE6
:107FE000534041F04001EB83697701233B72FCF77A
:107FF000E3F896F8232095F850308649520962F349
:10800000840385F8503094F8203131F8122031F88B
:108010001330134408FB03F303F574237E4A03F281
:108020003F23B3FBF2F36B654FEA5803963BAB6516
:10803000737D40F2E249002709FB03F3AB66394642
:108040006F66384606F0D3F87449834600F2524012
:108050006BA3D3E90023A0FB0101F8F7A1F8D4F842
:1080600084316B602722934238BF134620F07F4053
:108070009A466B6D2A60E860AF60A8EB030806F0D3
:108080008FFA0B90F08A394609FB0099384606F0C2
:10809000ACF80B9BA9F130099944A9EB0009A9EBB5
:1080A0000B030B9340F28343009305225C4BDFF8F4
:1080B0006CB139463846FAF7EDFE40F28441FCF7E0
:1080C000B1F90A9BE35C03F00F03012B06D1009783
:1080D0003B46032239463846FAF7DCFEA8FB0B89FB
:1080E00047A3D3E9002340464946F8F759F895F8E5
:1080F0002030A4684B4A0733DBB20A9340F29B431B
:108100000893494BCDE90653484B0593EB6853441C
:108110000646049320F07F4007230021434302FBDF
:108120000133A0FB02121A440846B8EB00001146C6
:1081300069EB010100254FF47A7200230395F8F7EB
:108140002FF80B9902902EA3D3E9002326F07F4647
:10815000A1FB0B010196F8F723F8A4EB0A0420F029
:108160007F40009023460A9A29462846FAF7FEFDEA
:1081700030F002033FF463AD40F29D41AEE50A9B4F
:10818000E25C3378C3F38013B3EBD21F7FF4F8AD16
:108190000622394605F10800F9F719FEB0FA80F019
:1081A00040093BE694F82930DB090DD094F82930DA
:1081B000DB093FF4E5ADB9F1000F0DD19DF84800A2
:1081C00004F064FF40B9DBE512AAB11CC0F38010D3
:1081D00005F018F90028E9D031462846FBF7C8FF1A
:1081E0001CE619464A465846F9F72EFE33780B9896
:1081F000C3F38013BB724A465146C3E6AFF3008017
:108200008D49FD1A07000000FF5962027FC3C901B2
:108210009A1601008A16010040420F0000CA9A3BDC
:10822000254400008D49FD1A114400003964000006
:10823000B9F1000F1CD094F8E1004146C0F30010E2
:1082400004F0CCFE804647B194F8E130DA0619D547
:1082500094F8E130DB0600F195800323637505F0A7
:10826000E3FF94F8E0306FF3410384F8E030E6E494
:10827000BAF1000F03D0584604F0DEFEE2E74FF0FB
:10828000FF08E0E7B9F1000F74D100238DF8483002
:1082900094F84121D4F83C3153F82290D4F80031BD
:1082A00009F10806002B78D199F8083013F00F0374
:1082B00002D0062B40F0AE8294F8E120170740F17F
:1082C0009382D4F80021002A40F08E82BAF1000F88
:1082D00014BF4146FF212846FCF73EF80028BCD1D8
:1082E00005F0F8FF0378032262F30303037099F8A3
:1082F00008300278C3F3801363F3C7120C23437072
:1083000005460270404604F04BFE94F8E230014608
:10831000284613F0010F10F8023B00F05C820029A0
:1083200000F0598243F040032B700622F9F75FFDFD
:10833000062209F10A0105F10800F9F758FD94F841
:10834000E03043F0020384F8E030962002236375A6
:1083500006F062F8002005F0C1FF284605F036FF60
:1083600006F016F905F07EFF00283FF468AC4FF4E4
:10837000D361B3E44146504604F0F6FF00283FF4D1
:1083800067AF82E7B9F1000F7FF47FAF404604F09A
:108390007DFE00283FF461AF77E794F8823133B176
:1083A00094F8803194F881219A427FF47DAF94F85B
:1083B000E130C3F30010002800F09F8199F8080015
:1083C00010F00F0040F0D08106F0EAF8D4F8DC306D
:1083D00000F21627D4480722A3FB000102FB031179
:1083E000CDA3D3E90023F7F7DBFEA0F59670874213
:1083F000BFF45AAF0420FAF7BFFE074600283FF447
:108400002CAF042363750023D4F80061C4F8003155
:1084100005F060FF037803F0D00343F025030370F9
:1084200099F80830C3F340128DF83020D2B20D9283
:108430000278C3F3801363F3C71222230546437007
:108440000270404604F0ACFD94F8E23013F0010FE6
:1084500001462B7805F1020000F09281002900F01E
:108460008F8143F040032B70062205F1080BF9F7CA
:10847000BEFC09F10A0106225846F9F7B8FC0422AD
:1084800006F1100105F10E00F9F7B1FC032206F127
:10849000140105F11200F9F7AAFC01236B75B4F879
:1084A000F43040F2E24253430A9306F079F8E3686D
:1084B000D4F80491002BCCBF00F5DB6000F2BA6069
:1084C000B9F1000F40F0678185F8169085F8179094
:1084D00081460021084605F07FFE0021A9EB000936
:1084E000084605F082FEA9EB000909F11E03DFF83A
:1084F0004C920E93B9F8F4302B83B9F8F6306B83B5
:10850000B9F8F830AB8306F11701052205F11E001A
:10851000F9F76DFCB27F95F8233062F3040385F818
:10852000233099F8202162F3471385F8233005F0B2
:10853000EBFE284605F04AFE05F094FE20B140F21D
:10854000CD517A48F8F7BAF84FF4AA72D9F8081161
:108550003046F9F7D4FD4FF00603308429463B71CD
:1085600000233B727B7211F8023BF880C3F3801347
:10857000FB75062207F11800F9F739FC07F10B0328
:108580000B9307F11103BAF1000F00F01481B8F159
:10859000FF0F00F010810B9A0F9307F10A0140467C
:1085A00004F006FFBA7A0F9B0232BA7259460622CD
:1085B0001846F9F71CFCB9F8F430FB83B9F8F6302B
:1085C0003B84B9F8F8307B8495F82330C3F3421329
:1085D00087F82430308CFBF701FFFBF7EDFD03201B
:1085E000FAF7CAFD054620B940F212614F48F8F784
:1085F00065F8338CEB800B232B710D9B002B00F067
:10860000E780727C337CF17C43EA0223B27C42EA4D
:108610000122717F534041F04001F38371770123C0
:108620002B72FBF7C9FD2723D4F884713360D4F88B
:10863000FC30F360002540F23B63272F77604FF05A
:108640000602B560294600932846394BDFF8F0A0B2
:1086500038BF2727FAF71EFC40F23C61FBF7FCFE0F
:108660002B460422294600952846FAF713FC0A9B5C
:10867000A3FB0A89A36896F82040A3EB070B40F2FE
:10868000536308932B4BCDE906632B4B0593F3689B
:1086900040461F44494622A3D3E90023CDE90357AE
:1086A000F7F77EFD104619464FF47A720023F7F76C
:1086B00077FD1BA3D3E90023029049464046F7F714
:1086C0006FFD0E99019016A3D3E90023A1FB0A01C7
:1086D000F7F766FD073420F07F40E4B200905B4678
:1086E000224629462846FAF741FB30F002033FF4C0
:1086F000A6AA40F25561FFF7F1BAB8F1FF0F21D0F9
:1087000094F8E300A0EB080CDCF1000040EB0C0057
:1087100000287FF453AEC7E500CA9A3B0000000072
:108720008D49FD1A070000008D49FD1A9A160100B7
:1087300059440000114400003D6400003002002054
:1087400000CA9A3B99F80820C3F38013C2F3801241
:108750009342DDD1062209F10A01C248F9F737FB3D
:10876000B0FA80F04009D3E701287FF49DAD0023E3
:1087700042463146FBF7A4FD00287FF425AE93E581
:1087800094F8E120B849D20962F386132B700622CF
:108790006BE60A9B9944B9F1000FFADB8145F8D3E7
:1087A00040F2E243A9EB0000B0FBF3F06B7DE882FE
:1087B00001336B758DE6062200211846F9F744FB5C
:1087C0002B780B98C3F3C013BB7206225946F0E610
:1087D0009DF8303024E794F8E120A349D20962F3F0
:1087E00086132B700622A1E5A3B999F80930002B56
:1087F0003FF433ADD4F80031002B7FF42EADBAF145
:10880000000F9DF8482014BF4146FF212846FBF782
:10881000A3FD22E5012B0ED099F8083003F00B02DE
:10882000022AE2D003F00F03072B0DD194F8E130B8
:108830005807DAD111E512AB424631460020FBF76A
:108840003FFD0028D1D1E7E7042B7FF406AD94F873
:10885000E03099077FF501AD05F03CFD99F808304F
:108860000278C3F38013B3EBD21F7FF4F6AC062279
:1088700009F10A010830F9F7AAFA0028B5D0ECE4AA
:1088800094F8183194F84121D4F81451013384F844
:1088900018310026D4F83C318DF8476053F8228017
:1088A000012388F80430002F00F0908295F8F8300A
:1088B00098F8081003F00102C1F38001914200F022
:1088C000738182F0010262F3000385F8F830237DA2
:1088D000032B02BF95F8503043F0010385F8503068
:1088E00095F8F8301A0600F15A81D5F83C6195F8F0
:1088F0005111301D00EB010A9AF80190B9F1000FF7
:1089000000F0A2809B060BD5D5F82AB1D5F82EC170
:108910001BF101024CF10003C5F82A21C5F82E31E4
:10892000435C03F00303032B40F08E809AF803307E
:10893000023B162B00F28880DFE813F017006A0074
:10894000B9008600860086008600860088009A00AE
:108950008600C000860086008600860086008600AD
:10896000CA008600DE00E50001010323637505F0FF
:108970005BFC05F077FC20B140F2DD613B48F7F786
:108980009DFE9AF80410D4F81401132908BF16218B
:10899000FBF766FC0125D4F8140190F85131994495
:1089A00090F850315FFA89F94B4580F8519100F009
:1089B000CD800026002D00F0F780D4F81401FAF7DE
:1089C000B3FF0023C4F8143105F0D6FD18B905F043
:1089D000C7FD05F0CBFDD4F81431002B3FF42FA9CF
:1089E0001EB13146188CFAF723FF9DF84730002B53
:1089F0003FF425A9D4F81431188CFBF7EFFCD4F818
:108A000014311B8CA8F80630FBF7D6FBFFF717B91B
:108A100008220AF10E0105F19400F9F7E8F9D4F8FB
:108A2000140104220AF1160100F58970F9F7DFF943
:108A3000D4F8143193F8F82042F0080283F8F820B3
:108A4000B3F84220A3F844200025A4E795F8F830B5
:108A500043F0480385F8F830B5F84230A5F84430C3
:108A6000F2E700BF1A030020140300209A16010049
:108A7000237D042B1BD1337943F003033371172378
:108A800073710323F371082205F17A010430F9F7B9
:108A9000AEF995F88230337495F88330737406F12B
:108AA00012010C226068FCF737F80026CCE795F835
:108AB000F83043F0080385F8F830C5E795F8F8304A
:108AC00003F0FB036FF3C30385F8F8300023C5E719
:108AD00095F8E82095F8E9309A42B5D095F8EA3053
:108AE00003F00302012AAFD143F00403022262F330
:108AF000010385F8EA30A7E795F8F630022262F321
:108B0000010385F8F630237D032B9DD1AA484FF051
:108B10000433CDE9120395F8F63095F83820C3F305
:108B20008203C2F3C202134314AA134495F83920F6
:108B300013F8083C63F3020285F8392084E795F8BE
:108B4000783095F83920C3F38203F3E7D0F83C314D
:108B5000D0F840114FF0000C8B42A0F850C114D156
:108B6000002E3FF426AFD0F844211968C0F83C111C
:108B7000934212BFC0F84011C0F840C1C0F844C1D0
:108B80008E493046F9F79DFA13E7D0F84821196865
:108B9000C0F83C11934208BFC0F848110AE76FF3D0
:108BA000C71385F8F8300026D4F8143198F8082057
:108BB00093F8F830C2F3C002C3F340039A4240F086
:108BC000CE800320FAF7D8FA002800F0C88094F885
:108BD000823183B3D4F84C31D4F85021934205D17B
:108BE00094F8802194F88111914224D0D4F8502136
:108BF000934200F0B48094F8803194F881219A4235
:108C000000F0AD8094F88031D4F8142123B9B4F881
:108C10007E11138C99420ED094F88031002B00F015
:108C20009E8094F8803104EB4303B3F87811138CE1
:108C3000994240F09480D4F8142198F8095092F8A1
:108C4000F830002D00F0948013F0100508D005F0E6
:108C500033FD20B940F669515948F7F72FFD01253A
:108C6000D4F8143193F8F830D9062CD4D4F8140180
:108C700098F8083090F8F82012F0040F39D100224B
:108C800013F00303A0F84820A0F84C2004D0022BD6
:108C90005ED801238DF84730D4F8143193F8F820CA
:108CA00082F0020283F8F820002D58D0D3F8099101
:108CB000D3F80DA119F101004AF10001C3F809012F
:108CC000C3F80D114BE005F015FD0028CED10323AC
:108CD000637505F0A9FA05F0C5FA20B140F679519F
:108CE0003748F7F7EBFC3D21D4F81401FBF7B8FA4D
:108CF00063E603F003010329E9D190F91DC098F858
:108D00000B10BCF1000F02F0400215DB22B9022962
:108D1000B5D01129DBD809E08A1ED2B2092AF8D8C9
:108D200040F2052C2CFA02F2D207A8D4254A22FAE6
:108D300001F1CA07CBD5A2E72AB902299FD0112990
:108D4000C5D8214AF3E78A1E012A98D90B29F5E7ED
:108D50000DF147014046FDF7C1FD00289CD0D4F835
:108D60001421002384F819319946A2F8403044E0D8
:108D700013F0140F90D0D08CB2F84A10831D994292
:108D8000C4BF8B1F1B1AB2F84600CCBF9BB20B4668
:108D900098421EBFA2F846300023A2F84C30B2F829
:108DA0004C30002B7FF478AFB2F84630A2F8483050
:108DB000A2F84C1070E700BF010102018C030020F3
:108DC0009A160100602002004020020094F8193138
:108DD00013B9022384F8193194F81931013BDBB23D
:108DE00084F81931B5F84060B3FA83F94FEA59199C
:108DF000002E4BD1EB8FA5F84030D4F8140112A906
:108E000090F8F850FDF71CFB637D032B4FEAD51556
:108E100040D0B9F1000F3BD137B198F80830D806EF
:108E200002D4129B5B789BB3D4F8143193F8B3301F
:108E300073BB02239620637505F0EEFAD4F8143163
:108E400093F83A0000F0070005F048FA05F0A0FB9F
:108E5000D4F81401129990F8F8200B78C2F30002AC
:108E600062F3C30390F8F820C2F3400262F3820376
:108E70000B70FAF7EFFD05F0F5F900283FF4A4AD0B
:108E800040F66A61BC48F7F719FC9DE50026B4E797
:108E900003236375237D042B0AD1D4F8143193F88E
:108EA000F82065F3C71283F8F82005F0BDF98BE5CB
:108EB00005F02AFACCE740F63171FEF70FBF227DAC
:108EC000042A00F2FF81DFE812F0F10105004700FB
:108ED00098009800032B09D194F82830590705D041
:108EE000FAF706FE05F09AF9FEF775BE05F056FA98
:108EF000637D032B63D194F8285015F040055ED1B3
:108F0000022212A96068FBF707FEBDF8481040F284
:108F10004712B1FBF2F302FB131340F66B72069299
:108F2000964A01339BB2CDE90452CDE90255CDE911
:108F30000055052229462846ADF84830F9F760FF6C
:108F400030F002033BD0A37C052B38D040F66F7184
:108F50008948F7F7B3FB32E0032B24D1962005F0C4
:108F60005BFA002319461A46184605F0C3F994F82F
:108F70004121D4F83C3153F82200083005F020F9A3
:108F800005F0D0F904F09AFA38B112A804F01CF8F0
:108F900001469DF8480005F0B7FB0123637505F015
:108FA00037F9FEF718BE05F0F9F9637D052B06D1F8
:108FB00000230093042219461846F9F76BFF002599
:108FC00025756575657405F09FFA6D4B2A4629462F
:108FD0002846F9F725F920B141F214216648F7F740
:108FE0006DFB2068436800215B68984701221146A9
:108FF0000020F9F7EDF8FEF722BED4F8140100289E
:10900000DDD090F8B31081B1237D032B03D090F80D
:109010005030DA0709D5FBF723F9D4F81401FAF731
:1090200083FC0023C4F81431C9E7B0F82AB094F8DF
:1090300018710BF10106B6B2002F00F08480237D79
:10904000032B73D105F098FA814605F09BFAD4F80A
:10905000147197F83A3003F00703022BA9EB0009CB
:10906000386E52D0042B0CBF4FF4BC784FF0280858
:1090700000F13003434499450A93DFF808A13CA36B
:10908000D3E9002344D8A0FB0A01F7F789F80A9B2B
:1090900085B2A3EB090036A3D3E90023A0FB0A01A4
:1090A000F7F77EF800233B66BB66D7F83C311FFA22
:1090B00080F8ABB35B7913B997F851310BB100234A
:1090C0007B85D4F8143100229A87D4F81401B0F8C3
:1090D0004030C3B19E4280F0B7809B1B9BB2002200
:1090E000062BA0F84030428540F2B080237D032B50
:1090F00009D1BBF1000F40F0A980C76E7B0817F0C3
:1091000001074BD1C36600274BE04FF01808AFE7CB
:10911000A9FB0A01F7F744F885B208F13000BAE775
:1091200097F85030DB07CCD5FB8CC9E749B190F8F4
:10913000503043F0010380F850304FF000084546AE
:10914000BFE78846FBE7858FF5B1AE4204D2AD1B81
:1091500085873D46A846B8E73E21FBF781F8D4F85D
:109160001401FAF7E1FBC4F8147128E7AFF30080AB
:109170008D49FD1A070000009A1601008D44000079
:109180000C45002000CA9A3BB0F84080B8F1000FAF
:10919000E0D1C38FA0F84030454696E743F0004346
:1091A000C366B0F8443023B19E4251D29B1BA0F855
:1091B0004430B0F84C3023B19E424BD29B1BA0F8F8
:1091C0004C30D4F81421B2F8483092F8741023B11E
:1091D0009E4257D29E1BA2F8486092F875308B428F
:1091E00006D092F87630013B012B9CBF00235385BB
:1091F000538D0FB99B4557D001339BB235B9B8F1A8
:10920000000F03D113B9002F3FF4D9AE92F82020FC
:1092100003930732D6B22F4A06960021CDE9047295
:109220002B46CDE90111CDF8008032460846F9F70A
:10923000E7FD30F002033FF4C2AEA37C9E423FF450
:10924000BEAE41F2DC0183E60821E4E60127A8E78F
:109250002221E0E60023A0F84C300220F9F78CFF31
:10926000814620B941F284011B48F7F727FAD4F868
:1092700014311B8CA9F806300A2389F80430FAF758
:109280009BFF9EE70020A2F84800B2F8440092F845
:1092900075300028A1D19942A3D1072382F87630F6
:1092A0004B1E82F8753098E73B46A7E7043B012B3D
:1092B00004D941F2FB010848F7F700FA002363756F
:1092C000FEF7BDBC41F2021142E641F25E11FEF72B
:1092D00005BD00BFAD4400009A1601002DE9F04124
:1092E0003E4C0A9F9DF818C09DF81C80BDF82C507C
:1092F00020604FF4AA70BDF820E084F82011C4F873
:10930000087100FB03707E190CF1030108F10107DD
:109310000CF1040C08F102085FFA8CFC5FFA88F883
:10932000626084F874810EF10302C4F83C01C9B292
:1093300000EB8C004FEAC8082A2A84F85411C4F8BC
:109340006C0189B240442246A4F834E1C4F87001AB
:1093500088BF0EF10E0E84F8103184F840C199BF19
:1093600001EB410401EB84012EF0030E1EFB01F121
:1093700098BF8900A2F83611B2F836414044342132
:10938000A2F83811C2F82C01B4FBF1F120440CEB27
:109390000304C2F8440100EBC400BDF82440C2F845
:1093A00058010A3424F003044830A4B2FFB2A2F8F2
:1093B000684107FB0404A41B82F83A11C2F860015B
:1093C00003D02C442046BDE8F081012382F882318D
:1093D000F9F7CAFF04F01AFEF4E700BF30020020DC
:1093E000014B1868704700BF3002002038B50321D8
:1093F0000520FAF78FF804210620FAF78BF8214CA4
:10940000002594F81021ABB29A4205F1010532D83B
:1094100094F828306FF3C71384F8283094F8E030BC
:10942000002060F3000384F8E0303422B4F83631D1
:10943000B3FBF2F384F83A3194F8403184F84101F7
:10944000013B84F8750184F8780184F8543194F86C
:109450008031C4F8CC00C4F80001A4F8382184F8A5
:109460004201A4F8760184F8813104F081FBBDE863
:109470003840F9F779BFA81DFF21C0B2FAF74AF8C2
:10948000BFE700BF30020020004870475B020020A9
:1094900000487047AB020020024B93F82800C00937
:1094A000704700BF30020020044B93F92820002AA7
:1094B000BABF93F8290080090020704730020020CD
:1094C000094A92F8E03092F8E100D2F80021C0F3A6
:1094D000C000002A03F0010303FA00F314BF0420C4
:1094E00000201843704700BF30020020054B93F85E
:1094F000E00010F001001CBF93F8E100C0F3011080
:10950000704700BF300200202DE9F04FDFF8908156
:1095100085B0D8F80051019383468A469146464665
:10952000002D40F0B38008F5A470F8F7B1FD0746B0
:1095300050B108F58670F8F7ABFD044630B908F570
:10954000A4713846F8F7BDFD0720D7E198F8E1305F
:109550006BF38613062288F8E130514608F1EA00E1
:10956000F8F745FC019BA8F8F6302946BDF83830DD
:10957000A8F8F8302846A8F8F49004F02DFE4649E3
:1095800000F2524042A3D3E90023A0FB0101F6F709
:1095900007FE4FF6FF7320F07F40C8F8FC002384DD
:1095A00003F59443C4F8A43003230193019B013BCA
:1095B000DBB2042103A8019302F0ECFFDDF80C807C
:1095C0004FF0000A4FEAD8701F23D1464FF0010B2D
:1095D0005246D646013BDBB2FF2B0FD1BAF1000F4A
:1095E00000F0A780CDF80C80A3E0019B002BDDD11B
:1095F00041F208712948F7F761F8D7E728FA03F52F
:1096000005F00105854218D10BF1010C072B5FFA1B
:109610008CFC24D8002845D00132BCF1060FD2B210
:109620002BD8BCF1060F23D1714648460C2972D0C5
:109630008146E34628468E46CCE709F101000E2B11
:10964000C0B200F265810EF10101C9B2072B00F230
:109650007A81002D40F073814FF0010C28E0BCF1BD
:10966000060F00F25E810028DBD1714648462AE0F1
:10967000484671462AE001222FE0714648462FE015
:109680004846DC463CE0013B134351E00C2035E109
:109690008D49FD1A0700000000CA9A3B9A16010086
:1096A00030020020BCF1060F00F23D8171464846B1
:1096B000052B08D88AB1052B05D0012ADBD9042B4C
:1096C00001D0022A09D0BCF1060F22D01C2B20D8D1
:1096D00018B11C2B1DD001281BD1002D00F02581B5
:1096E00001259D40072B28EA050801D8013AD2B28E
:1096F00000258145C4D109F10100C0B24FF0010C31
:109700000E2B04D88E4540F0FC800131C9B24FF0D9
:10971000010A18288AD9BAF1000F01D0CDF80C80BF
:109720005A1C01239340039A002DACD05B42134096
:109730000393039B83F00E4383F4090304A883F48B
:109740003E4383F0D60340F8083D0421F8F748FE75
:1097500001287FF64AAF039B9AB2B2EB134F04D1B4
:10976000DAB2B2EB136F3FF440AF042203A904F165
:1097700010000393F8F73BFB032104F1140002F0FF
:1097800009FF0522744904F11700F8F730FB96F839
:109790001F21637F94F8381062F305036FF386137B
:1097A00063770025B6F8F420A562B6F82231B6F842
:1097B000F600A3851B23E3852386B6F82431638650
:1097C000664B6363B6F82631A28463F3020101237A
:1097D00063F3C50101F0BF0165F3C71184F83810C8
:1097E00094F83910E08463F3020184F83910B6F874
:1097F00028E165846EF3C50184F8391094F83A10B5
:1098000063F30201637F84F83A1094F8501065F313
:10981000C713637701F0DF0140F2E2435A4365F377
:109820000001B6F8F83084F850104FF0060C511EC5
:1098300042F21076A4F81EC0A4F83CC006FB031345
:10984000B3FBF2F3E387464BA4F840501344B3FB59
:10985000F2F3A4F84230434BA4F8445000EB0C015F
:109860001344B3FBF2F39AB28A421346C4BFC0F565
:109870007F43FA33A4F84A20C8BFD21894F8A8301E
:10988000C4F8B4704FF0000503F0FE0365F3410324
:1098900084F8A83094F8C230A4F84C5065F304134F
:1098A00084F8C23094F8EA30A4F8485065F3820393
:1098B000C8BF92B284F8EA30A4F84620A4F87450E5
:1098C000A4F8B05084F8B350A4F8C050A4F8E850FD
:1098D000A4F8F45084F8F850C4F83C51C4F840514E
:1098E000C4F84451C4F84851C4F84C51A4F850513C
:1098F000FBF71EF91C4B2846C3F8004105B0BDE834
:10990000F08F18283FF60AAF71464FF0010A8FE634
:1099100071469BE60121994028EA0108002571461D
:10992000E9E60028F6D17146484601259D40072BFF
:1099300048EA050801D80132D2B20125D9E6013240
:10994000D2B2AC46C2E615B94FF0010CBEE61C2BF4
:10995000AC463FF6DEAEBCE64A03002048014801B3
:10996000FF5962027FC3C901300200202DE9F8438C
:109970000C4690469946BDF82070BDF82460BDF8AD
:109980002850F9F7B1FD002868D094BB90F8C23098
:10999000D90607D490F850309A0629D5D0F8A430CB
:1099A0009B0725D490F91D30002B55DB90F87430BF
:1099B00090F875209A4251D190F87830A0F87A70DA
:1099C0000124002164F3010361F38203224480F83F
:1099D0008840C0F88410A0F87C60A0F87E5080F821
:1099E000783080F8764080F874200020BDE8F88355
:1099F0000124013C14F0FF0490F8C01090F8C1203D
:109A000011D091422AD090F8C23003F00702032A05
:109A100024D164F30203DBB243F0080380F8C3806F
:109A200080F8C230E1E7914218D190F8C23080F856
:109A3000C34064F30203DBB243F008030131A0F832
:109A4000C490A0F8C670A0F8C860A0F8CA5080F80A
:109A5000C23080F8C010C8E71A20C7E70C20C5E75D
:109A60002DE9F0411E4C01460522054604F58D7096
:109A7000F8F7BDF904F58D700521F8F7B1FC84F80D
:109A80001F0194F81041013CE4B201274FF0020895
:109A9000FF2C02D10020BDE8F0812046F9F724FD1B
:109AA0000646B8B190F91D30002B13DB90F87420F6
:109AB00090F875309A4210D1052229467930F8F78E
:109AC00096F996F8743086F87870013386F87680C7
:109AD00086F87430013CE4B2DAE70120DBE700BF2E
:109AE00030020020F8B50D46F9F7FEFC044660B1DF
:109AF000002700F117062777052231462846F8F798
:109B000076F9207F0028F6D1F8BD0120FCE770B57A
:109B10000D461646F9F7E8FC044608B9012070BD69
:109B200015B390F8F80010F0400010D194F87420AC
:109B300094F875309342F1D10322013384F87950BF
:109B400084F8780084F8762084F87430E7E794F895
:109B5000B12094F8B0309342E0D1013384F8B25090
:109B600084F8B0300020DAE7102231468430F8F76C
:109B70003EF994F8742094F875309342CED10322C4
:109B80000133A4F8785084F8762084F8743028469D
:109B9000C5E708B5F9F7A8FC68B190F8742090F80B
:109BA0007530934207D10422013380F8762080F883
:109BB0007430002008BD0120FCE708B5F9F794FCDB
:109BC00068B190F8742090F87530934207D105225F
:109BD000013380F8762080F87430002008BD012021
:109BE000FCE710B50C46F9F77FFC60B190F8B120A6
:109BF00090F8B030934206D1013380F8B24080F83B
:109C0000B030002010BD0120FCE710B51446F9F774
:109C10006BFC10B10020207010BD0120FCE710B5D6
:109C20000C46F9F761FC60B1838CB0F84A205A43C6
:109C30007D23534300204FF47A7293FBF2F3238089
:109C400010BD0120FCE710B50C46F9F74DFC70B1D2
:109C5000828C40F2E243534342F2107101FB043420
:109C6000013C94FBF3F4A0F84A40002010BD012011
:109C7000FCE770B50E461546F9F736FCD0B190F802
:109C8000742090F875309A4214D190F8E82090F83A
:109C9000E93093420ED190F8EA40A0F8EE606FF3FD
:109CA0000104013380F8EA40A0F8F25080F8E8306F
:109CB000002070BD0120FCE7034BB3F82221028095
:109CC000B3F824310B80704730020020034BA3F817
:109CD0002201A3F824110020704700BF30020020A9
:109CE00010B51B2404804FF429600880148018806C
:109CF00010BD38B50D461446F9F7F6FB58B190F88B
:109D00003830C3F3C2032B7090F83A30C3F3020328
:109D10002370002038BD0120FCE70000034BA3F8AE
:109D20002601A3F828110020704700BF3002002050
:109D30002DE9F843894690461F46F9F7D5FB20B335
:109D400090F8742090F875309A421ED190F8F43053
:109D500090F8F5509D4218D190F8F64090F8F760D1
:109D600004F0FC0469F3840446F00201224668F31F
:109D7000000167F34712013580F8F71080F8F620EC
:109D800080F8F4500020BDE8F8830120FBE70000D4
:109D90002DE9F341054608461849D1F84C31D1F870
:109DA000502193420F461FD0D3F8048001F277115F
:109DB00098F80020F9F74EFB0446E0B902AE97F898
:109DC000773106F8033D97F8782131460DF106000A
:109DD000F9F740FB34B928B9C5F80080204602B035
:109DE000BDE8F0810446EEE791F8782101F27711A1
:109DF000F9F730FB044600232B60EFE73002002028
:109E0000914210B5144B19D1D3F85021D3F84C41DD
:109E1000944211D1002914BF0A460322013AD2B25A
:109E200003EB420483F8812193F88021A4F87A019E
:109E300091420FD083F88111012005E029B9B3F8D0
:109E40007E31181A18BF012010BD03EB4103B3F88F
:109E50007831F6E70020F7E73002002030B4144BE9
:109E600093F882210D4602B393F88021D1B293F882
:109E7000812135B14FF6FF73984216D030BCFFF701
:109E8000BFBFD3F84C01D3F85041A0420DD191424D
:109E90000BD0D3F8504183F88111A04205D093F83C
:109EA0008001884208BF83F88121002030BC7047C0
:109EB000300200200148F8F7EBB800BF94030020FF
:109EC0000149F8F7FEB800BF940300202DE9F041E6
:109ED0002E4C94F8765194F87431013588B0EDB277
:109EE00080460F46AB4208BF0025F9F7FDFA06464B
:109EF000002848D094F87531AB4244D0B4F86831AA
:109F00007A79073B9A4204D942F696512048F6F7EF
:109F1000D5FB94F87621D4F86C3103EBC20123F819
:109F200032804F6084F8765196F91D30002B03DBA8
:109F3000002008B0BDE8F081738D002BF8D096F8B2
:109F4000503013F00204F3D143F0020386F850308E
:109F500096F820200F4B0696CDE9044307320123E3
:109F6000CDE90243CDE900442346D2B20321204685
:109F7000F8F746FF30F00203DAD042F6A951044860
:109F8000F6F79CFBD4E70120D3E700BF30020020A6
:109F90009A160100AD3200002DE9F84307468846C5
:109FA00016469946F9F7A0FA054610B90120BDE812
:109FB000F88390F8742090F875309A42F6D1FFF744
:109FC00079FF04460028F1D01022494605F18400AB
:109FD000F7F70DFF95F8F83013F0300324D123790B
:109FE00043F0030323711723082263710323E371F2
:109FF0004146A018F7F7FBFE337823747378637437
:10A00000082104F1120002F0C5FA042104F11A003B
:10A0100002F0C0FA21463846FFF758FF0126D0B1BA
:10A020002046FFF74DFFC1E7302BF9D1082241460A
:10A0300005F17A00F7F7DBFE337885F88230737824
:10A0400085F88330237943F003032371012363717F
:10A050000A23E371DEE7032385F8763095F8743040
:10A0600085F87860013385F87430A0E700000000BF
:10A070002DE9F04FCA4F8FB09A4602230D9397F9FE
:10A0800028308DF82F20002B834688463D4601DA84
:10A090000C207BE197F87A202B234FF0270919FB3E
:10A0A000023917F8093003F00F03012B00F2278162
:10A0B000D7F8CC60002EEBD107F5A470F7F7E8FFD6
:10A0C0000A9058B107F58670F7F7E2FF0A9A04463E
:10A0D00030B907F5A4711046F7F7F3FF072055E1F3
:10A0E0004FF6FF73038403F59443C0F8A430437F15
:10A0F000866266F386134377B7F8223183851B2384
:10A10000C3850386B7F824314386A64B4363B7F86B
:10A11000261190F83830C67761F30203012161F30C
:10A12000C50366F3861366F3C71380F8383090F8DA
:10A130003930468461F3020380F83930B7F82801DA
:10A14000A4F8406060F3C50384F8393094F83A30DD
:10A15000A4F8446061F3020384F83A30637F43F06B
:10A16000800363770623A38794F8503066F3451382
:10A1700066F3000366F3410384F85030C4E91766C0
:10A18000A4F84C6094F8A830A4F8486066F3000383
:10A1900066F3410384F8A83094F8C230266766F36A
:10A1A000041384F8C23094F8EA30A4F8746066F3BB
:10A1B0008203A4F8B06084F8B360C4F8B420A4F8B3
:10A1C000C060A4F8E86084F8EA30A4F8F46084F889
:10A1D000F860C4F83C61C4F84061C4F84461C4F854
:10A1E0004861C4F84C61A4F85061FAF7A1FCC7F8C3
:10A1F000CC400EA895F8293010F8092D6BF3020316
:10A2000062F3C5036AF3871385F829309DF860303F
:10A2100085F82A30D5F88431EB612723AB61012121
:10A2200000232B62F8F7DCF817F8096006F00F0638
:10A23000012E66D14FF42773584300F59C705A499C
:10A2400055A3D3E90023A0FB0101F5F7A9FFD5E948
:10A2500006739F42686238BF1F46B8F1000F58D19D
:10A26000721E5342534195F82860DFF85091DFF891
:10A2700050B163F3861685F8286016F040060DF19C
:10A28000340A4ED0F8F7CEFE6B6A06461F44002013
:10A29000CDE9079ACDE905B0CDE90307CDE9017015
:10A2A0000090334605220321F8F760FD022834D0E0
:10A2B0000D98B8B902230D933C4B0690CDE9079A4F
:10A2C000CDE90200CDE9040303224AF2FE330093F4
:10A2D000019033461146F8F749FD022843D00D9806
:10A2E000002844D0002C3FF4D3AED4F8B400304959
:10A2F000F7F7E7FE2F492046F7F7E3FEC8E600240C
:10A3000077E7022E0CBF4FF4297340F2FC535843F9
:10A3100095E70023A7E7F8F7C5FE0D9B022BFAD0BF
:10A32000C6E7F8F77FFECDE9079ACDE905B60A90B2
:10A330006B6A214802961FFA88F81F44A8FB0001A7
:10A34000912303FB081114A3D3E90023CDE903678C
:10A35000F5F726FF0A9BCDE9006005220321304670
:10A36000B9E7F8F79FFE0D9B022BFAD0B7E795F8F7
:10A37000283043F0800385F8283095F8E03013F05A
:10A38000010403D1012003F0F5F920460FB0BDE828
:10A39000F08F00BFAFF300808D49FD1A0700000069
:10A3A000300200204801480100CA9A3BD94A000007
:10A3B000780300203C030020002AE784E9300000F5
:10A3C000FD49000070B503210520F9F7A3F8054603
:10A3D000E8B9104C94F8282060F3C71284F82820BC
:10A3E00094F8E020D30701D403F0C4F9D4F8CC608A
:10A3F0005EB100230849D6F8B400C4F8CC30F7F7B2
:10A4000060FE06493046F7F75CFE284670BD0C2515
:10A41000FBE700BF30020020780300203C0300204F
:10A420002DE9F047684C94F8E0508EB01F4615F0C7
:10A4300001054FF002030E460B93114603D00C208A
:10A440000EB0BDE8F08794F8E13094F8E22060F3B4
:10A45000C303400860F302039DF8600060F300024C
:10A4600084F8E2209DF8642084F8E32066F3C713A3
:10A47000062204F1E40084F8E130544EF7F7B7FC0B
:10A48000BDF858204FF09109A2FB060109FB02110B
:10A490004BA3D3E90023F5F783FE94F8E1309DF850
:10A4A0005C20D4F88481C4F8F00062F30513BAB2DA
:10A4B000A2FB066709FB027784F8E130272300F14D
:10A4C000090AC4F8D480C4F8D030C4F8D8503CA3EA
:10A4D000D3E9002330463946F5F762FEA0F12703A1
:10A4E0009A4594BFC4F8DCA0C4F8DC30B8F1270F5B
:10A4F000814638BF4FF02708F8F794FDD4F80031B3
:10A500008246002B45D00C950C9831492CA3D3E9F9
:10A510000023A0FB0101F5F743FE0BAB08932D4B85
:10A5200007932D4B0593D4F8DC30002520F07F40B5
:10A5300043448244CDE90353304621A3D3E90023A9
:10A5400039460695F5F72CFE104619464FF47A72F7
:10A550000023F5F725FE0095CDE90190534606222C
:10A5600003212846F8F702FC022823D00B9D002D7A
:10A570007FF465AF94F8E03043F0010384F8E030F5
:10A5800094F92830002B02DB022003F0F3F8284670
:10A5900056E7D4F8DC100D930DAA0CAB4144032010
:10A5A000F9F7EAFC0C9B002BAED0DDF834A0ABE74A
:10A5B000F8F778FD0B9B022BFAD0D7E7AFF30080BA
:10A5C0008D49FD1A0700000030020020002AE784B0
:10A5D00000CA9A3BE9300000454A000010B504214A
:10A5E0000620F8F797FF0C4C70B9D4F800215AB93F
:10A5F00094F8E03062F3000384F8E03094F92830F6
:10A60000002B01DB03F0B6F894F8E03013F0010FF3
:10A6100014BF0C20002010BD3002002018B1044BE4
:10A62000D3F800310BB9FFF7D9BF0C20704700BF3A
:10A6300030020020F8B5104ED6F800310746CBB1F5
:10A64000FFF7CCFF054698B9D6F8004106F5A4718E
:10A65000D4F8B400F7F735FD062384F8B8304FF688
:10A66000FF73A4F8BA30022384F8BC30B4343C60E1
:10A670002846F8BD0C25FBE73002002037B5414CD9
:10A6800002AA002342F8043DD4F8500104F5A67153
:10A69000F7F766FD054620B942F65C413A48F6F701
:10A6A0000DF83A492846F7F70CFD019B1A790C2A58
:10A6B00007D80123934041F67E72134207D11A0650
:10A6C00016D442F693413048F5F7F8FF10E094F8BD
:10A6D000403194F85421013B9A4204DB42F689410F
:10A6E0002948F5F7EBFF94F85431013384F85431DD
:10A6F000019B1A79062A36D11A7A3C2A11D05B7A44
:10A700009BBB94F8E030DB0704D442F6A8411E4816
:10A71000F5F7D4FF94F8E0306FF3000384F8E030ED
:10A7200014E00023D4F8CC50C4F8CC3094F928308D
:10A73000002B04DB42F6A5411348F5F7BFFF94F860
:10A7400028306FF3C71384F8283085B994F8E000F7
:10A7500000F0010394F82800C0F3C01050EA430051
:10A7600001D103F007F803B030BD0025DEE7D5F8CE
:10A77000B4000649F7F7A5FC05492846F7F7A1FC00
:10A78000E4E700BF300200209A16010078030020A1
:10A790003C0300202DE9F843244CDFF8988006465E
:10A7A000006804F5867728B93060FF20BDE8F843DB
:10A7B000F8F78EBD0279D0F800900C2A2FD801232B
:10A7C000934041F63E751D4025D15A060AD41B061A
:10A7D00025D5C288D4F808014FF4AA71F7F78CFC8C
:10A7E000394619E0037A022B15D1D4F80001C4F8D8
:10A7F00000513946F7F765FC94F8E03065F3000343
:10A8000084F8E03094F92830002B02DB284602F06F
:10A81000B1FF4846C7E70649F7F753FCF9E742F6A8
:10A8200011514046F5F74AFFF3E700BF3002002020
:10A83000600300209A16010038B50B4CD4F8402173
:10A84000D4F8445122B10020C4F84001F8F77CFA52
:10A850002DB10023C4F844310120F8F775FA002027
:10A86000BDE83840F7F72ABD00B000400120F7F7F7
:10A8700025BD684620F007018D4601B5F7F770F950
:10A8800003F0A8FBF7F75EF9F6F72AFFBDE80140F1
:10A890008546704770470000014B186805F041BEBF
:10A8A0008424002010B5374B86B01860364805F078
:10A8B00077F918B96FF0120006B010BD4368012196
:10A8C0001B689847314805F06BF904460028F1D021
:10A8D00003F0D6F9F7F752FC2D4B08221A70032229
:10A8E0001A7202221A7600202A4A187405922A4AFD
:10A8F00004922A4A03922A4A02920D22CDE900329A
:10A9000017210423274AF8F7E3F918B19E212648B6
:10A91000F5F7D4FE254805F043F90028CAD041F6E2
:10A9200004230593224B04931B23CDE90233072113
:10A930000623CDE9003122461023FEF7CFFC044662
:10A94000E0B9012003F014F9224621460120F7F76F
:10A95000DFF8224621460B20F7F7DAF82246214697
:10A960001820F7F7D5F80120F7F7A0F80B20F7F734
:10A970009DF81820F7F79AF820469DE76FF00B0036
:10A980009AE700BF84240020841101005B110100BC
:10A990006424002005E9000079E800004DE800008B
:10A9A000F42100205C1E0020E11601008F1101003F
:10A9B0005804002008B50248F7F7FEFA002008BD49
:10A9C00028170100838937B505461BB3037D8BB17A
:10A9D000022B1FD101A901F01FF90446019808B10B
:10A9E000F7F71CFB1CB9284604F04CF8002420465D
:10A9F00003B030BD02A941F8043D00F01FFB002860
:10AA0000F1D0F7F70BFB01990029ECD0034805F0D2
:10AA1000E3FAE8E76FF01504E9E700BFBC47002060
:10AA200013B50190081E03DB022807DD032822D09E
:10AA30008B211648F5F742FE00240DE001280EBFD9
:10AA400000214FF0FF310120F7F7C8FA044618B192
:10AA50000146019801F094F9019B0021D888FFF785
:10AA6000FDF902A8002250F8043D1A60FFF792FE9B
:10AA7000204602B010BD4FF0FF31F7F7AFFA0446A1
:10AA80000146019801F026F9E6E700BF3C170100F6
:10AA9000F7B5144D144E0DF1020101A8FFF778F936
:10AAA000044640B9019BBBB1FFF7E8FD0199304670
:10AAB00005F092FAEFE74FF0FF310120F7F78EFA39
:10AAC00022460746BDF8021001F030FD3846F7F780
:10AAD000A5FA05F0EDFCDEE74FF0FF31284605F062
:10AAE00047FDD8E790470020BC470020044B18687A
:10AAF00028B1596802681A60884208BF5A607047D6
:10AB00008C24002010B5154886B0FFF7CBFE044614
:10AB100000BB134801F036FD6FF00903CDE9024395
:10AB20004FF4E0720F4B10491048CDE90444CDE9D1
:10AB3000004405F0C7FD6FF00703CDE90243CDE9FE
:10AB40000444CDE900440A4B0A490B484FF4007213
:10AB500005F0B8FD204606B010BD00BF90470020AC
:10AB60003446002091AA0000E0330020682C002029
:10AB70007DAB0000A0350020FC2B00202DE9F74F15
:10AB8000694E37464FF0FF320221304606F0CEF8CC
:10AB900020B140F231116548F5F790FDF36803F4F8
:10ABA000F833B3F5805F05D13269002393604FF02D
:10ABB00000090AE0336A03F4F833B3F5804FF6D1A5
:10ABC0000021706A05F02CFA8146FA686FF31032A2
:10ABD000FA603A6A6FF310323A62554A1568554A7C
:10ABE000BFF35B8F52E8001F21F0010342E8003001
:10ABF0000028F7D1BFF35B8FCA0748BF4E4A4F4CBE
:10AC000044BF0021C2E90011002D06DC4FF0FF32E5
:10AC10002260B9F1000F21D16BE0DFF828B1DFF835
:10AC200028A1DBF80020444BDAF800101B680193E0
:10AC3000AA1A0A442260002BEBD0184601F08AFCC5
:10AC40008046B9F1000F18D0022803D0032805D19F
:10AC500022681AB100213A4806F0FAF8484601F095
:10AC600079FC21684B1C05464AD0334A1068032DF5
:10AC700051D8DFE805F045453441022808D00328C3
:10AC800004D0FD212948F5F719FD03E0236883B3BB
:10AC9000FFF72CFF41460198FFF7C2FEDBF80030BA
:10ACA000ED1ADAF800301D44234B25608146186800
:10ACB00058B101F04FFC022803D0032805D12368C6
:10ACC0001BB100211E4806F0C3F8B9F1000F10D0E7
:10ACD000B9F80C3048461BB3F7F796F909E00121A3
:10ACE000216068B10021C9F80010516871B9C2E94A
:10ACF000009905F0DDFB45E70028F3D10029F1D0EC
:10AD000048462946FFF78CFE8146DEE7C1F80090F1
:10AD1000C2F80490EDE7B4210448F5F7CFFCEFE763
:10AD200003F0B0FEE5E700BF0C4600203C17010031
:10AD3000F42C0020FC2C00208C24002088240020EF
:10AD400034460020F82C0020002D0020C0F30723FB
:10AD50000870000C8870000A4B70C870704738B5D6
:10AD600008300D460221144603F0BAFE0570447007
:10AD700038BD000038B505464FF0FF30F7F738F919
:10AD8000042204460F21FFF7EAFF042104F1080022
:10AD900003F0A6FE01234370024B05701B8843801D
:10ADA000204638BD9424002038B504464FF0FF30CB
:10ADB0000D46F7F71DF9EA1C2060D2B20E21FFF70D
:10ADC000CEFF20680321083003F08AFE01230370C0
:10ADD000054B1B88A0F80130206829460830BDE8E3
:10ADE000384003F07DBE00BF9424002070B50446B7
:10ADF000154601320E460834D2B23E21FFF7AFFFAE
:10AE00000121204603F06CFE067029462046BDE86D
:10AE1000704003F065BE00000F4B70B51546D3E9D6
:10AE2000002304460E4602F08000002150EA010390
:10AE300010D0042208212846FFF791FF042105F1D4
:10AE4000080003F04DFEB4FA84F35B090470A0F827
:10AE50000160C37070BD00BF484600202DE97848EE
:10AE600004461846154B1646D3E900234FF0000B55
:10AE700003F0005C5BEA0C030D461DD0104BD3E9D8
:10AE800000234FF0000C02F0080B5BEA0C0313D018
:10AE90000B220421FFF7AAFF08220470A0F801602A
:10AEA000033024B9291DBDE87848F6F7A0BF00217A
:10AEB000BDE87848F6F7C8BFBDE878884846002066
:10AEC0005046002070B503788AB004460E4607ADA0
:10AED000032B20D8DFE803F002191B1D1149284677
:10AEE000F6F75EFF62780492A2780392E27802920B
:10AEF0002279019262790092A37905950A4A1B2171
:10AF00003046F6F74FF80AB070BD0849E7E7084940
:10AF1000E5E70849E3E7084A0A212846F6F742F838
:10AF2000E0E700BF9D170100C6170100A41701004C
:10AF3000AB170100B5170100BF17010010B503786A
:10AF400003F00F02072A8AB016D14278A2B18278A4
:10AF5000910611D0C278D2070ED50AACC3F3801384
:10AF600004F8243D011D06220DF10500F6F73FFF10
:10AF700003A92046FFF7A6FF0AB010BDF8B5224B83
:10AF80004FF0FF321A60214B4FF0FF3641F6FF774A
:10AF9000C3E900671E4B00260027C3E900671D4B6D
:10AFA0001F2600270C46C3E90067054638B1FEF7A7
:10AFB0001DFA01212046FFF7F7FE00230370164B10
:10AFC000164800241C60164B1C60164B202221469C
:10AFD0001C60F6F739FF144B1C609DB1BFF35B8F0B
:10AFE000124B53E8002F42F0010243E800210029F0
:10AFF000F7D1BFF35B8F0E4B21461868BDE8F840D0
:10B0000005F026BFF8BD00BF9C2400204846002064
:10B010002825002050460020F42C0020D42C0020AD
:10B02000F82C0020002D002098240020FC2C00206B
:10B03000302500200346006859687047F0B50E4679
:10B04000818993B00025022904460C9502D800207E
:10B0500013B0F0BD8368B34F1A7858789B7842EAF2
:10B0600000228B423A80F2D8032104F1080003F059
:10B0700046FD3B88C3F309029B0A042B00F02281A2
:10B0800009D8012B26D0032B3AD001210CA8FFF7B9
:10B090008BFE01235BE0082B00F0C9813F2BF4D12C
:10B0A000013A092AF1D801A353F822F029BA000085
:10B0B00059BA000083BA00008BB000008BB00000CA
:10B0C000D1BA00008BB000009BBA0000DDBA0000CE
:10B0D0004BBB0000062A06D01D2AD6D1A3681888CB
:10B0E000FEF76BFD04E0A36899781888FEF779FDF8
:10B0F000002814BF0C200020FFF73CFE0C9052E00B
:10B10000332A00F08C8024D8032A48D00DD8012A95
:10B11000BBD1A068FFF78EFF834BC3E9000101217B
:10B120000CA8FFF741FE002311E02D2A49D0312A57
:10B13000ABD1A3687D4C1D7801210CA8FFF734FE2C
:10B1400023681BB17A4A1268002A50D00C2303707E
:10B1500029E0632A29D00AD8352A96D1734B1B6877
:10B16000002B6DDC01210CA8FFF71EFEEEE77B2A09
:10B1700000F091807C2A88D1A3681C8859882046D9
:10B18000FEF761FD054603210CA8FFF70DFE002D1B
:10B1900014BF0C2300230370A0F8014003E00CA9A6
:10B1A0002046FFF7EBFE0C9852E7A068FFF742FF3E
:10B1B000604BC3E9000101210CA8FFF7F5FD057004
:10B1C000F1E7A36804210CA81D889F78FFF7ECFD28
:10B1D000AEB20446C21C39463046FEF716FD0028C2
:10B1E00014BF022300232370A4F80150DBE7027090
:10B1F0001DB1012D10D01223A9E7002BD3DB4E4B3C
:10B200004E48002119604E4B20221960F6F71CFEB3
:10B2100023685B422360C6E7002BC4DCEFE7A3682A
:10B2200001210CA8B3F803401D88FFF7BDFD3F4B7B
:10B230001A68002A8AD11A2DDDD964421C60B2E74F
:10B240003B4B1B68E3B1A5683C4E2F7800231946A1
:10B25000BB4209DB3A4A13680B441360394B0021A7
:10B26000186805F0F5FD9EE705EB8302B2F8014092
:10B27000B2F803000F2C03D836F81420904204D9FA
:10B2800001210CA8FFF790FDB5E7121A26F814204B
:10B2900001440133DCE7A3681C880DA92046FEF7B2
:10B2A000BEFC052105460CA8FFF77EFD002D14BF4E
:10B2B0000C2300230370A0F80140BDF83430A0F83F
:10B2C000033070E7013A082A3FF6DFAE01A353F8D6
:10B2D00022F000BFF9B2000049B30000FBB3000048
:10B2E0008BB000008BB000008BB000008BB0000072
:10B2F0008BB0000017B4000009210CA8FFF754FD23
:10B30000002303708370C3706FF00E034371052335
:10B31000092283714FF0FF3342700271C3710372CF
:10B3200041E700BF9424002048460020F42C002070
:10B330009824002028250020F82C0020D42C002060
:10B34000002D00203025002041210CA8FFF72CFD06
:10B3500000210446402200F8011BF6F775FDE37852
:10B360006278617F94F8210063F07F03E370A37932
:10B3700063F03F03A371E37A63F01B03E372E37BA3
:10B3800043F02803E373237C43F002032374E37D3B
:10B3900043F00403E375A37E63F00803A37642F051
:10B3A0002002FF23E3766270237794F8222084F84A
:10B3B000243094F8283062F00F0241F07F0143F00E
:10B3C000040384F82220617794F8232094F8251050
:10B3D00084F8283094F8273040F0300041F0010123
:10B3E00062F0060263F07F0384F8210084F82510E0
:10B3F00084F8232084F82730D5E609210CA8FFF72C
:10B40000D3FC00210446082200F8011BF6F71CFDBE
:10B4100060236371C7E607210CA8FFF7C5FC01464E
:10B42000002301F8013B1846F7F702FEBBE6013A9C
:10B430004D2A3FF62AAE01A353F822F075B500005D
:10B440007FB5000097B500008BB00000BBB50000D1
:10B450006BB6000039BB00009BB60000A7B6000029
:10B46000B3B60000D1B60000E9B6000009B700008D
:10B4700033B70000D1B50000E7B50000F9B5000012
:10B4800001B6000095B700003BB7000071B700009F
:10B490008BB7000009B600002FB6000043B70000CC
:10B4A00057B7000067B7000045B60000DFB90000DD
:10B4B000EDB90000FDB90000B3B70000DDB7000032
:10B4C000EDB70000FDB7000015B800008BB000001C
:10B4D0008BB0000025B9000033B900003BB9000073
:10B4E0004BB900005DB900007BB9000099B90000BC
:10B4F000AFB9000031B8000055B80000ABB800008B
:10B50000C9B800001BBA000023BA00008BB00000CD
:10B510008BB000008BB000008BB000008BB000003F
:10B520008BB000008BB000008BB000008BB000002F
:10B530008BB000008BB000008BB000008BB000001F
:10B540008BB000008BB000008BB000008BB000000F
:10B550008BB000008BB000008BB000008BB00000FF
:10B560008BB00000C5B900008BB000008BB00000AC
:10B57000BBB90000A068FFF75DFDB34BCDE504212A
:10B580000CA8FFF711FC002303701B228370072314
:10B590004270C37007E609210CA8FFF705FC0021E3
:10B5A0000446082200F8011BF6F74EFCFF236370E7
:10B5B0004923A3700123E370F5E5A1680120F7F7A3
:10B5C00051FD044601210CA8FFF7EEFB0470EAE5EB
:10B5D00002210CA8FFF7E8FB00230370044601F0EA
:10B5E0007DFD6070DFE501210CA8FFF7DDFB04465F
:10B5F00001F076FD2070D6E5A06801F05DFEE0E781
:10B60000A06801F0A9FDDCE7A06800230DAA00F105
:10B61000100102F0A5FB11210CA8FFF7C5FB0023C8
:10B6200000F8013B10220DA9F6F7E1FBBBE509216B
:10B630000CA8FFF7B9FB002300F8013B082100F03C
:10B64000A9FFB0E509210CA8FFF7AEFB01460023D6
:10B65000024601F8013B6FF44000FFF777FB40F230
:10B66000FF30511DFFF772FB9DE5A06800210379B3
:10B670000288CDE90911CDE90711CDE90511847BD7
:10B680000494447B0394C41D02948479019440790A
:10B690000090084600F0A2FF93E7A368591C1878B1
:10B6A00001F0A6F83BE5A368591C187801F0F8F8FA
:10B6B00035E5A368187801F039F9044601210CA892
:10B6C000FFF772FB002C18BF0C2308BF00233EE5D8
:10B6D000A4686379B4F80320B4F801102078A47941
:10B6E000009401F0A1F9E8E7A268584B107840B146
:10B6F000527832B100221A60554B1A6001F0B4F949
:10B70000DBE74FF0FF32F8E7A468B4F81350637931
:10B710002279618820880495B4F811500395B4F813
:10B720000F500295257B01950634009401F0DAF95B
:10B73000DEE43046FEF77EFFBFE7A068FEF790F933
:10B74000BBE7A06800F10C0300F10A02811C00882D
:10B75000FEF722FCCCE4A26832F8024B002120461E
:10B76000FEF7D5F90EE5A36800221C880621F6E74E
:10B77000A36808210CA81D88FFF716FBAEB204468B
:10B78000C11C3046FEF7AEF929E5A3681888FEF71C
:10B7900000FAADE4A2681189538810880291D1881B
:10B7A00001919288009200221146FEF7DFF8C0B2A4
:10B7B000A2E4A2681189148853880291D18801916A
:10B7C00092880092002202212046FEF7CFF8032142
:10B7D00005460CA8FFF7E8FA0570DDE4A3681C88AD
:10B7E0009A780023CDE901330093ECE7A3681C8825
:10B7F0009A8859882046FEF73CFAC3E405210CA834
:10B80000FFF7D2FA0446C11C0130FEF755FA0023B7
:10B810002370C8E4A36859881888FEF757FA0446CD
:10B8200001210CA8FFF7C0FA002C18BF1E234CE71B
:10B8300009210CA8FFF7B8FA0446C31D421DC11C1C
:10B840000130FEF74DFAE2E7504600209C2400202C
:10B85000A0240020A36805210CA81D88FFF7A4FAE6
:10B86000AEB20446021DC11C3046FEF742FAE27831
:10B87000A4F80150002814BF0C2300232370002AD1
:10B8800092FAA2F3B3FA83F3227908BF4FF0FF33A1
:10B890000133E370002A92FAA2F3B3FA83F308BFEC
:10B8A0004FF0FF33013323717DE4A3681A78D10789
:10B8B00044BF07215970920744BF07229A709978B4
:10B8C0005878FEF72BFAAAE7A36899781888B3F896
:10B8D0000540CF0742BFDA7842F00702DA708E07E0
:10B8E00048BF1A79D97844BF42F007021A711B7910
:10B8F00041EA030212F0F80F02D01120FFF7FCBB5F
:10B900004D0701D05A0702D11220FFF7F5BB14F002
:10B9100003021CBF04F1FF3404F00102FEF708FA31
:10B92000FFF7E6BBA06800F11702C11D01F07AFF26
:10B9300047E6A06802F016F843E601210CA8FFF7DD
:10B9400033FA044601F030FF54E602210CA8FFF759
:10B950002BFA044601F026FF607058E70722A16821
:10B960000DA8F6F744FA07210CA8FFF71DFA0446C4
:10B97000411C0DA802F082F83CE60722A1680DA840
:10B98000F6F735FA07210CA8FFF70EFA0446411C1A
:10B990000DA802F093F82DE6A36801210CA81D78EC
:10B9A000FFF702FA0446284602F0A0F822E6A36850
:10B9B000188802F0ADF8FFF7B2BBA068C17902F0B9
:10B9C000AFF8FEE503210CA8FFF7EEF901460023CE
:10B9D00001F8023B0130F7F761FBFFF7E4BBA36816
:10B9E00000220121187801F0D9F9EAE5A0680123C5
:10B9F00082784178007801F06DF9E2E50DA801F058
:10BA0000F5F903210CA8FFF7CFF900230370BDF867
:10BA10003430A0F80130FFF7C6BBA3689A78597894
:10BA2000E0E7A068C378E3E70D210CA8FFF7BCF9B5
:10BA300002224270C270012282710D220023C27163
:10BA400063220370837003714371037242728372C5
:10BA5000C3720373FFF7A7BB41210CA8FFF7A4F93A
:10BA600000210446402200F8011BF6F7EDF9637847
:10BA700063F058036370A37843F00303A370FFF7E8
:10BA800092BB09210CA8FFF78FF9002100F8011BD8
:10BA90000822F6F7D9F9FFF786BB5E4B0DAA03F132
:10BAA0001006154618685968144603C40833B34293
:10BAB0002246F7D119889B782180A37014210CA805
:10BAC000FFF772F9002300F8013B13222946ABE58A
:10BAD000A1680020F7F7C6FAFFF721BB4FF08053AB
:10BAE000D3F8A420013206D1D3F8A8304FF6FF7264
:10BAF0009BB2934220D04FF08055D5F8A030DB07A1
:10BB00001AD518210CA8FFF74FF900260123044687
:10BB100043700670D5F8A400A11CFFF717F9D5F8FB
:10BB2000A830A371C3F3072363F03F03E37110222E
:10BB3000314604F10800ACE702210CA8FFF734F904
:10BB4000002303704370FFF72EBB21210CA8FFF7E1
:10BB50002BF90346002203F8012B4FF080520446D4
:10BB6000D2F8901001314BD0D2F89410013147D067
:10BB7000D2F89810013143D0D2F89C1001313FD057
:10BB8000D2F890001946FFF7E1F8611DD2F8940051
:10BB9000FFF7DCF804F10901D2F89800FFF7D6F8B6
:10BBA00004F10D01D2F89C00FFF7D0F84FF080525D
:10BBB00004F11103D2F88010013127D0D2F884109B
:10BBC000013123D0D2F8881001311FD0D2F88C1067
:10BBD00001311BD0D2F880001946FFF7B7F804F105
:10BBE0001501D2F88400FFF7B1F804F11901D2F879
:10BBF0008800FFF7ABF804F11D01D2F88C0031E5A5
:10BC0000102200211846F6F71FF9CFE71022002175
:10BC100018463EE72D1801002DE9F84300230B607C
:10BC20008389032B0646884603D86FF01500BDE8CC
:10BC3000F88350F8083F04215F881D8802F05FFFF9
:10BC4000B389BB42F1D3FEF735F94FEA1539044603
:10BC5000C5F30B05F0B91E4BD3E90023002102F018
:10BC6000007050EA010312D04FF0FF310120F6F7C7
:10BC7000B5F90122C8F800001A21FFF770F8D8F8CA
:10BC800000000121083002F02BFF012303706FF048
:10BC90003600CCE70379B9F1000F02D0B9F1020FF9
:10BCA00013D1022262F30103B168237167713A462E
:10BCB000E01DF6F79CF821462846FEF707F9002814
:10BCC000B5D02046FEF7FCF8AFE70122EAE700BF57
:10BCD00048460020037A03F00303013B012B70B5B3
:10BCE00004463CD801F10806C5880421304602F01C
:10BCF000F7FE237A617A418003F00303022B0CBF25
:10BD000045F4005345F480530380304602F0E8FECA
:10BD1000627A04F10B01F6F76AF8144B1A68002AEC
:10BD20001CDD134C1349236809685B1A934204D342
:10BD300040F682311048F4F7C1FC23680F2D03F15F
:10BD40000103236004D940F687310B48F4F7B6FCB1
:10BD50000A4A32F81530013322F8153070BD40F62A
:10BD60008E310548BDE87040F4F7A8BCF42C0020E3
:10BD7000F82C0020002D0020E9170100D42C002011
:10BD80002DE9F04F0379C688012B91B004460D468A
:10BD900000F1080900F0C782023B0A2B00F2BD82C5
:10BDA000DFE813F00B001E011E0122015801E10122
:10BDB00011023B0254026A028702C54B09934FF6F7
:10BDC0000473ADF8283002238DF82A30437A0344F7
:10BDD00093F80BB0037A580606D5002104F10A0344
:10BDE0005A46084601F028FEBA4BD3E9002300204A
:10BDF00003F0005150EA01034FD0637A23441B7BC8
:10BE00000493B54BD3E90001049B002B48D100F00B
:10BE100002020023134340D0B04F3B68002B80F256
:10BE20009780237A627A03F00F03012B18BF961FC5
:10BE3000224418BFF6B2977A049AC7F1000708BFE8
:10BE400000267FB2002A00F09380012B04D040F638
:10BE5000A401A348F4F732FC11220B212846FEF777
:10BE6000C5FF012303704370054601F09BFC834529
:10BE700005F1030072D20246A91C584601F098FA57
:10BE8000AB780233AB7001236B72062209F1080113
:10BE900005F10A00F5F7ABFF2F7411B0BDE8F08F84
:10BEA00000F00B02B5E78F4905934FEAC80A184620
:10BEB00006225144F5F78BFF059BB8B9B244217AAD
:10BEC0009AF801000A46C1F3801181420ED116F89A
:10BED000383002F00F0223FA02F1C907DDD4012144
:10BEE00001FA02F2134306F838309AE708F1010824
:10BEF0003A689045D7DBDFF8F881D8F8000006EB08
:10BF0000C000194606220230F5F771FFD8F800206C
:10BF1000237A06EBC201C3F380134B70237A03F03C
:10BF20000F0101238B40396806F832300F29D5BF45
:10BF300001310132C8F80010C8F80020D8F80020FC
:10BF4000D8BF3960102A04BF0022C8F8002068E773
:10BF50004FF0000804F10A03634EC9E7237AC3F3E4
:10BF60008013AB70062204F10A01F5F740FF8AE75F
:10BF700006F10B02D2B202212846FEF737FF012359
:10BF80000370237A10AA03F00F031344054613F835
:10BF90001C3C4370637A234493F80B8001F002FC4D
:10BFA000804505F1030011D20246A91C404601F06C
:10BFB000FFF9AB780233AB706E720A35324609F185
:10BFC00008012846F5F713FFAF5566E7237AC3F358
:10BFD0008013AB70062204F10A01F5F708FFEBE7C6
:10BFE0004846FEF7ABFF58E73A4BD3E9002300F190
:10BFF0000A0603F00051002050EA010308D0364B36
:10C00000D3E90023002102F4802050EA010310D17B
:10C01000237A10ACC3F3801304F8243D3146062282
:10C020000DF11D00F5F7E3FE09A92046FEF74AFFD2
:10C0300033E7082213212846FEF7D8FE00230370B9
:10C04000237AC3F380134370062231460230F5F79A
:10C05000CEFE22E7077A3FB900F1110300F10B0190
:10C06000FF22807A01F0E8FC1A4BD3E9002300207C
:10C0700003F0005150EA01033FF40FAF164BD3E930
:10C0800000AB40F2012000210AEA00020BEA0103A2
:10C0900013430AF400784FF000093FF4FEAE002F7E
:10C0A00040F01282114A13680133136058EA090301
:10C0B00040F01A82284612220121FEF797FE05461B
:10C0C000BFB312220021F5F7BFFE2F70E5E600BFD7
:10C0D000000103FF48460020504600209C24002019
:10C0E000E9170100A6240020A424002098240020A1
:10C0F000A0240020637F03F0C003402B40F00D829A
:10C10000062204F11801F5F772FE062204F111016E
:10C1100005F11100F5F76BFEE38BA5F81730238CC2
:10C12000A5F81930638CA5F81B3094F824306B7790
:10C13000B3E60770A0F80160637AC370A37A037155
:10C14000062204F10B010530F5F751FEE38BA5F84B
:10C150000B30238CA5F80D30638CA5F80F3094F8C4
:10C1600024306B7499E6BA4BD3E90023002102F026
:10C17000100050EA01033FF490AE04220521284646
:10C18000FEF7EDFD042105F1080002F0A9FC0023F3
:10C190000370A0F80160237AC3700F2E04D940F613
:10C1A000CE11AC48F4F78AFAAB4AAC4932F81630F3
:10C1B000086803440B60002322F81630A84A13686D
:10C1C000013B136069E6A24BD3E90023002003F092
:10C1D000005150EA01033FF460AEA24BD3E90023C3
:10C1E000002102F0040050EA01033FF456AE092298
:10C1F00003212846FEF7FAFD237A0370B4F80930CC
:10C20000A0F80160A0F80330B4F80B30A0F80530B6
:10C21000B4F80D30A0F807303FE68D4BD3E900238A
:10C22000002003F4004150EA01033FF436AE03223C
:10C2300030212846FEF793FD032105F1080002F0A6
:10C240004FFC00230370A0F8016026E6864BD3E97B
:10C250000023002102F4000050EA01033FF41DAE68
:10C26000022257212846FEF77AFD022105F1080037
:10C2700002F036FC068010E6754BD3E9002300205F
:10C2800003F0005150EA01033FF407AE754BD3E9C8
:10C290000023002102F4002050EA01033FF4FDAD29
:10C2A000032214212846FEF7A1FD0680237A83701D
:10C2B000F3E5674BD3E90023002003F0005150EA77
:10C2C00001033FF4EAAD674BD3E90023002102F4F8
:10C2D000006050EA01033FF4E0AD05220C2128463E
:10C2E000FEF784FD237A0370A0F80160627A002AC9
:10C2F00092FAA2F3B3FA83F308BF4FF0FF3301338E
:10C30000C370A27A92FAA2F3002AB3FA83F308BFA9
:10C310004FF0FF3301330371BFE540F69C214D48D8
:10C32000F4F7CCF9B9E5C37A033B122B00F2C980CC
:10C33000DFE803F00AC7C731BEC737C7C73E5EC7CD
:10C3400062C7C7C7C79C9C00414BD3E900230020AC
:10C3500003F0005150EA01033FF49FAD414BD3E994
:10C360000023002102F0100050EA01033FF495ADD4
:10C370000C2205212846FEF739FD0822054604F166
:10C380000C0120F8026BF5F732FD022204F11401D2
:10C3900005F10A005BE60A4600203146FEF73CFD47
:10C3A0007BE50B46324649460020FEF757FD74E513
:10C3B000274BD3E90023002102F4006050EA010377
:10C3C0003FF46BAD08220C212846FEF7C8FC08217B
:10C3D000681802F085FB00230370A0F80160237B3E
:10C3E000C370B4F80D308380B4F80F30C38054E5C7
:10C3F0000A46007B3146D1E7154BD3E900230020E4
:10C4000003F0005150EA010308D0164BD3E9002392
:10C41000002102F0200050EA010309D10023CDE9F8
:10C42000013300931A2202213046FDF79FFA34E5CA
:10C430000A2206212846FEF7D9FC0680A3894380FC
:10C44000E3898380238AC380638A038125E500BF53
:10C4500048460020E9170100D42C0020002D0020C0
:10C460009824002050460020282500202D4BD3E999
:10C470000023002003F0005150EA01033FF40DAD0A
:10C48000294BD3E90023002102F0400050EA0103C8
:10C490003FF403AD0A2207212846FEF7A7FC0680D9
:10C4A000238A4380638A8380A389C380E389CCE79E
:10C4B000037B0E2B7FF4F1AC0B46324600211A2091
:10C4C00073E740F661312AE758EA09033FF4F2AD19
:10C4D0001E220A212846FEF789FC04461E2200215E
:10C4E000F5F7B2FC2770D8E41E220A212846FEF791
:10C4F0007DFC0770A0F80160637AC370A37A0371B2
:10C500000546062204F10B010530F5F770FCE37DCA
:10C5100005F10B00002B7FF4EDAD06220021F5F7AD
:10C5200093FCF2E5484600205046002070B50646D0
:10C530000D46144613210522FEF711FC052106F1D4
:10C54000080002F0CDFA01230370A0F80150A0F812
:10C55000034070BD0379012B06D0023BDBB20A2BEE
:10C560000AD8074AD0567047037A03F00303032B17
:10C570000CBF0220032070474FF0FF30704700BF10
:10C5800092170100024B002118600846FEF7F6BC26
:10C590003025002073B50C464618351B8CB1F4F7D6
:10C5A0001FFE032C019007D904220DEB020128463F
:10C5B000F5F71DFC043CF0E7224601A92846F5F7F3
:10C5C00016FC002002B070BD08B5002301F0C8FBC6
:10C5D000002008BD00487047342500202DE9F04FA9
:10C5E00087B098467E4B049340F201730E46144682
:10C5F0009DF840B09DF844A09DF85890ADF81430D7
:10C60000FCF74AFF0746002840F0E58075490B7AA1
:10C61000012060F30203B8F1040F0B720BD9F2068C
:10C6200006F003030FD5704A0392350706D406AA15
:10C63000134413F80C8CB8F1010F12D10023CB6016
:10C640004FF001080EE0032B00F0C78006F00C034A
:10C650000C2B00F0C2800B7A69F302030B724FF0CF
:10C660000508CC600B789DF84C00019160F3020343
:10C670009DF8500060F3C4030B70FCF705FF90F8C1
:10C680004F500199034606AA05EB8500C5EBC0058E
:10C6900002EB08005A5D10F8080C60F303026FF318
:10C6A00004125A55D2B202F00F00012894BF42F092
:10C6B00020026FF345125A550A786BF346120A703E
:10C6C000D2B2500603EB050409D56AF3C7120A700B
:10C6D0004648129901930622F5F789FB019B5A5DA2
:10C6E0000BF0010B6BF386126FF3C7125A55D2B2DF
:10C6F00002F00F0101290BD16AF3C7125A551299A2
:10C70000062204F10800F5F772FB0C2363703FE08A
:10C7100007295BD1A17801F0C00166F38711A170F0
:10C72000B0064FF0000104F1020304F10402E170CD
:10C730000AD4A17811F0C00F06D1B9F1040F1EBFC1
:10C740000122E27004F10A02710644BFE17801326D
:10C75000A2EB030348BF41F04001DBB248BFE170E8
:10C76000022B8ABFA178012303F1FF306370E378C5
:10C7700084BF60F30501A1705B0609D5159B1BB34F
:10C780001B787F2B02D1159900230B7002F8013C16
:10C79000FCF77EFE90F84F2002EB8203C2EBC3024F
:10C7A0000424835C64F3030303F0CF036BF3861369
:10C7B0006FF3C713811883544B780BB906234B7062
:10C7C000384607B0BDE8F08F159BDFE76378002B94
:10C7D000DED106239AE70C27F2E71227F0E700BF25
:10C7E0000001060234250020030402003625002043
:10C7F0002DE9F0410F460646FCF746FE90F84F50F3
:10C8000005EB8502C5EBC202044610F802C00CF02D
:10C810000F03012B00EB020140D0072B3ED090F814
:10C820004E30AB4204D10135EDB2022D08BF0025D8
:10C8300005EB8503C5EBC30304EB0308E05C6CF375
:10C8400003006FF30410E054A05C14F803C0C0F3BD
:10C85000401060F3451C04F803C0A05C5FFA8CFC38
:10C86000C0F3801060F3861C04F803C0A25C5FFA7A
:10C870008CF0D20962F3C710E0540622023108F1AD
:10C880000200F5F7B4FA3246394608F108000636D8
:10C89000F5F7ADFA88F8016084F84F50BDE8F081F3
:10C8A0002DE9F04106460F46FCF7F2FD90F84F30B7
:10C8B00090F84E209A42044636D15D1CEDB2022D0E
:10C8C00008BF002503EB8302C3EBC2022BB203EBCC
:10C8D0008300C3EBC0034FF0040CE05C6CF3030077
:10C8E00000F0EF006FF34510E054A05CA118E25C8B
:10C8F000C0F3801060F3861204EB03086FF3C712D5
:10C90000E254B31D88F801300622023108F102001A
:10C91000F5F76DFA3246394608F10800F5F767FA7F
:10C9200084F84F50BDE8F0811D46CBE72DE9F34771
:10C9300020B902B0BDE8F047FDF744BDFCF7ACFDFF
:10C94000814600286BD1FCF79FFD0746FCF7A0FD50
:10C9500097F84F40334D04EB8403C4EBC30407EB5B
:10C9600004083B5D03F00F02072A10D198F803205A
:10C97000D2070AD54946C3F38010F6F759FB0622C1
:10C98000014608F10400F5F732FAFF2438E090F888
:10C990004F3003EB8306C3EBC603C6182878C0F3F9
:10C9A000C10000F00FFC287810F0400A15D1385D66
:10C9B0005146C0F38010F6F73BFB0622014608F112
:10C9C0000200F5F714FA385D5146C0F38010F6F70F
:10C9D0002FFB06220146B01CD5E74A46A91CC00918
:10C9E00000F034FCFF28044602D0484600F0CAFD9F
:10C9F0004146204600F06AFD3146204600F066FDC3
:10CA00002A78287AA9890094C2F3C10300F00700AC
:10CA100002F00702FDF72CFB02B0BDE8F087002012
:10CA2000FAE700BF342500202DE9F8438146884607
:10CA300017461E46FCF744FD88B90A4D2C79A5F827
:10CA4000008069F30304224666F3051213469DF83D
:10CA500020206F8062F387132B71BDE8F8830C20D0
:10CA6000FBE700BF44250020F0B585B028B90120C0
:10CA700005B0BDE8F040FDF7D1BDFCF721FD06464D
:10CA800010F0040029D136BB154C2079800900F044
:10CA9000BBFB237913F0010506D013F0200503D06A
:10CAA000304600F06FFD0125267906F00F07C6F32A
:10CAB000001600213046F6F7BBFAFF22CDE90252FC
:10CAC00022792388920901926288009231460246B7
:10CAD0003846FDF7A5FC05B0F0BD0C20FBE700BF14
:10CAE000442500202DE9F04F85B01E46BDF84830A2
:10CAF0000E9F9DF83C40BDF840A0BDF844B00393A4
:10CB0000804689461546FCF7DBFCA0BB039B0093DF
:10CB100052465B4639463046FCF7F6FC60BB284679
:10CB200000F072FBD5B1FF27A31E012B21D80020F6
:10CB300000F028FD04F00104012600212046F6F74C
:10CB400077FA4346024621460020CDE91067CDE939
:10CB50000E9505B0BDE8F04FFDF762BC00F0AEFCED
:10CB60000028E0D039462A46304600F06FFB0746E1
:10CB7000DAE70026E1E70C2005B0BDE8F08F000001
:10CB800070B501F063FB01F037FC1B4B1B4A1978B1
:10CB90001378CB1ADB0701D4117070BD01F000FDD2
:10CBA000064601F0EFFC361A01F0FAFC144B197836
:10CBB000144B0546187801F00FFB281A40F271213A
:10CBC000801B06F26934B4FBF1F401FB040401F0AC
:10CBD000F3FC01F0F7FCA0420BD801F095FB2146D5
:10CBE000012001F089FC01F0A7FCBDE8704001F0D4
:10CBF000CFBC04F27124EEE751250020502500201F
:10CC00004F2500204E25002038B501F035FBC4B279
:10CC10008CB101F051FBC5B201F018FB01F0ECFB47
:10CC200044B1064B187801F059FB1DB1044A138832
:10CC30000133138038BD2546EEE700BF4E250020A6
:10CC40004C25002070B515460C46064601F026F826
:10CC5000FCF7C6FB436801211B68984701F0F8F90F
:10CC6000284601F0BFF9174D174B032C8DBF042246
:10CC7000012204F1FF342A7094BF02FA04F4002266
:10CC80001A7098BF2C701978287801F0FBF996205B
:10CC900001F0C2FB01F02AFA7000023001F02EFA16
:10CCA0000A4801F043FA0A4940F25B6001F0F8FAE1
:10CCB0002A78520002F0FE02FF21082001F04EFA0D
:10CCC000002070BD4E2500204F250020401A010095
:10CCD00055555500072A2DE9F0410C46904651D88C
:10CCE0005A1E032A4ED8284E3278002A4AD1274AA3
:10CCF0001946FFF7A7FF054650BB254A13780133B5
:10CD0000137001F0E7FA08F1FF3307460230062BF3
:10CD100005D8DFE803F02025282B2E3134001D49EB
:10CD20002246F5F764F8384687F800807C7001F0F9
:10CD30004DFA01F0E9FA00F0D9FF0022C11C0120F0
:10CD400001F076FB01F0F8FB01F022FC01233370C7
:10CD50002846BDE8F08122460F21F5F775F8E2E795
:10CD600022465521F9E722460B49DAE72246FF2100
:10CD7000F3E722460021F0E72246F021EDE72246C4
:10CD8000AA21EAE70125E3E74A25002081CB00003C
:10CD9000512500203F1901004018010038B54B1EF5
:10CDA000022B1AD80E4D2B78BBB90E4AFFF74AFF5B
:10CDB000044680B901F08EFA01F002FA0A4B1878A5
:10CDC00001F08CFA00F092FF2246C11C204601F0CF
:10CDD0002FFB01232B70204638BD0124FBE700BF49
:10CDE0004A25002009CC00004E25002010B5154C26
:10CDF000237823B3144B15491A88028000221A8025
:10CE0000134A0B781078DBB298420ED101F00CFA7D
:10CE100001F07AFBFCF7E4FA436800215B6898476D
:10CE200000F04AFF0020207010BD023313700B7811
:10CE300010789842ECD020BF40BF20BFF7E7012018
:10CE4000F2E700BF4A2500204C2500205025002095
:10CE5000512500202DE9F041884615460AB1FF23EF
:10CE60001370144F002400F0010617F83430DA076D
:10CE70001CD5C3F34003B34213D10F4806224146E9
:10CE800000EBC400F4F7A3FF10B9E0B2BDE8F081F5
:10CE90003DB117F83430DB0703D42B78FF2B08BFE4
:10CEA0002C700134082CE0D1FF20EFE7002DF4D1E5
:10CEB000F7E700BF7F27002081270020F8B5104D3D
:10CEC000104E0024AF1C28216143735CDA0712D591
:10CED000012202FA04F02A780243C3F380132A7075
:10CEE0006A78A34013436B70074B0622194402FB78
:10CEF0000470F4F77CFF0134082CE4D1F8BD00BFC6
:10CF00004D2700200C2600200D26002008B5FCF738
:10CF1000C3FA28B9FCF7D4FAB0FA80F0400908BD8A
:10CF20000020FCE7F8B5194D194F00242E4615F8DE
:10CF30003430D90726D53B78E1005BB16B185A78BD
:10CF4000072A07D828235343124AD35C5A0701D52E
:10CF5000DB0617D5104816F83430012202FA04FC1B
:10CF6000027842EA0C020270C3F340034278A34005
:10CF700013434370094B02300622194402FB04009C
:10CF8000F4F735FF0134082CD1D1F8BD7F270020FC
:10CF90004C2700200C260020BF27002081270020DE
:10CFA00007280CD828235843064A135C1118C3F3EA
:10CFB000C00028B1C3F3400010B1486A7047002098
:10CFC000704700BF0C260020024B1B7803700248FC
:10CFD000704700BF822500208B25002038B50C4605
:10CFE00098B1072903D9F2211048F3F767FB104DD8
:10CFF00015F83420D20703D4F3210C48F3F75EFB75
:10D0000005EBC4046478204638BD072903D9F6210E
:10D010000648F3F753FB28236343064AD35CDB0738
:10D02000F1D4F8210148F3F749FBECE7441A010079
:10D030007F2700200C26002010B5104B1B78834260
:10D04000044604D84FF481710D48F3F737FB0D4BBC
:10D050001C5D072C04D94FF482710948F3F72EFBAD
:10D0600028236343084AD35CDB0704D440F205114C
:10D070000348F3F723FB204610BD00BF82250020A4
:10D08000441A0100832500200C260020072838B50B
:10D09000054610D82822094C4243A25CD30704D489
:10D0A0004FF488710648F3F709FB28206843205C99
:10D0B000C0F3401038BD0020FCE700BF0C26002064
:10D0C000441A0100034A044B002814BF10461846B6
:10D0D000704700BFBF2700204D2700200820704761
:10D0E00010B5FCF7E1F9044610B10C24204610BD40
:10D0F000FCF7FCF9C307F8D4154B1A7864F3000267
:10D100001A701A7A64F300021A721A7C64F300022D
:10D110001A741A7E64F300021A7693F8202064F3DE
:10D12000000283F8202093F8282064F3000283F89B
:10D13000282093F8302064F3000283F8302093F81D
:10D14000382064F3000283F83820024B1C70CDE7CE
:10D150007F270020102D002038B50546FCF7A4F9E4
:10D16000044610B10C24204638BDFCF7BFF9C307B4
:10D17000F8D42878FF2802D10F4B1C70F3E7224621
:10D18000691CFFF767FE072813D80C4B03EBC0029E
:10D190005578072D06D8282209496A438D5C64F327
:10D1A00045158D5413F830206FF3000203F830203A
:10D1B000D9E70224D7E700BF102D00207F270020E9
:10D1C0000C26002008B50D4B00221A705A7028B1A9
:10D1D000FCF78CF9C30701D4FFF7A4FE084B00222B
:10D1E0001A705A70074B1B7833B1FCF769F918B9FC
:10D1F000BDE80840FFF762BE08BD00BFBF270020A2
:10D200004D2700204C27002008B50D4B00221A7036
:10D210005A70C30704D5FCF747F908B9FFF782FE37
:10D22000084B00221A705A70074B1B7833B1FCF779
:10D2300033F918B9BDE80840FFF740BE08BD00BF8C
:10D24000BF2700204D2700204C2700202DE9F04764
:10D250008A4614460AB1FF231370DFF85890002560
:10D2600000F0010828266E43EFB219F80630DA07FD
:10D270001AD5C3F3801343450FD10D4806225146FA
:10D280003044F4F7A4FD60B13CB119F80630DB0777
:10D2900003D42378FF2B08BF27700135082DE1D177
:10D2A000FF273846BDE8F087002CF2D1F5E700BF34
:10D2B0000D2600200C2600202DE9F3410746FCF73F
:10D2C000F3F8054620B10C25284602B0BDE8F081F0
:10D2D000FCF70CF9C307F6D43878FF2803D11F4BAD
:10D2E00001221A70F0E707F101080DF1070241462B
:10D2F000FFF7B0FD07282DD99DF80760072E2BD822
:10D30000174C3A7814F8363004EBC60062F3410348
:10D3100041460622023004F83630F4F768FD2A460A
:10D3200041463878FFF792FFF300072823440ED8D0
:10D33000587028230B4A5843135C43F020031354BE
:10D3400014F8363043F0010304F83630BCE7FF220E
:10D350005A70F5E71225B7E70725B5E7102D00202D
:10D360007F2700200C26002038B50E4B1B780D4679
:10D37000ABB1072913D890B928220B4C4A43A25CC1
:10D38000D20704D44FF4E3710848F3F797F9282142
:10D390006943605C430702D5C0F3001038BD01202B
:10D3A000FCE700BF4C2700200C260020441A010097
:10D3B0000728F8B504460F46164604D940F2CD11A9
:10D3C0000E48F3F77BF928230D4D6343EB5CDB0735
:10D3D00004D44FF4E7710948F3F770F9282101FBF1
:10D3E00004F301FB0451EB5CC3F380133B70304644
:10D3F00006220131BDE8F840F4F7F9BC441A0100F7
:10D400000C2600202DE9F04F1A4B1B7883B31378BC
:10D41000FF2B2DD1184E00234FF02808B44606F1FB
:10D42000060908FB03F45FFA83FE375D17F0010F6E
:10D4300006EB040519D0C7F38017874215D14F1E9C
:10D440004C4415F801BF17F801AFD3450DD1A542E3
:10D45000F7D182F800E0282253431CF80300430769
:10D4600006D5C0F30010BDE8F08F0133082BD8D1EA
:10D470000120F8E74C2700200C26002070B40D4C4A
:10D480002478A4B1072A12D828250B4C05FB02F6F4
:10D49000A65D36070BD550B14B7903F0C003402B86
:10D4A00005D105FB0242D01D70BCF4F75ABD002027
:10D4B00070BC70474C2700200C260020024B1878C7
:10D4C000003018BF012070474C2700202DE9F041A3
:10D4D00005460C4601F10208FFF77CF8072D0646C9
:10D4E00033D82822254F6A43BA5C11072DD59307FC
:10D4F00004D440F211212248F3F7E0F8237843F0F6
:10D5000040032370282303FB05730622596A404613
:10D51000F4F76DFC237803F00F02012A2CD1072DBC
:10D5200004F108001ED82822144902FB05F7CF5D3C
:10D530007F0717D502FB051143F0800323700622F5
:10D540001E31BDE8F041F4F752BC30782378C0F3C7
:10D55000411060F386132370414600F00100F5F797
:10D5600067FDD7E73146227811F8023BDB0963F308
:10D57000C71222700622E4E7BDE8F0810C260020E5
:10D58000441A01002DE9F04F87B0824603F02AFBD0
:10D59000CDE90001BAF1000F40F0C980654BD3E935
:10D5A00000014E1C08BFB0F1FF3F00F0C080DDE974
:10D5B00000341B1A1846604B1A6864EB0104002300
:10D5C000904274EB0303ACBF01270027DFF87C9186
:10D5D00000244E4609F1070B2823634319F8033052
:10D5E000DD0744D50FB9980741D428236343F218C7
:10D5F000F15C490718D5D17D504A02EB011202F1C6
:10D6000010010DF1070011F8015D00F8015F914272
:10D61000F9D14B4902A81944F4F7B6FC20B140F205
:10D6200083214848F3F74AF828256543735D1A07B4
:10D6300017D502A90BEB0500F4F7A6FC20B140F2C8
:10D640008A214048F3F73AF8354402AB6B623E4B0F
:10D65000062202FB043802A94046F4F7C8FBC5F8CD
:10D66000248028236343F25C42F00202F254013426
:10D67000082CB1D127B1DDE900122E4BC3E900120D
:10D68000BAF1000F50D0FBF707FF00284CD0FEF78F
:10D69000A1FF03785B06804646D5FBF7F5FE90F8C0
:10D6A0004F4090F84E3004EB8402C4EBC202A34218
:10D6B000054600EB020704D10134E4B2022C08BF96
:10D6C000002404EB8403C4EBC303A95CE85C61F3AE
:10D6D00003006FF30410E854AA5CC1B2C2F3401215
:10D6E00098F8000062F34511E954002208F10201A4
:10D6F000C009EE18FFF7AAFD0728804604D940F2BA
:10D700004F211048F2F7DAFF31464046FFF7DEFEC0
:10D710007A7807F10801063A06F10800F4F767FB8A
:10D720007B78737085F84F4007B0BDE8F08F012714
:10D730004CE700BF082D0020342D00208B25002051
:10D740002A260020441A0100522500200C26002021
:10D7500008B50120FFF716FF034B04491A68044877
:10D76000BDE8084003F0DEB8342D0020142D002061
:10D77000682D0020074B1B7830B14BB1064B074991
:10D780001A68074803F0CEB813B1044803F07BB819
:10D79000704700BF4C270020342D0020142D00209E
:10D7A000682D00200820704708B5FFF7AFFB90B345
:10D7B0001A4B1A786FF300021A7093F828206FF34F
:10D7C000000283F8282093F850206FF3000283F8BA
:10D7D000502093F878206FF3000283F8782093F8B4
:10D7E000A0206FF3000283F8A02093F8C8206FF305
:10D7F000000283F8C82093F8F0206FF3000283F84A
:10D80000F02093F818216FF3000283F81821044BDD
:10D810000020187008BD0C20FCE700BF0C2600207B
:10D82000822500202DE9F04F85B0074689469246B3
:10D83000FFF76CFB002800F0858007F101080DF16F
:10D840000F0241463878FFF701FD07287CD99DF883
:10D850000F50072D7AD805EB850B3D4C4FEACB0BCB
:10D8600028266E430BF10100062241462044F4F7BE
:10D87000BEFA3978A35DA21961F3861348461021D8
:10D880000192A355F4F74FFCA35D102160F38203CE
:10D890005046A355F4F747FCA35D019A00F0010040
:10D8A00060F3C30313F0040FA35512D0294B19786A
:10D8B000D175294A55544A1C1A70284B03EB0113A1
:10D8C00009F11002013B12F8011D03F8011F4A453E
:10D8D000F9D158B10BF10700102251462044F4F75A
:10D8E00086FA282303FB054300225A6228266E434A
:10D8F0000BF11800062200212044F4F7A5FAA35DDD
:10D9000003F0FD036FF30413A3550022414638785A
:10D91000FFF7A0FA0728A35D9DBF114A43F020033B
:10D9200002EBC0006FF34513A3554FF0280398BFD7
:10D9300045705D430020635D43F00103635505B00E
:10D94000BDE8F08F0C20FAE71220F8E70720F6E791
:10D950000C26002082250020832500208B25002016
:10D960007F2700202DE9F84F8146FFF7CFFA0028E6
:10D9700053D009F1010A0022514699F80000FFF73F
:10D9800065FC072880464AD84FF0280B254C0BFB36
:10D9900000F3E218E35C5B0724D5234E3578013DA4
:10D9A00015F0FF051BD0D77DAF4218D01F481022BD
:10D9B00000EB051100EB0710F4F719FA00230BFB3D
:10D9C00003F16218615C11F0010FD8B221D0490750
:10D9D0001FD5D17DA9421CD1154BD775D8553378A9
:10D9E000013B33700022514699F80000FFF732FAEC
:10D9F00007289FBF0F4B03EBC000FF234370282075
:10DA000000FB08F0235C6FF3000323540020BDE803
:10DA1000F88F0133082BD2D1E1E70C20F7E7022081
:10DA2000F5E700BF0C260020822500208B25002072
:10DA3000832500207F27002070B55C7904F0C004A6
:10DA4000402C1D4617D119B10022FFF7FFFB0246FB
:10DA5000072A10D82821084C01FB02F3E35CDB07FE
:10DA600009D5182011FB0200204429460622BDE8F2
:10DA70007040F4F7BCB970BD0C26002038B5002208
:10DA80000D46411C0078FFF7E1FB072801D9022071
:10DA900038BD2824182314FB0030074C0444062109
:10DAA0002046F4F740FB0028F1D006222146284604
:10DAB000F4F79DF90020EBE70C26002010B50022BA
:10DAC0000C46411C0078FFF7C1FB07280AD8064B1B
:10DAD000282202FB00300622416A2046F4F787F92B
:10DAE000002010BD0220FCE70C26002010B50446E3
:10DAF000FFF70CFA40B11CB1012C01D0122002E05A
:10DB0000024B00201C7010BD0C20FCE74C270020AD
:10DB10004FF47A735843014B18607047342D00203E
:10DB200038B505460C46FFF7F1F9D8B10022691C5B
:10DB30002878FFF78BFB072816D81CB1012C0AD0D8
:10DB4000122007E02823094A5843135C64F30413A6
:10DB50001354002038BD2823044A5843135C43F073
:10DB60001003F5E70C20F5E70220F3E70C26002070
:10DB7000394A002330B41370384A117863F3000136
:10DB80001170117A63F300011172117C63F30001CB
:10DB90001174117E63F30001117692F8201063F383
:10DBA000000182F8201092F8281063F3000182F837
:10DBB000281092F8301063F3000182F8301092F8C8
:10DBC000381063F3000182F83810254A2549137094
:10DBD000254A1160254A4FF0FF344FF0FF35C2E966
:10DBE0000045234A117863F30001117092F8281060
:10DBF00063F3000182F8281092F8501063F30001DB
:10DC000082F8501092F8781063F3000182F87810CF
:10DC100092F8A01063F3000182F8A01092F8C810E7
:10DC200063F3000182F8C81092F8F01063F300016A
:10DC300082F8F01092F8181163F3000182F81811BD
:10DC40000C4A137020B10C490C4830BC02F012BED3
:10DC50000A4830BC02F017BE102D00207F2700209C
:10DC60004C270020A0BB0D00342D0020082D0020E3
:10DC70000C2600208225002051D70000142D002002
:10DC8000054B0022C3F808254FF44032C3F8442363
:10DC9000C3F80423704700BF00B00040044A137863
:10DCA000591C1170012013B9024A106018467047C0
:10DCB000F127002000B0004010B5094C23781BB9B3
:10DCC0002E210848F2F7FAFC20780138C0B2207003
:10DCD000012310B9044A136010BD1846FCE700BFC9
:10DCE000F1270020901A010004B00040014BD3F846
:10DCF0000405704700B0004000F5A870014B43F8E0
:10DD00002010704700B00040F0B5134B134C0125B4
:10DD100084462E460027A6461A462660C3F804C548
:10DD2000C3F80071C3F804711E60D3F8001131B953
:10DD3000D3F8041119B9D3F804150029F5D1CEF898
:10DD40000050D2F804110029E7D1D2F804050028C8
:10DD5000E3D0C2F80415F0BD00E0004004E000404C
:10DD600070B58CB00E4615460146102268461C461A
:10DD7000F4F7CAF910220DEB02003146F4F7C4F9AA
:10DD80006846FFF7C1FF25B1102208A92846F4F71D
:10DD9000BBF924B1102208A92046F4F728F80CB0EA
:10DDA00070BD00000028084B14BF4FF400124FF460
:10DDB0008012C3F8082514BF4FF480124FF40012EC
:10DDC000C3F80425704700BF00F00140DFF8F0C140
:10DDD0002DE9F0479CF80060744D754FC5F86075EB
:10DDE00034B24FEAC40909F1804303F5F833C5F8AA
:10DDF000643506F10B05EDB2ED00DFF8C8E1DFF8A0
:10DE0000C88105F18045A70005F5F835BE4406F147
:10DE10000803C5F810E5C844DBB2002800F086808E
:10DE2000022A00F09B80042A00F0BC80022949F6F7
:10DE3000C47278D0042914BF42F2B84047F274206B
:10DE4000DFF870A1C5F814A510444D0700F5FA706D
:10DE50004FF47A79B0FBF9F040F18F8042F2B84E7E
:10DE600044F69045042918BF754602F5FA71A200E0
:10DE700002F18042294402F51045DFF850E1D5F85F
:10DE80004055CEF84855DEF84855B1FBF9F1A942A6
:10DE900036BFDEF848550121691ACEF848154349C6
:10DEA000DFF82CE1434DC1F890E502F5F832C1F8F6
:10DEB0009455DB00D2F8005803F1804303F5F833A2
:10DEC00045F48035C2F80058C3F810E5C3F814854E
:10DED000394BC1F8983503F5FD4370333B44C1F825
:10DEE0009C354FF40033C1F80435A30003F180439F
:10DEF00003F510430136D3F8402582428BBFD3F897
:10DF000040250122101AC3F8402588BFC3F84005F8
:10DF1000264B4FF4906206F00106C3F804258CF8F6
:10DF20000060BDE8F08741F2883089E7DB0003F14B
:10DF3000804303F5F83307F1804707F5F8371F4AA8
:10DF4000C5F81425C3F810E5C3F81485D7F80038D0
:10DF500023F48033C7F800382C20C6E749F6404246
:10DF600002297FF467AF02F5AB521C324FF47A708E
:10DF7000B2FBF0F00F4AC5F81425A20002F180426E
:10DF800002F5F832DB00D2F8001803F1804303F504
:10DF9000F83321F48031C2F80018C3F810E5C3F853
:10DFA0001485A2E74AF65C02DAE700BF00F0014000
:10DFB0000C110040001000405011004004100040BF
:10DFC000142A00204091004004F0014000900040DD
:10DFD00048910040024B1B6803B11847704700BFCF
:10DFE000102A0020064B1860064B1022C3F80423A9
:10DFF000054B0222C3F880210120F3F757BD00BF73
:10E00000102A00200010004000E100E04FF08043A3
:10E010004FF0FF320021C3F8002EC3F8042EC3F8DE
:10E02000081EC3F80C2EC3F8101EC3F8142EC3F834
:10E03000182EC3F81C2EC3F8202EC3F8242EC3F8C4
:10E04000282EC3F82C2EC3F8302EC3F8342E704778
:10E0500008B50120F3F73AFD084B0022C3F8FC2F66
:10E060000122C3F8FC2F064A136823F0807323F0C3
:10E07000010343F08073136008BD00BF001000402F
:10E08000741700400228144B10D0042814D01A68CA
:10E0900022F000421A600321104BC3F81015D3F888
:10E0A000502642F00102C3F8502670471A6822F049
:10E0B00000421A600421EFE71A6842F000421A6039
:10E0C0001A6822F0FF0211F0010F42F05C0214BF47
:10E0D000052106211A60DFE73C17004000100040D0
:10E0E000014BC3F80C05704700100040024B08229A
:10E0F000C3F80C25704700BF00100040014BC3F867
:10E100000805704700100040074BC3F85405D3F8CA
:10E11000182522F00072C3F81825D3F8182542F00C
:10E120000072C3F818257047001000400A4A002307
:10E13000C2F82C350123C2F83035C378C2F8243533
:10E14000437881781B0443EA0163017843EA0123A1
:10E15000C2F81C35704700BF0010004002F00103F8
:10E16000C2F34202022A23D0042A0CBF4FF0C74256
:10E1700000220BB142F48012C0F108031B0400F02E
:10E180000F0040F4807003F47023034313430A4AE2
:10E19000C2F81435D2F81805084B0340C2F81835F8
:10E1A000D2F8183543F440331943C2F818157047B4
:10E1B0004FF08072DDE700BF001000400000F8FE65
:10E1C000014BC3F80405704700100040014BC3F831
:10E1D0000405704700100040022804D004280CBF3A
:10E1E0002B202920704728207047012070472920C4
:10E1F0007047022803D0042803D00A207047052066
:10E20000704711F0010F14BF1E201420704700004A
:10E21000014B01221A60704704100040014B01229B
:10E220001A60704700100040074A4FF49063C2F82C
:10E23000083501235360D360A2F5F0320021C2F803
:10E2400000121361704700BF00F00140044B002230
:10E25000C3F80021C3F80C21C3F81021704700BF98
:10E2600000100040034BD3F80001003018BF01201C
:10E27000704700BF00100040034BD3F80C01003082
:10E2800018BF0120704700BF00100040034BD3F8B7
:10E290005005B0FA80F04009704700BF0010004000
:10E2A000044B40F20312C3F83425C3F83805C3F811
:10E2B0003C15704700100040034BD3F800040030B9
:10E2C00018BF0120704700BF001000400048704791
:10E2D000042900200048704708290020044B03222D
:10E2E0000021C3F8002202460846FFF76FBD00BFB9
:10E2F00000100040034B0321C3F800120146012027
:10E30000FFF764BD00100040054B0322C3F8002254
:10E3100003F5F0334FF49062C3F80825704700BF4F
:10E3200000100040034AD2F8003243F48873C2F868
:10E330000032704700100040014BD3F84805704789
:10E3400000100040024B0022C3F81C21704700BFA0
:10E3500000100040034BD3F81C01003018BF01200F
:10E36000704700BF0010004030B50024A30003F147
:10E37000804303F580531568C3F80056013495882F
:10E38000C3F82056082C02F10602EFD1024B40EAF6
:10E390000120C3F8400630BD00100040034AD2F807
:10E3A000403623F0FF03C2F84036704700100040AB
:10E3B000024B0022C3F81421704700BF0010004038
:10E3C000034BD3F81401003018BF0120704700BF81
:10E3D00000100040014BD3F81004704700100040BB
:10E3E000044BC3F86005D3F8002242F04002C3F8A2
:10E3F0000022704700100040054B4FF48022C3F804
:10E40000482303F5A033034AC3F80825704700BF2B
:10E4100000B000406020720E034B044A1B7803F5E5
:10E42000A87342F823007047142A0020009000408F
:10E43000F8B5A2F57423294CA3F51073A34288BF45
:10E4400002F1E872264B274C84BF02F5D43202F564
:10E45000A5724FF00105B2FBF4F44FF000064FF047
:10E4600004074FF002021D60C3F8F864C3F8047596
:10E47000C3F8FC241C4AC3F8344588BF01F1FF31BE
:10E48000C2F848154FF48021C2F84413174902F529
:10E49000A4720C3BC1F83825C1F83C352023C1F8E3
:10E4A0000435FFF77FFC124B124A1560C3F8046570
:10E4B000C3F81075C3F808651D60A3F5FD43743BF0
:10E4C000C1F848354FF41063C1F84C25C1F8003845
:10E4D0004FF49053C1F804382046F8BDBFBDF07F1B
:10E4E0000C80004040420F0000B0004000F00140AE
:10E4F000009000400C900040024BC3F84015FFF71D
:10E5000051BC00BF00800040044A01231360D36067
:10E510000C3202F6F4721360D3607047048000403E
:10E52000044BC3F8440503F5B8334FF08862C3F8D1
:10E530000425704700800040064B074AC3F8402579
:10E5400002F5DE424032C3F84425044AC3F80425EC
:10E55000704700BF00F0014000110040400000047F
:10E56000014BD3F84405704700800040014B186010
:10E57000704700BF0C2A0020014B1868704700BF8D
:10E580000C2A0020014BD3F8400570470080004062
:10E59000024B4FF00062C3F80425704700F00140C1
:10E5A000014BD3F84805704700800040014BD3F879
:10E5B0004805704700800040014B01221A607047F7
:10E5C0004C800040014BD3F84C0570470080004060
:10E5D0001E4B10B50024C3F800450224A142C3F825
:10E5E000004503D004291ED0194900E01949174BF2
:10E5F000C3F80415C3F808051748C3F80C05C3F899
:10E600001025164AC3F814250022C3F80022C3F8C7
:10E610000421C3F80821124A4FF00071C2F8041512
:10E6200001221A6010BD0321C3F81C150C4B0D49C3
:10E63000C3F8781501F55E41BC31C3F87C154FF481
:10E640000051C3F804150849D1E700BF00F00040AD
:10E65000010000010100010108290020F827002025
:10E6600000F00140501100400100020110B50E4BB6
:10E6700000220224C3F80025C3F800450B4CC3F860
:10E680000445C3F80805C3F80C1509480949C3F83F
:10E690001005C3F814150121C3F80012C3F80421B2
:10E6A000C3F80821196010BD00F00040000001010E
:10E6B00008290020F82700200C4B0222C3F804236D
:10E6C000D3F804216AB10222C3F80823084A4FF4A0
:10E6D0000041C2F88011D3F80801B0FA80F0400977
:10E6E000704720BF40BF20BFEAE700BF00F00040F6
:10E6F00000E100E0034BD3F80004003018BF012014
:10E70000704700BF00F00040114B10B50322114CC0
:10E71000C3F80025C3F80405C3F80815D4F8042588
:10E72000013AC3F8102500210B4AC3F814254020F4
:10E73000C3F80011C3F80411C3F80811FFF750FE25
:10E74000064BC4F828114FF40002C3F8042510BD8D
:10E7500000F0004000100040F427002000F00140CD
:10E76000014BD3F80004704700F00040044A002336
:10E77000C2F8283102F56042C2F80035704700BF88
:10E7800000100040084BD3F8280160B103F5604346
:10E79000D3F8000138B1D3F8040120B1D3F808014F
:10E7A000B0FA80F04009704700100040012910B510
:10E7B000144603D01D210648F1F780FF18201CB134
:10E7C000BDE81040F3F772B9BDE81040F3F77EB929
:10E7D000DA1A010008B539B101290AD032210648F8
:10E7E000F1F76CFF002008BD0B20BDE80840F3F7EF
:10E7F00081B91820F9E700BFDA1A010088420AD06F
:10E8000018B94B1E584258417047012805D1B1FA3A
:10E8100081F04009704701207047002070470000D8
:10E8200029B1012909D055210648F1F747BF064B08
:10E830004FF40062C3F800217047034B4FF0807221
:10E84000F8E700BFDA1A010000E100E0032810B584
:10E85000044603D92A210648F1F730FF054B1C5D19
:10E860001CB92D210248F1F729FF204610BD00BF39
:10E870002A1B0100261B0100023810B41C46032885
:10E8800031D8DFE800F002101827032906D1174B12
:10E8900000219C60002010BCF3F7C2BC4C2114483E
:10E8A00010BCF1F70BBF042903D1124B01219C606E
:10E8B000F0E76321F3E7032903D0042906D0892177
:10E8C000EDE70D4B00219C600120E4E70B4B01219B
:10E8D0009C60F9E7042904D1094B01219C600320C5
:10E8E000D9E7A121DBE7A721D9E700BF58460020DF
:10E8F0002A1B010068460020784600208846002038
:10E900009846002001460020FFF7F6B97047000046
:10E910008279044B03EB4213DB69C01A024BC0102F
:10E9200058437047EC470020ABAAAAAA10B5094B80
:10E93000827903EB42130A689B695C6823689A42F8
:10E9400094BF0A600B60FFF7E3FFD4E9002302FBEA
:10E95000003010BDEC4700202DE9F3410546019140
:10E96000164602F033F907464FF02003EFF3118803
:10E9700083F311886B8A002B3DD02A8A9A422AD9C8
:10E980000021284601F04CFB044620B388F311888F
:10E99000019B002B3CD0731C012B06D902F016F909
:10E9A000C01BB04294BF361AB61BA3791E4F07EBAB
:10E9B000431332469B691B6801A91B682046984790
:10E9C0000546206128BBA079214607EB401001F0E5
:10E9D00008FB2C4618E06B8A5A1E6A8288F311885D
:10E9E0002C8AE41AEB69182202FB04340E4BED1A50
:10E9F0006D11A571CCE788F311883146284601F0E6
:10EA00000FFB04460028C3D1204602B0BDE8F081C8
:10EA10002361002323600122A280A381019A23693C
:10EA2000E281A360F0E700BFEC47002083695B68E8
:10EA30000A461968FFF790BF70B5064601F0F0FA74
:10EA4000054628B10446637913F0010302D123601F
:10EA5000284670BD0021304601F0E2FA637920605B
:10EA600023F0010363710446EDE710B40A4614680D
:10EA700014B910BC01F0BABA537943F001035371D1
:10EA80002246F4E7F8B5154D0446002604B9F8BD52
:10EA900023792768013BDBB22371002BF7D1216971
:10EAA00059B163799B0707D4A37905EB431320463B
:10EAB0009B691B689B6898472661A079A66005EB57
:10EAC000401326605B691BB1204698473C46DDE752
:10EAD000214605EB401001F084FAF7E7EC470020EF
:10EAE0008388026819448180D018704730B48388C5
:10EAF00004689D188580E01830BCF3F778B98388E6
:10EB00005B1A83800368194401600846704708B5A2
:10EB1000036801211A78FFF7F2FF104608BD02686A
:10EB20008168C3888088521A9B1A181A704710B5DA
:10EB300004688068A468C0692468012904D1584029
:10EB4000C4F80405002010BD003320FA02F04FF095
:10EB5000010118BF012300F001009140834214BF5E
:10EB6000C4F80815C4F80C15ECE770B504688068A3
:10EB7000A468C0692568D5F81465D5F81045D5F89E
:10EB8000045560406C403440604001291CBFD040B7
:10EB900000F001001860002070BD8368186872B131
:10EBA00008605A68196002B9596000207047106007
:10EBB0005868814208BF5A600DE00246006800288C
:10EBC000F3D08842F9D10868002AF0D15A68186059
:10EBD000914200D1586000230B60E6E7836870B56E
:10EBE0001C6805460E464CB1A3681E4204D06368FB
:10EBF00032462146284698472468F4E770BD000055
:10EC000008B5094B1A786AB9012119700620052147
:10EC1000F2F77EFF0620F2F749FF044B4FF0004267
:10EC2000C3F80423002008BD402A002000600040F3
:10EC30001F288ABF094B4FF0A04300F01F0003EBD1
:10EC40008000D0F8003723F44033C0F80037D0F804
:10EC5000003743EA0141C0F8001770470003005035
:10EC6000F8B5026883689768DC69D3E902120A4044
:10EC7000D3E90510014322EA010239681B69D1F882
:10EC800010155C404C4022EA0404012500260AB914
:10EC90002046F8BD2A4209D03B7906F01F0000212A
:10ECA00040EA4310FFF7C4FF22EA050201366D0077
:10ECB000EDE7F8B5846803689D68D4E902321A402C
:10ECC000D4E905310B4322EA03020127002602B9E9
:10ECD000F8BD174212D0E169236995F804C04B4092
:10ECE000F34013F0010F06F01F0014BF02210321AF
:10ECF00040EA4C10FFF79CFF22EA070201367F0032
:10ED0000E5E70000F7B5036886689B6801F01F041B
:10ED10000D464C491B79D1F8042344EA4314D2B27E
:10ED2000002303F5A27051F82000C0F305208442AF
:10ED30006CD122FA03F0C00768D59A0002F1804234
:10ED400002F5C042D2F8100520F00100C2F810050B
:10ED5000012202FA03F3C1F8083320460021FFF72D
:10ED600067FFB068E84010F001004DD0F068E8405F
:10ED700010F0010048D07069E84010F0010251D055
:10ED8000B369EB40DB0745D43369F269EB4022FA03
:10ED900005F503F0010305F00105AB420CBF0225A8
:10EDA0000125284F002101F5A27357F8230010F028
:10EDB000030031D18A0002F1804303F5C0432402ED
:10EDC000D3F8106526F44F3626F44076C3F8106564
:10EDD000D3F8106504F47C5402F1804202F5C2427B
:10EDE00044EA05453543C3F8105510601268019296
:10EDF000019AD3F8102542F00102C3F8102501232F
:10EE000003FA01F1C7F8041303B0F0BD0133082B76
:10EE100087D1A2E70325C4E701310829C3D16FF0E8
:10EE20001200F1E7F16933694B4023FA05F515F05B
:10EE3000010F20460CBF03210221FFF7F9FE104607
:10EE4000E2E700BF006000402DE9F84F0746856803
:10EE500003F47040B0F5804F1E4647D02ADCB0F571
:10EE6000805F3BD0B0F5405F3CD050BB06F44078AB
:10EE7000B8F5807F3CD0A8F500746342634106F08A
:10EE8000010C4FEA4C08012948EA0C0818BFD4B21B
:10EE900048EA0020DFF8D4A012BFA1464FF01F09B6
:10EEA000002440EA83084FF0010BA14522D2002044
:10EEB000BDE8F88FB0F5E04F16D005DCB0F5A04FF7
:10EEC0000ED06FF01500F3E7B0F5404F04D0B0F569
:10EED000504FF6D10720C9E70620C7E70120C5E754
:10EEE0000320C3E70420C1E70520BFE70220BDE7F8
:10EEF0000323C4E73B689B681A7904F01F0343EAC5
:10EF000042131F2BC6BF03F01F0352464FF0A0420F
:10EF100003F5E073B10742F82380AB680BFA04F203
:10EF20004CBF13439343AB606B69B0064CBF1343B4
:10EF300093436B61AB6971064CBF13439343AB6161
:10EF40002B6970074CBF134393432B61EB69310668
:10EF50004CBF1A4323EA0202EA6121463846FFF712
:10EF6000D1FE0028A4D10134E4B29EE70003005092
:10EF700001292DE9F04118BFD4B28768064612BFB7
:10EF800025461F2500244FF00108AC4202D900207D
:10EF9000BDE8F081FB6808FA04F223EA0203FB6093
:10EFA00021463046FFF7AEFE0028F1D10134E4B22D
:10EFB000EBE70000F0B5002685B0CDE90266294DEB
:10EFC0002C68012C0BD12848FFF74AFE02902748F5
:10EFD000FFF746FE03902E602B680093009B244EA3
:10EFE000002301279C46D6F8042307FA03F11142B7
:10EFF0001ED003F1805202F5C2529200116801291D
:10F0000016D103F5A2700DF1100E56F82050C2F87B
:10F0100000C0C5F340300EEB8000C5F30425A940C5
:10F02000126850F8085C01922943019A40F8081CC4
:10F030000133082BD7D1029911B10B48FFF7CEFD50
:10F04000039911B10948FFF7C9FD012C08D1064801
:10F05000FFF72FFE054805B0BDE8F040FFF729BED9
:10F0600005B0F0BD7C61004054470020604700209F
:10F070000060004001292DE9F04118BFD4B2876833
:10F08000064612BF25461F2500244FF00108AC425A
:10F0900002D90020BDE8F081FB6808FA04F21343AE
:10F0A000FB6021463046FFF72DFE0028F2D10134E7
:10F0B000E4B2ECE7054B1B682BB9054B1878003020
:10F0C00018BF012070470120704700BF1C2100407D
:10F0D0008C2A0020034B186818B1D3F85C03C3F8DE
:10F0E0005C0370472421004082680B4692E80300CD
:10F0F00083E8030000207047024B0422C3F8042376
:10F10000704700BF00200040024B0422C3F80823D0
:10F11000704700BF0020004008B5FFF7CBFF08BDD7
:10F12000024B1868003018BF0120704708210040CA
:10F13000024B4FF40072C3F80423704700200040D4
:10F14000024B4FF40072C3F80823704700200040C0
:10F1500001207047024B1960024B1A60704700BFD4
:10F16000842A0020882A0020034B1B6813B1034A1D
:10F1700010681847704700BF842A0020882A0020A2
:10F18000034B8022C3F808230122DA6000F02FBD70
:10F190000020004008B500F029FD0B4B01221A6049
:10F1A0008022C3F8FC224FF02002EFF3118382F398
:10F1B0001188064A12781AB1054A0421C2F80011D2
:10F1C00083F3118808BD00BF082000408C2A00206E
:10F1D00000E100E030B54B79012B20D18B79032B76
:10F1E0001DD1CC792CB1012C19D103689B681B78F7
:10F1F000ABB10A7912B1022A11D10E220B6847F67F
:10F200001225AB426CD027D8B3F5965F61D012D8E7
:10F21000B3F5167F4CD005D8B3F5967F70D06FF05C
:10F22000220052E0B3F5966F50D0B3F5166FF6D1C9
:10F230004FF41D233EE0B3F5615F4CD004D8B3F525
:10F24000165FECD1304B35E0B3F5964F46D0B3F5B1
:10F25000E14FE4D12D4B2DE0B3F5E13F48D011D87B
:10F260004DF6C025AB423ED004D8B3F5164FD6D1EB
:10F27000274B1FE0B3F5614F38D0B3F5963FCED1A1
:10F28000244B17E0B3F5E12F36D008D8B3F5613F32
:10F2900030D0214DAB42C2D14FF080630AE0B3F5CC
:10F2A000612F2BD01D4DAB42B9D14FF0805301E0FF
:10F2B0004FF41C331A4D2243C5F82435C5F86C258C
:10F2C000836803C983E80300002030BD4FF49E2308
:10F2D000F0E7144BEEE74FF46C13EBE7124BE9E762
:10F2E0004FF40003E6E74FF46503E3E70F4BE1E774
:10F2F0000F4BDFE70F4BDDE70F4BDBE70F4BD9E79A
:10F300004FF4A033D6E700BF0050270000F075008F
:10F3100000509D0000903A0190D0030040420F0041
:10F320000020004000B0130000A04E0000F0EB00F1
:10F3300000E0D70100B0AF0300705F0700D0BE0E41
:10F3400008B50C4BD3F8042312F0800F1A4605D1F0
:10F35000D2F8040310F0040006D108BDFFF7AAFE9E
:10F360000028F5D00120F8E7034B1868003018BFDB
:10F370000120F2E70020004008210040F7B50023FB
:10F38000094C0A4F1E46D8B2151A002D02DD256819
:10F3900001330DB903B0F0BD266025680195019DCC
:10F3A000D7F818550D54EEE7082100400020004022
:10F3B00007B50B4A0023136012680192019A094AAB
:10F3C0001370094B01221A60C3F81415FFF772FE7F
:10F3D0000028FBD0054B01221A6003B05DF804FB46
:10F3E0001C2100408C2A0020082000400C200040F6
:10F3F000084B1A6882B052B1002018601B68019354
:10F40000019B054BD3F818350B7002B070474FF0D5
:10F41000FF30FAE708210040002000402DE9F341C9
:10F420000D4E0E4FDFF838800024E5B2531B002B41
:10F4300003DDFFF73FFE013418B9284602B0BDE8EE
:10F44000F081002333603068019001983B704B5D80
:10F45000C8F81C35E9E700BF1C2100408C2A0020B9
:10F46000002000404FF0A04373B520221B4CC3F88E
:10F470000825002103220525C3F81427C3F80C171B
:10F48000C4F81425C4F80C55154D4FF48076C5F812
:10F490000865C5F82027C3F81C172823C4F80835C9
:10F4A0000723C4F810358168FFF794FE054690B92C
:10F4B0000423C4F800350B4B18601B680193019BB3
:10F4C000094B01212160024602201970F2F720FB4E
:10F4D0000220F2F7EBFA284602B070BD002000408F
:10F4E00000030050082100408C2A002000234350D4
:10F4F00082B043580193019B02B0704783681A7D24
:10F5000072B1026892681268D2F8201141B14FF4CA
:10F510008071C2F808130121D16000221A7570476A
:10F520009A680AB1D86810477047000070B54B79E7
:10F53000012B23D18B79032B20D1CC792CB1012C39
:10F540001CD103689B689B79C3B10A7912B1022A66
:10F5500014D10E2203689B681D680B6847F61226BB
:10F56000B3426BD027D8B3F5965F61D012D8B3F50C
:10F57000167F4DD005D8B3F5967F74D06FF022007A
:10F5800052E0B3F5966F50D0B3F5166FF6D14FF445
:10F590001D233FE0B3F5615F4CD004D8B3F5165F8F
:10F5A000ECD1324B36E0B3F5964F45D0B3F5E14F91
:10F5B000E4D12F4B2EE0B3F5E13F48D012D84DF601
:10F5C000C026B3423DD005D8B3F5164FD6D14FF47F
:10F5D0001D031FE0B3F5614F36D0B3F5963FCDD193
:10F5E000244B17E0B3F5E12F37D008D8B3F5613FCE
:10F5F00030D0214EB342C1D14FF080630AE0B3F561
:10F60000612F2DD01D4EB342B8D14FF0805301E091
:10F610004FF41C33C5F82435836803C92243C5F869
:10F620006C2583E80300002070BD4FF49E23F1E7B2
:10F63000134BEFE7134BEDE7134BEBE74FF40003EE
:10F64000E8E74FF46503E5E74FF46B03E2E74FF0BB
:10F65000EB73DFE74FF06C73DCE74FF0E863D9E75B
:10F660004FF07063D6E74FF4A033D3E70050270084
:10F6700000C0750000903A0190D0030040420F0096
:10F6800000B0130000F03A0000A04E0082680B4664
:10F6900092E8030083E80300002070470268926844
:10F6A000126808B58368D2F8100150B15B7D0B7009
:10F6B00010464FF48871FFF719FF012313600020F3
:10F6C00008BD4FF0FF30FBE713B5036802AC9B6841
:10F6D00004F8011D1A684FF490711046FFF706FFF9
:10F6E0000123C2F84445C2F848359360D2F820118E
:10F6F0000029FBD0D36002B010BD03689B681B6873
:10F70000D3F8240118B1D3F88004C3F880047047FB
:10F71000036870B50D4699680C68D4F82031CBB1F8
:10F720008B8886689A424FF490712046A8BF1A468B
:10F73000FFF7DCFE00239342316907DB0123C4F8A5
:10F740004415C4F84825A360104670BDE85CC85451
:10F750000133F0E71A46F7E738B503689B681A6883
:10F76000D2F810310C4653B185684FF488711046B9
:10F77000FFF7BCFE6B7D23700120106038BD18467A
:10F78000FCE703689B681A6883684FF48071C2F8CD
:10F79000041300221A757047836801221A75704796
:10F7A00003689B681B68D3F8200118B1D3F80403E1
:10F7B000C0F30020704703689B681B68D3F81001F2
:10F7C000003018BF0120704703689B681B68102237
:10F7D000C3F80423704703689B681B681022C3F8B2
:10F7E0000823704703689B681B684FF40072C3F8D6
:10F7F0000423704703689B681B684FF40072C3F8CA
:10F8000008237047012070478368C3E902127047DC
:10F8100008B503689B681968D1F80433DB05024614
:10F8200005D4D1F8040310F0100006D108BDFFF78D
:10F83000B7FF0028F5D00120F8E71046FFF7BBFF1F
:10F84000003018BF0120F1E770B500220646012103
:10F850002820F2F75DF92820F2F728F93368B56817
:10F860009B681C684FF0A0434FF40032C3F8082592
:10F87000032100221120C3F84417C3F85027C4F80D
:10F880000C051420C4F814054FF40040C3F8080513
:10F89000C3F83C17C3F858270F23C4F808351623BC
:10F8A000C4F8103529463046FFF740FE0246B0B98D
:10F8B0000823C4F800354FF488712046FFF716FE80
:10F8C00005F11503C4F8343529690123C4F8383526
:10F8D0002360C4F84415C4F84825A360E3601046CB
:10F8E00070BD0000F0B58378C7784FF02004EFF3C7
:10F8F000118E84F31188067890F801C09B1B3B4061
:10F900009A4288BF9AB2B4183C40354604708EF3D0
:10F9100011880A440C46A24216D1664509D14FF01F
:10F920002005EFF3118285F311880578457082F385
:10F930001188641AA2B201799C1AA14222BF074B16
:10F94000012119601046F0BD00EB050E01359EF84F
:10F9500005E004F801EB3D40DDE700BF00D00040CA
:10F960002DE9F843114D0E46144605F1450805F101
:10F97000180914B92046BDE8F8834FF0FF31284636
:10F9800000F0F6FD224631464046FFF7ABFF074642
:10F99000284600F0C6FD2FB94FF0FF31484600F071
:10F9A000E7FDE6E7E41BA4B23E44E2E7B02A00200C
:10F9B00082B04FF02003EFF3118283F31188094BDB
:10F9C000196861B10849D1F80805002119601B6860
:10F9D0000193019BC0B282F3118802B070476FF0AF
:10F9E0000A00F8E700D1004000D00040DB072DE915
:10F9F000F3478846144605D41D48FFF773FF02B04D
:10FA0000BDE8F08772B34FF02003EFF3118583F365
:10FA100011880D20F2F76EF807460D20F2F756F820
:10FA200085F31188134EDFF854900022326032685B
:10FA30000192019A104A0121116025464FF4005AA3
:10FA400033688BB1FFF7B4FF0028C9F880A1F7DB5A
:10FA5000013DADB208F80500002DF1D117B10D2020
:10FA6000F2F724F82046CAE720BF40BF20BFE7E7EF
:10FA7000E02A002000D1004000D0004000E100E07A
:10FA800037B51D4C01221146204600F041FD04F11E
:10FA900018000122002100F03BFD072384F84830C4
:10FAA000042384F849304FF0706323630C2384F8F7
:10FAB00034300025114B84F8455084F8465084F8C2
:10FAC0004750D3F8042542F00102C3F804250C4A3C
:10FAD000156012680192019A0122C3F804230521DE
:10FAE0001A600D202A46F2F713F80D20F1F7DEFF19
:10FAF000284603B030BD00BFB02A002000D000402F
:10FB000000D1004010B5FFF753FF002820DB174B52
:10FB100093F8322093F8311093F83340511A34EAB5
:10FB20000101C0B20DD193F8472093F8461093F825
:10FB30004840511A34EA01010BD10D4B01221A60E1
:10FB40000EE099180132224081F8350083F8322006
:10FB500010BD99180132224081F84A0083F84720ED
:10FB60000448BDE8104000F0DCBC00BFB02A002013
:10FB700004D00040C82A002038B5084B53F8204074
:10FB8000013053F820502046854204F10C0400D87F
:10FB900038BD54F80C3C5B689847F4E75C1C0100E6
:10FBA000104B70B5104C05461E469C4204D10E4CBD
:10FBB000B44209D1002412E062681AB122681268C6
:10FBC000AA420CD00C34F0E763680BB90C34EFE7B1
:10FBD000236828461968F2F7EDF80028F6D1204688
:10FBE00070BD00BF90470020D0460020704770478E
:10FBF000F1F7A6BC08B50A4D4FF02002EFF31183D0
:10FC000082F3118800F0FEFE012102280446D8BFCD
:10FC1000084600F0ADFF2C62F1F7AAFDECE700BF4B
:10FC2000382D00200248034A0021121AF2F70CB9BD
:10FC300000000020E42D00200248034A0349121A64
:10FC4000F2F7D5B8E04400204C480020C41C010065
:10FC500008B50220FFF790FF0748F1F795F9032058
:10FC6000FFF78AFF00F06EFDF0F77AFD034A137B81
:10FC700023F00103137308BD841C0100702B0020C6
:10FC800080B586B0314B06AF83F30888304B314ED8
:10FC9000314D0024E02283F82220DC771C765C764C
:10FCA0009C765A6A42F4E0225A62F1F7F7FEF1F7C5
:10FCB00059FD2046FFF760FF0120FFF75DFF00F0D0
:10FCC000EBFB264B756205930123CDE90343CDE998
:10FCD00001440094224B23494FF40072284600F05F
:10FCE000D7FC6B7B23F0040213F01B0F6A733446BE
:10FCF00005D12B6A013302D1284600F007FB1A4BCD
:10FD00001A4E059301220F23CDE903320023CDE9DA
:10FD1000013300934FF4A072154B1649304600F0A2
:10FD2000B7FC737BE66023F004037373124BA5608A
:10FD3000C4E906330A4A114B114C83F3098863B6B0
:10FD4000002181F311881046204700BFE0420020C7
:10FD500000ED00E0382D0020702B0020741C010005
:10FD600051FC0000A0370020791C0100042B00206A
:10FD7000F5FB0000A0390020502D0020A039002004
:10FD8000ED07000038B5074C074DAC4201D3002009
:10FD900038BD04F114032046C4E90533F0F78BFDA8
:10FDA0001C34F2E790470020904700202DE9F04FE7
:10FDB0001D1E85B006460C46174657DD00F0ECFECA
:10FDC00080462B484FF4004C00214FF4A022002322
:10FDD000CCFB0501F0F794F918EB0002254B904697
:10FDE000F31A254A9B1002FB03FA5FFA8AFA06F11E
:10FDF000140B009403AB02AA39463046F0F7A6FD77
:10FE000010F10B0F0BD1009403AB02AA3946304618
:10FE1000F0F79CFD10F10B0F08BF6FF00B0063793A
:10FE2000029A84F804A062F3030363716368039A7F
:10FE300062F31F336360B0B1ADB110F10C0F12D19A
:10FE40004FF02003EFF3118083F311882A465946BF
:10FE500000F004FB6B1CCCD000F09EFEB8EB00055C
:10FE6000C7D56FF00A0005B0BDE8F08F0022B5E7F6
:10FE7000FFFF040090470020B76DDBB670B5047833
:10FE800002684178134EC4EBC404A400120B01F0C5
:10FE90000F013019F0F729FE4FF02003EFF3118521
:10FEA00083F3118804F11400304400F0E5FA68B1DE
:10FEB000EFF305830D2B09D81BB1074B5B681B05BE
:10FEC00004D52846BDE8704000F0CEB985F311880E
:10FED00070BD00BF9047002000ED00E013B5042482
:10FEE0000A1904D200236946FFF760FF10B1002011
:10FEF00002B010BD224601A90098F1F778FF0098E2
:10FF00000430F5E710B10438FFF7B8BF70470000C0
:10FF1000034B9B680146186E08B1FFF7DFBF7047BF
:10FF2000382D0020F8B504460E4617464FF0200243
:10FF3000EFF3118582F311889BB10820FFF7E8FFEA
:10FF4000002832D0012347600360036803F00302F6
:10FF500056B9236813430360636820606BB960601F
:10FF60000BE03B603846F0E7336833F0030314D10D
:10FF7000026062685AB9C4E90000042104F1080073
:10FF800000F05AFF284600F06FF90020F8BD136812
:10FF900003F0030303431360E1E713430360336893
:10FFA00003F0030318433060E7E76FF00B00EDE761
:10FFB00010B5044630B10268930703D0446809B114
:10FFC000FFF7A0FF204610BD0023C0E9003300F179
:10FFD0000803C0E9023370470A4600234168FFF76F
:10FFE000A1BF00230A461946FFF79CBF38B54FF062
:10FFF0002003EFF3118583F31188436853B901603F
:020000021000EC
:1000000042600421083000F017FF2846BDE8384060
:1000100000F02AB91C6804F0030421431960EFE7DB
:100020002DE9F041044686B00D464FF02003EFF372
:10003000118783F31188026882B11368416823F045
:1000400003038A42036008BF436001211046FFF7A3
:10005000AFFF87F3118806B0BDE8F08119B987F3C7
:1000600011880020F7E787F31188042103460DEB80
:10007000010000F045FE6A1C02D000F0A7FD064614
:100080000027049BEA1B6FF31033012101A804939E
:1000900000F04CFE08B10B30E3D14FF02003EFF33A
:1000A000118883F31188206838B10368626823F0EF
:1000B00003039042236008BF63600121FFF778FFCC
:1000C00088F311880028C6D16B1CDAD000F07EFDC1
:1000D000871BBD42D5DAC4E7D0E900231A60026865
:1000E0005360704708B5F1F7CFFA054B054A1B6816
:1000F0001844106100211846BDE8084000F038BDE2
:10010000E02B0020382D00204FF02003EFF311806A
:1001100083F311887047000038B5104C234653F81C
:10012000285F9D4200D005B9E568A36878B973B12E
:100130005A7BD2060BD11A6A013208D1DA897F2A9A
:1001400005D9074A1268934201D0636238BDAB42B9
:1001500001D0FFF7C7FF6562F8E700BF382D002028
:10016000801C010090F90E0091F90E309842ACBF4E
:100170000020012070470000F8B50D460746FFF744
:10018000C3FF0C4B04460C4800224FF400460021EC
:100190001A61C6FB07014FF4A0220023EFF7B0FF5E
:1001A000064B1860064B1D60FFF79CFF84F3118817
:1001B000F8BD00BF382D0020FFFF0400E02B002019
:1001C000DC2B002010B50146FFF79EFF4B7B5A0643
:1001D00004460DD50846FFF77FFF4B7B23F0400315
:1001E0004B73054B9868431A58425841FFF794FFE8
:1001F00084F3118810BD00BF382D002008B50246D9
:10020000FFF782FF13689A4208BF002380F311882A
:10021000184608BD10B50146FFF776FF04460846AC
:10022000FFF75AFF4B7B23F002034B7384F31188D3
:1002300000238B6010BD10B50021FFF7DFFF0446DF
:1002400028B1FFF7E7FF04F1180000F0CBFB2046D0
:1002500010BD10B50446FFF7DDFF04F11800BDE83E
:10026000104000F0BFBB0000EFF305830D2B0BD84F
:100270001BB1074B5B681B0506D5064B9A685B6A8A
:100280009A4201D0F1F7BABA80F31188704700BFE3
:1002900000ED00E0382D002010B5FFF735FF0A4BC8
:1002A0009A68D37B01330446D3730120FFF734FFF0
:1002B00084F311884FF02003EFF3118083F311884A
:1002C000BDE81040FFF7D0BF382D002003689842EA
:1002D00010B513D093B191F90E2093F90E409442CA
:1002E00006DD5A68C1E900325A681160596010BDD4
:1002F0004468A34202D01B68002BEED143684B60D8
:100300004368086019604160F1E7000038B50446B1
:10031000FFF7FAFE214605460648FFF7D7FF637B45
:1003200043F0400363730020FFF7F6FE85F3118866
:1003300038BD00BF602D0020427BD20604D1036A85
:10034000013301D1FFF7E2BF704738B550F8103CD8
:100350000446A0F1180513B12846FFF75BFF14F817
:100360000B3C23F0040304F80B3C2846BDE838405E
:10037000FFF7E2BF70B50446FFF7C6FE0B4D064619
:100380002046FFF7A9FE21462846FFF79FFF637B23
:1003900055F8200C43F040036373031B5842584147
:1003A000FFF7BAFE86F3118870BD00BF602D0020F4
:1003B000114B1B6810B5EBB110498B68DA897F2AA5
:1003C00018D80F4A93F90E401268944212DB0D4A76
:1003D000126893420ED01A6A01320BD10A69824226
:1003E00006DC1846FFF7C6FFBDE81040FFF77ABEEF
:1003F000121A0A6110BD00BFE02B0020382D00202A
:10040000DC2B0020801C010070B504460D4616460A
:10041000FFF7D8FE637B43F00203637325B1A56049
:1004200021462846FFF752FF731C12D009484FF4AB
:10043000004500214FF4A022C5FB06010023EFF781
:100440005FFE0549421C04F11800BDE8704000F051
:1004500007BB70BDFFFF04004B03010010B5054B47
:1004600004469868FFF7D0FF2046BDE81040F1F73A
:10047000C5B900BF382D002038B5054600202C68CE
:10048000A54200D004B938BD2046FFF7E2FE204661
:10049000FFF752FF0120F2E7044B002103F128028D
:1004A000C3E90A220846FFF767BE00BF382D0020C7
:1004B00038B5124C124BA2681B689A420FD0FFF756
:1004C00023FE0546A068FFF707FEA16804F1280097
:1004D000FFF7FCFE0120FFF71FFE85F31188A268DD
:1004E000636A9A4209D04FF02003EFF3118083F33F
:1004F0001188BDE83840F1F781B938BD382D0020AA
:10050000801C0100014B9868704700BF382D002007
:1005100000F11003C0E90212C0E90000C0E9043391
:10052000704770B504464FF02003EFF3118683F354
:100530001188FFF780FE054670B1437BDB0604D1CE
:10054000036A013301D1FFF7E1FE0023AB663046B9
:10055000BDE87040FFF788BED4E902329A4218BF66
:100560000133A360022104F1100000F065FCEEE706
:1005700010B40A4604464FF02003EFF3118083F3D2
:100580001188A36833B1013BA36080F31188002078
:1005900010BC704721B980F311886FF00F00F7E7A6
:1005A000214610BCFFF75ABF10B5084C08494FF060
:1005B000FF334FF40072204600F038F904F11000C8
:1005C000044900F04DF8002010BD00BF682D002048
:1005D000E0420020B11C0100F8B505460F464FF07F
:1005E0002003EFF3118483F311880A484FF4004687
:1005F000002100234FF4A022C6FB0701EFF780FD86
:100600000549421C05F1180000F02AFA84F311880C
:10061000F8BD00BFFFFF04004B030100427BD20680
:1006200004D1036A013301D1FFF770BE70470000A7
:10063000EFF305800D2807D838B1044B586880F4D3
:100640000060C0F3C02070470120704700ED00E05B
:10065000024B9B68187B00F001007047382D00208A
:10066000704710B54FF02003EFF3118483F3118826
:10067000437B590702D484F3118810BD23F004038F
:100680004373FFF7CBFF2046BDE81040FFF7ECBDFA
:1006900030B587B004460E9D04950D9D03950C9DC5
:1006A00002950B9D01950A9D0095F1F75BFA044BAD
:1006B0009B6813B9236607B030BD1B6EFAE700BF15
:1006C000382D002070B586B0002605960E9E049643
:1006D0000D9E03960C9E02960B9E0F9D01960A9E00
:1006E00000960446FFF7D4FF6B1C03D02DB92046BB
:1006F000FFF7B7FF204606B070BD29462046FFF73A
:100700006BFFF7E7036D10B5044603B19847637BB1
:10071000DA060AD1226A013207D12046FFF752FDDC
:10072000637B43F00803637310BD9B0702D520462B
:10073000FFF770FD236A0133F2D004F1180000F0D6
:1007400051F9EDE7F0B5234F234D87B03E46BD424A
:1007500005F1300414D3214B9A68D37B013BD3734A
:100760004FF02003EFF3118583F311881A4CB44244
:1007700023D385F3118807B0BDE8F040FFF78CBDA7
:1007800054F8043C059354F8103C049354F8143C7A
:10079000039354F8183C029354F81C3C019354F80A
:1007A000203C009354E90A2354E90C01FFF770FF41
:1007B00054F8303CDD642546C9E7616A4B1C03D020
:1007C000206819B9FFF74DFF3034D0E7FFF704FF79
:1007D000FAE700BF9047002090470020382D002006
:1007E00003730023C3734FF0FF33427381730362BB
:1007F000704700B501F10803BFF35B8F53E8002F8A
:1008000042F0010C43E800CEBEF1000FF6D1BFF379
:100810005B8FD30703D45DF804EBFFF7DDBB5DF816
:1008200004FBA0F10C010069FFF7E3BF2DE9F041E3
:10083000054686B098460E46174605F11004FFF7A8
:10084000C3FB0020CDE90400CDE90208CDE900504A
:100850003146064B3A462046FFF734FF044920460E
:1008600006B0BDE8F041FFF7FBBE00BF0108000085
:10087000BA1C010000234FF0FF32C0E90031836051
:100880004261C3617047F8B504464FF02003EFF3AF
:10089000118583F31188C36923B985F311886FF03B
:1008A0001500F8BDBFF35B8F8368BFF35B8FDB0779
:1008B00000F1080632D5C26913680021002BECD084
:1008C0009C4226D12368576823F00300C1B9BC427B
:1008D000106000D15060236803F003032360002000
:1008E000E061BFF35B8F56E8003F23F0010346E869
:1008F0000032002AF7D1BFF35B8F85F31188D0E770
:100900000B6803F003030343BC420B6008BF516054
:10091000E1E71868194620F00303CFE70C3000F038
:1009200061F8DCE7F8B505460C4616464FF02003A3
:10093000EFF3118783F31188CB6923B183420BD086
:100940006FF02F000DE038B1E5616EB92146284601
:10095000FFF74FFF002004E02046FFF794FF002838
:10096000F2DA87F31188F8BD08484FF400450021FA
:100970004FF4A0220023C5FB0601EFF7C1FB044999
:10098000421C04F10C0000F06BF8E3E7FFFF0400E9
:1009900023080100034B1B680BB9F0F775BE00205C
:1009A000704700BFE42B00204FF02003EFF31180CD
:1009B00083F3118870470000036840B1084A526809
:1009C000904204D01BB19A6881680A449A604268D8
:1009D000136003685A604FF0FF338360704700BFB5
:1009E000C846002010B50246FFF7DEFF04469068B7
:1009F000431C03D01046FFF7DFFF002084F311886B
:100A000010BD0000134B1B7870B5002B14BF4FF0C6
:100A1000FF326FF00042FFF7C7FF0F4B1C689C428C
:100A200006460AD04CB1A568FFF7B4FF281A002883
:100A30000DDBA468FFF7AEFF221A86F31188074B7F
:100A40001B6913B19A42A8BF1A46104670BD002216
:100A5000F3E700BFE82B0020C8460020382D002017
:100A600070B5C16016460446FFF79EFF0546FFF7C6
:100A700091FF184B1A68012EACBF801901309A42C1
:100A8000A06001D05E6832B95A6862605A6823601B
:100A900014605C600BE09068A168884214DD411A24
:100AA00091605168C4E9002151680C6054601A6873
:100AB0009A4206D0944204D1FFF7A4FF0021F0F738
:100AC000AFFD85F3118870BD091A9642A160DBD095
:100AD0001268D8E7C84600202DE9F04B214D224E80
:100AE000224F04464FF00008FFF762FC2C60FFF72E
:100AF0005BFF3468B44281461CD094B1A1682B6876
:100B0000994215DC5B1A2B60D7E9002312EB010B2D
:100B100043EBE17CC4F808802046C7E900BCFFF73E
:100B20004BFF89F311883CB1E36820469847DEE724
:100B3000C91AA1600024F4E7FFF736FF0B49D1E999
:100B40000023064628682C60171843EBE078C1E9BB
:100B50000078FFF757FF2146F0F762FD86F3118812
:100B6000BDE8F08BE42B0020C8460020F02B0020CD
:100B700070B50E460446FFF717FF0546FFF742FF24
:100B8000431C01D0A04203DD31462046F0F748FD6A
:100B900085F3118870BD00002DE91848FFF704FFA8
:100BA0000446F0F771FD064BD3E9002312EB000B6E
:100BB00043F1000C5846614684F31188BDE818885B
:100BC000F02B002008B5FFF7E7FF08BD08B5FFF7D9
:100BD000F9FF4FF47A7164220023A0FB0101EFF7C3
:100BE000DFFA08BD38B5FFF7D7FF4FF47A73A0FBE3
:100BF000034503FB01556422002320462946EFF7F5
:100C0000CFFA38BD836870B505460E46D3B10022D1
:100C10001C685A60637B9A0714D5236A02331BD081
:100C20002046FFF716FB082E0CBF6FF003030023CE
:100C3000A366637BDB0605D1236A013302D120461C
:100C4000FFF764FBEB68C3F304321643002066F33E
:100C50001033A860EB6070BD6FF00A00FBE7F8B5D9
:100C60001746D0E90023904204460D4606D163683A
:100C70006B6063682C601D60656019E0002BF6D026
:100C80009B6839681868FFF76DFA0028EFD126686D
:100C9000B442ECD0002EEAD0B36838681968FFF788
:100CA00061FA30B17368C5E9006373681D607560EF
:100CB000F8BD63689E42DAD03668EBE7142330B59E
:100CC00003FB01000024002900DA30BD437B84606F
:100CD00003F00F03022B03D0042B01D0012B04D10E
:100CE000D0E900531D6005686B6082F311884FF0F6
:100CF0002003EFF3118283F3118801391438E2E7FE
:100D000030B5457B036161F303054573C168002479
:100D100064F31031C160C1F3074162F34101817393
:100D2000C289846064F38F02C28130BD2DE9F04F27
:100D3000404B85B09B6800930026012307468A46F6
:100D40009046019304464FF0FF35B146564510DBFF
:100D50004FF02003EFF3118683F31188019C002CE0
:100D60004BD1324629463846FFF7A8FF86F3118853
:100D70004CE04FF02003EFF3118B83F31188637B7A
:100D800003F00F03022B03D0042B04D0012B15D149
:100D90002269926801E0226912687AB1E268C4F8B7
:100DA0000890C2F304310B4363F31032E260CDF8D4
:100DB00004908BF3118801361434C7E7B8F1000FA3
:100DC000F7D0019A002AF4D0022B07D0042B0FD0C1
:100DD000012B09D16A462146206903E020696A4651
:100DE00021461030FFF73BFFC4F808D00135E0E79B
:100DF00020696A4621460830F4E700230193B8F1E0
:100E0000000F07D186F311886FF00A04204605B061
:100E1000BDE8F08F02A942463046CDE90211FFF746
:100E20001DFB04464FF02003EFF3118683F3118876
:100E300097E700BF382D00200368984207D0D3E918
:100E400000021060186842601846FFF7DBBE70476A
:100E500038B54FF02003EFF3118583F31188036851
:100E6000C16098424FF00101816004D185F311887F
:100E70000024204638BDD3E90002106018684260A3
:100E80001846FFF7BFFE04462846FFF7EDF9F0E7E6
:020E90007047A9
:020E9200FFFF60
:080E94003CF3FE7F01000000A9
:100E9C00000000005D14000000000000411B000079
:100EAC000C47002069F1000000000000411B00000D
:100EBC0000000000411B000000000000411B00006E
:100ECC0000000000B5EF000000000000411B000016
:100EDC0000000000411B000000000000411B00004E
:100EEC0000000000411B00000000000039A80000B9
:100EFC0000000000411B0000B02A002005FB000090
:100F0C0000000000411B000000000000411B00001D
:100F1C0000000000411B0000000000005115000003
:100F2C0000000000411B000000000000411B0000FD
:100F3C0000000000411B000000000000411B0000ED
:100F4C0000000000411B000000000000411B0000DD
:100F5C00000000006DA8000000000000411B000014
:100F6C0000000000411B000000000000411B0000BD
:100F7C0000000000411B000000000000411B0000AD
:100F8C0000000000411B000000000000411B00009D
:100F9C0000000000411B000000000000411B00008D
:100FAC0000000000411B000000000000411B00007D
:100FBC0000000000411B000000000000411B00006D
:100FCC0000000000411B000000000000411B00005D
:100FDC0018470020FDF4000000000000411B000039
:100FEC0000000000411B000000000000411B00003D
:100FFC0000000000411B000000000000411B00002D
:10100C0000000000411B000000000000411B00001C
:10101C0020110100E504000000000000A7120100EF
:10102C00E10F000000000000A71201007112000087
:10103C000000000084110100ED120000000000000F
:10104C008F110100ED120000000000009A11010048
:10105C009115000000000000A71201004D1D0000BA
:10106C0000000000A71201009D1E000000000000FF
:10107C00A7120100B5A9000000000000BF15010077
:10108C0001EC0000A81B0100B815010001EC0000E8
:10109C00A01B01006511010065F40000B01B0100EC
:1010AC00F610010049F800004C1C01005B11010016
:1010BC0081FA000000000000A712010085FD00006D
:1010CC0000000000A7120100A905010000000000AB
:1010DC000C0802170D010102090901010602091889
:1010EC0018030101090903030503554152545F31EB
:1010FC00000000001F000000D8310020781B010008
:10110C0000110100781B0100181101004C000000B7
:10111C00983000206863695F75617274000000008C
:10112C000200000034110100000000004C1101000D
:10113C0026000207000000205411010022000B11B0
:10114C00464C4153485F30005352414D5F3000458F
:10115C004E54524F50595F3000554152545F30003D
:10116C00B91300000000000000000000051300008F
:10117C008D12000000000000636C6B5F6B333273E8
:10118C00726300636C6B5F6D3136737263007379DD
:10119C00735F636C6F636B002A2A2A2A2A204255DC
:1011AC0053204641554C54202A2A2A2A2A0A002028
:1011BC002050726563697365206461746120627587
:1011CC0073206572726F720A0020204246415220D1
:1011DC00416464726573733A20307825780A002074
:1011EC0020496D7072656369736520646174612058
:1011FC00627573206572726F720A002020496E73DB
:10120C007472756374696F6E206275732065727287
:10121C006F720A0052657365727665642045786357
:10122C00657074696F6E20280053707572696F75E4
:10123C007320696E746572727570742028495251EE
:10124C0020002A2A2A2A2A20484152442046415565
:10125C004C54202A2A2A2A2A0A002020427573205C
:10126C006661756C74206F6E20766563746F722086
:10127C007461626C6520726561640A0020204661AD
:10128C00756C7420657363616C6174696F6E202872
:10129C007365652062656C6F77290A002A2A2A2AF1
:1012AC002A204465627567206D6F6E69746F7220B9
:1012BC00657863657074696F6E20286E6F74206931
:1012CC006D706C656D656E74656429202A2A2A2AF6
:1012DC002A0A002A2A2A2A2A202573202564292052
:1012EC002A2A2A2A2A0A002A2A2A2A2A204D505532
:1012FC00204641554C54202A2A2A2A2A0A0020200A
:10130C00537461636B696E67206572726F720A0049
:10131C002020556E737461636B696E672065727201
:10132C006F720A002020446174612041636365730D
:10133C00732056696F6C6174696F6E0A0020204DC2
:10134C004D46415220416464726573733A20307883
:10135C0025780A002020496E737472756374696F66
:10136C006E204163636573732056696F6C61746999
:10137C006F6E0A002020466C6F6174696E672D7069
:10138C006F696E74206C617A792073746174652056
:10139C00707265736572766174696F6E20657272B6
:1013AC006F720A002A2A2A2A2A20555341474520BF
:1013BC004641554C54202A2A2A2A2A0A0020204425
:1013CC0069766973696F6E206279207A65726F0A2B
:1013DC00002020556E616C69676E6564206D656DCB
:1013EC006F7279206163636573730A0020204E6FFE
:1013FC0020636F70726F636573736F7220696E73A5
:10140C007472756374696F6E730A002020496C6C7A
:10141C006567616C206C6F6164206F662045584372
:10142C005F52455455524E20696E746F2050430ADA
:10143C00002020496C6C6567616C20757365206FAA
:10144C00662074686520455053520A002020417470
:10145C0074656D707420746F206578656375746540
:10146C0020756E646566696E656420696E7374724E
:10147C00756374696F6E0A002A2A2A2A2A20486129
:10148C0072647761726520657863657074696F6EDC
:10149C00202A2A2A2A2A0A002A2A2A2A204B65725A
:1014AC006E656C20416C6C6F636174696F6E204665
:1014BC0061696C75726521202A2A2A2A0A002A2A57
:1014CC002A2A2A204B65726E656C204F4F5053218F
:1014DC00202A2A2A2A2A0A002A2A2A2A2A204B6562
:1014EC00726E656C2050616E696321202A2A2A2A4B
:1014FC002A0A002A2A2A2A20556E6B6E6F776E20D4
:10150C00466174616C204572726F722025642120D3
:10151C002A2A2A2A0A0043757272656E742074682E
:10152C0072656164204944203D2025700A4661752E
:10153C006C74696E6720696E737472756374696F0D
:10154C006E2061646472657373203D203078257859
:10155C000A0049535200657373656E7469616C209F
:10156C0074687265616400466174616C20666175B3
:10157C006C7420696E20257321205370696E6E691E
:10158C006E672E2E2E0A00466174616C20666175A2
:10159C006C7420696E2074687265616420257021FA
:1015AC002041626F7274696E672E0A004750494F72
:1015BC005F30004750494F5F310000000D000000C4
:1015CC0001000000180000000100000006000000EF
:1015DC00000000001A0000000000000008000000DD
:1015EC00000000000A000000000000000E000000D7
:1015FC00000000000C0000000100000005000000CD
:10160C0000000000070000000000000001000000C6
:10161C0000000000030000000000000009000000B2
:10162C0000000000781B0100381601004C0000007F
:10163C00FC320020443A2F576F726B2F6E6F72641E
:10164C0069632F6E63735F7461672F7A6570687955
:10165C00722F7375627379732F626C7565746F6F0B
:10166C0074682F636F6E74726F6C6C65722F746913
:10167C00636B65722F7469636B65722E6300F40182
:10168C00FA00960064004B0032001E001400443A2D
:10169C002F576F726B2F6E6F726469632F6E63734B
:1016AC005F7461672F7A65706879722F73756273D6
:1016BC0079732F626C7565746F6F74682F636F6EBE
:1016CC0074726F6C6C65722F6C6C5F73772F6374B4
:1016DC00726C2E6300443A2F576F726B2F6E6F72C1
:1016EC006469632F6E63735F7461672F7A657068CA
:1016FC0079722F7375627379732F626C7565746F61
:10170C006F74682F636F6E74726F6C6C65722F6C74
:10171C006C5F73772F6C6C2E6300000087170100D1
:10172C00000000000000000005AB0000C5A900008F
:10173C00443A2F576F726B2F6E6F726469632F6E02
:10174C0063735F7461672F7A65706879722F737534
:10175C00627379732F626C7565746F6F74682F6325
:10176C006F6E74726F6C6C65722F6863692F68632F
:10177C00695F6472697665722E6300436F6E747272
:10178C006F6C6C6572000101010100020202020221
:10179C00027075626C69630072616E646F6D0070CB
:1017AC0075626C69632069640072616E646F6D2090
:1017BC0069640030782530327800253032583A256B
:1017CC003032583A253032583A253032583A253092
:1017DC0032583A25303258202825732900443A2FA4
:1017EC00576F726B2F6E6F726469632F6E63735FCA
:1017FC007461672F7A65706879722F73756273796B
:10180C00732F626C7565746F6F74682F636F6E7471
:10181C00726F6C6C65722F6863692F6863692E63D5
:10182C00005A6570687972204F532076312E31330F
:10183C002E393900000000000000000000000000FC
:10184C00000000000000000000000000000000008C
:10185C00000000000000000000000000000000007C
:10186C00000000000000000000000000000000006C
:10187C00000000000000000000000000000000005C
:10188C00000000000000000000000000000000004C
:10189C00000000000000000000000000000000003C
:1018AC00000000000000000000000000000000002C
:1018BC00000000000000000000000000000000001C
:1018CC00000000000000000000000000000000000C
:1018DC0000000000000000000000000000000000FC
:1018EC0000000000000000000000000000000000EC
:1018FC0000000000000000000000000000000000DC
:10190C0000000000000000000000000000000000CB
:10191C0000000000000000000000000000000000BB
:10192C0000000000000000000000000000000000AB
:10193C00000000FFC1FBE84C90728BE7B351896348
:10194C00AB232302841872AA612F3B51A8E53749B7
:10195C00FBC9CA0C18532CFD45E39AE6F15DB0B6F1
:10196C001BB4BE2A50EAE90E9C4B5E5724CCA1B79F
:10197C0059B887FFE07D742648B9C5F3D9A8C4B11E
:10198C00D5911101420C39D5B0979D28D4F29BA466
:10199C00FD6465068C2996FEA2714DF3F82E58DB7A
:1019AC000D5A5F1528F57407CE25AF2B12E6D0DB48
:1019BC002CDCC37FF03E3A13A4DCE2F96C54E2D881
:1019CC00EAC8880021869C6AD8CB4E146AF94DD29D
:1019DC007EB23203C6144B7FD1B8A6797C17ACED1E
:1019EC0006ADAF0A947ABA03E792D7150973E86D7E
:1019FC0016EEE13F781F9D09526EF17C362A716C10
:101A0C007564448010434E35EC65270AB5FC266995
:101A1C003F599901638AA5BF685CD33CBE0BD6764F
:101A2C0083D657054A3DDD8173C9EB8A8439F43678
:101A3C000BF7000029417671443A2F576F726B2FC8
:101A4C006E6F726469632F6E63735F7461672F7A54
:101A5C0065706879722F7375627379732F626C7508
:101A6C0065746F6F74682F636F6E74726F6C6C65D6
:101A7C00722F6C6C5F73772F6C6C5F66696C74651E
:101A8C00722E6300443A2F576F726B2F6E6F726415
:101A9C0069632F6E63735F7461672F7A6570687901
:101AAC00722F7375627379732F626C7565746F6FB7
:101ABC0074682F636F6E74726F6C6C65722F6861D3
:101ACC006C2F6E7266352F636E74722E6300443AFF
:101ADC002F576F726B2F6E6F726469632F6E637307
:101AEC005F7461672F7A65706879722F7375627392
:101AFC0079732F626C7565746F6F74682F636F6E7A
:101B0C0074726F6C6C65722F68616C2F6E726635B7
:101B1C002F6D6179666C792E630003040005443ADD
:101B2C002F576F726B2F6E6F726469632F6E6373B6
:101B3C005F7461672F7A65706879722F7375627341
:101B4C0079732F626C7565746F6F74682F636F6E29
:101B5C0074726F6C6C65722F68616C2F6E72663567
:101B6C002F7469636B65722E630000002DE9000011
:101B7C00000000000DE9000049EE00002FEB000012
:101B8C006BEB00009BEB000075F0000071EF0000A8
:101B9C000000000000000050000000000003005096
:101BAC000100000001000000F1F30000B1F300009F
:101BBC00D5F00000D5F10000E9F000001DF40000A4
:101BCC007DF3000095F1000081F1000019F1000097
:101BDC00F9F0000009F1000019F1000021F10000FA
:101BEC0031F1000041F1000041F3000051F100001F
